:10000000D0620020B1270000D5F301009D27000039
:100010009D2700009D2700009D2700009D270000D0
:10002000000000000000000000000000E9270000C0
:100030009D27000000000000B12900009D2700005E
:10004000092A0000092A0000092A0000092A0000E4
:10005000092A0000092A0000092A0000092A0000D4
:10006000092A0000092A0000092A0000092A0000C4
:10007000092A0000092A0000092A0000092A0000B4
:10026000092A0000092A00007D5F0100092A000018
:10027000092A0000092A0000092A0000092A0000B2
:10028000092A0000092A0000092A0000092A0000A2
:10029000092A0000092A0000092A0000092A000092
:1002A000092A0000092A0000092A0000092A000082
:1004800053B94AB9002908BF00281CBF4FF0FF31FB
:100490004FF0FF3000F00CB8ADF1080C6DE904CE60
:1004A00023F080FADDF804E0DDE9022304B07047B0
:1004B000704700BF034611F8012B03F8012B002AF7
:1004C000F9D17047034613F8012B002AFBD1181A03
:1004D00001387047000000000022F0B585B01146D9
:1004E00040F6034002AF03F095FE044600285AD1BF
:1004F00003F07EFC214641F203003A1D03F08AFE20
:10050000044600284FD17A68294DD16805F1780357
:10051000D1F80100D1F8051003C3104602F002FE25
:10052000214641F201003A1D03F074FE0446002802
:1005300039D17868C3685A7885F86F205A88A5F849
:1005400072201A7985F87020B3F80720A5F8742076
:10055000B3F80530A5F8763002F0E4FD214641F20B
:1005600002003A1D03F056FE0446E0B9D7F804C075
:1005700005F18006DCF80C20531C41323446186823
:100580005968083303C493422646F7D1604602F007
:10059000C9FD95F87C305A0610D4064906481FF06C
:1005A0009EF96FF0120420460C37BD46F0BD00BF27
:1005B000000000201E6F020088480200002142F265
:1005C00003003A1D03F026FE04460028EBD17A68AA
:1005D000AB4BD168D1F80100D1F8051003C3104628
:1005E00002F0A0FD214642F202003A1D03F012FE85
:1005F00004460028D7D17E68F468B4F801309AB276
:1006000092B1E27882B1A5F8FC30E378032B06D0F2
:100610000322022100929B489B4A1EF0BBFDE27818
:100620009A48114621F09EFD304602F07BFD1F23C3
:1006300095F87C40A5F8103114F0200419D14FF042
:10064000FF304FF0FF3103F0F3FB0646002800F0C7
:10065000038102210C301EF0C3FF012344702246A7
:100660000370314640F66D4003F0D4FD0446002887
:1006700099D195F89C301B0712D5002142F21C003D
:100680003A1D03F0C7FD044600288CD17868C36882
:10069000D3F80120D3F80530C5E9382302F042FD34
:1006A00095F8D8309E0623D53846B91C03F04EFE87
:1006B000044600287FF477AF4FF0FF304FF0FF3152
:1006C00003F0B6FB0646002800F0C68004210C307B
:1006D0001EF086FF3B88224603807B88314643809C
:1006E00042F2240003F096FD044600287FF45BAF3D
:1006F00095F8D8305C0610D5002142F22A003A1D48
:1007000003F088FD044600287FF44DAF7868C36885
:100710005B7885F8123102F005FD4FF0FF304FF0A5
:10072000FF3103F085FB0446002800F09580082186
:100730000C301EF055FF95F8D81040F2022311F04E
:10074000400F08BF0323024688074CBF43F02C0329
:1007500043F00C038E0695F8D96048BF43F0400380
:1007600006F009060EB143F4006301F0010143EA0B
:10077000011000211FF0D4F82146002242F20100AE
:1007800003F048FD044600287FF40DAF95F87C3057
:10079000B5F8FC10980662D4C9B941F205003A1DBB
:1007A00003F038FD044600287FF4FDAEB5F8FC30B8
:1007B0007C684BB9E368B3F80120A5F8FC209A885F
:1007C0003248114621F0CEFC204602F0ABFC4FF03F
:1007D000FF304FF0FF3103F02BFB044600283BD0E5
:1007E00008210C301EF0FCFE95F8D8300246D907DF
:1007F0003ED44FF0005126481FF092F821460022C7
:1008000040F6014003F006FD044600287FF4CBAE1D
:1008100001463A1D4FF6014003F0FCFC00283DD094
:100820001C4A022117481EF0A4FCEB79002B00F0B3
:10083000D9802E78002E40F0D58095F8C1309B06E7
:1008400040F1DF804FF0FF304FF0FF3103F0F0FA5E
:100850000446002840F0B2806FF06804A3E6002947
:10086000B5D10D4907481FF03AF86FF004049AE635
:1008700001A1D1E90001BFE79088000200800020BB
:10088000D800002088480200426F020000010020CA
:1008900010880002AB6F0200886F02007B686E4612
:1008A000DC688AB0B4F80130042B96BF564A574A28
:1008B00052F8232009934FF400735549ADF82830BE
:1008C000544BCDE9071202AA42F8103F4FF41351DE
:1008D00051481EF0FCFFB4F80120B546022AB4F8D6
:1008E000033001D1052B47D9484A6E468AB0099397
:1008F0004FF400734949ADF82830464BCDE9071253
:1009000002AA42F8103F4FF4135143481EF0DFFF94
:10091000B5466379A679032B98BF414AB4F807001E
:10092000D4F8091098BF52F823206C4688BF374A84
:100930008CB0CDE909364FF40073DFF8E8C0ADF8AC
:100940003430394BCDE907C202AACDE90B0142F898
:10095000103F4FF4735130481EF0B9FFA546786838
:1009600002F0E0FB00214FF602403A1D03F052FC7A
:10097000044628B12D4A54E72D4A52F82320B4E703
:100980007868C368B3F80130A5F8C13002F0CAFB3B
:1009900095F8C1305A077FF548AF21464FF603401E
:1009A0003A1D03F037FC08B1224A3AE77868C36879
:1009B0005B7885F8C03002F0B5FB36E706210C30D5
:1009C0001EF00EFED5F80130214603601A4B324668
:1009D0009B8883804FF6064003F01CFC04460028E9
:1009E0007FF4E1AD04F0AAFB044600287FF4DBAD00
:1009F00006F004F8044600287FF4D5AD03F0F4FABD
:100A0000D1E56FF08504CEE5604C02005D6D02001B
:100A1000CF6F02000400000188480200E86F020066
:100A2000384C020000700200070000012D70020027
:100A3000484C02005670020001000020044B054A99
:100A40000548012914BF114619461DF03ABF00BFE1
:100A5000366002003E6002004760020010B50C469E
:100A600021B1BDE8104007481DF02BBF1FF0A5F9CC
:100A7000054B1860054B06481C60BDE810401DF092
:100A800020BF00BF5C600200FC180020F8180020A6
:100A9000776002002DE9F0411D461F4E074633687E
:100AA000144605EB0308B8F1F40F96B007D81B48BD
:100AB0002A462146184422F0C2FEC6F8008035B30B
:100AC0002C4414F8013C0A2B21D1316814480DF153
:100AD00018081DF0F6FE402140463368114A1DF00B
:100AE0008DF9041E11DD00211822684622F0CEFE89
:100AF0003F2C204628BF3F200B4BADF80C00694629
:100B00003846CDE9013808F0FFF800233360284665
:100B100016B0BDE8F08100BFF81800204A38002068
:100B20008260020096600200184A020001460748EF
:100B3000036982681B7803F001038B4218BFD368F6
:100B40004FF0010108BF1369184700BF983D02002C
:100B500070B50C4C0D46206818B105F091F90023D2
:100B600023600024084B294608481C601DF0A9FE9C
:100B70002046FFF7DBFFBDE8704000220023044859
:100B80001AF0AEBEFC180020F8180020C760020062
:100B90003008002030B5104D89B003AC0FCD0FC424
:100BA0002B680E492360012402220D4B009403A8F8
:100BB00004F082FB014628B10A481DF082FE0320A2
:100BC0001DF085FC2046FFF7B1FF074907481DF0DF
:100BD00078FE09B030BD00BF50490200E049020074
:100BE000D8490200DD600200F560020006610200E3
:100BF00010B517481DF065FE164802698168136834
:100C000043F0010313600B68134A00219847044620
:100C100050B90120FFF78AFF41F68560002121F0DD
:100C2000A5FC2046FFF782FF002003F0DBFC044612
:100C300030B1014609481DF044FE02201DF047FC7A
:100C40000749084821F077FBFFF7A4FF204610BDB5
:100C500019610200983D020001000A00346102009F
:100C600007E50100300800202DE9F84F884600AF65
:100C7000002974D004680E1F361BF50826F00706FD
:100C800004EB060999F802A01AF0010A16D1EB4606
:100C900088B0344B6A46CDE90531032342F8103F52
:100CA0004FF4C2515346304800F0A4FFDD468AF3AA
:100CB0001188BFF36F8F0423184602DF29462046B0
:100CC0001DF023FC284434F83030C01A854217D078
:100CD000EA4688B0254B6A46CDE90538032342F839
:100CE000103F00234FF4C2511F4800F083FF002340
:100CF000D54683F31188BFF36F8F0423184602DFB4
:100D0000B9F80230294623F00103A9F80230204641
:100D10001DF0FBFB05EB000804EBC8039B78DA072A
:100D200008D4414620461DF034FC42462946204660
:100D30001DF071FCA65BAE1B04EBC6039B78DB07C2
:100D400009D4314620461DF024FC2A46314620466F
:100D50001DF061FC3546294620461DF0DBFBBD46F3
:100D6000BDE8F88F97610200104902006E61020031
:100D700008B502481DF0A5FD002008BDC4610200B1
:100D80000E4A0346904204D30D4A904201D20120FC
:100D900070470C4A22B1934202D30B4A9342F6D3D6
:100DA0000A4A42B10A48834234BF012000209342DC
:100DB00038BF002070471046704700BF683C0200F3
:100DC0005089020000000000000000000000000048
:100DD000000000002DE9F04F984693B083070546C8
:100DE0000E46069240F0B881002843D101F0070674
:100DF000341DC6F1080600274FF00409069BBB46C8
:100E000003F004030393069B4FF0FF31C3F3C203C7
:100E10000133059308F1FF3302934B46C5F10802F5
:100E2000DDF870A00497019707920DB1C4F8008017
:100E30000598069A002802F0020207DC4046CDE938
:100E40000832FFF79DFFDDE9083220B1002A00F0EB
:100E5000E98001200222A4EB050C4FEA9C0C12B1A0
:100E6000BCF17F0F03D8019A0F2A40F2CA806FF0BD
:100E7000150074E0072970D9041DBCE77A2A05D84B
:100E8000692A06D8392A55D81F2A41D84FF0000BB5
:100E900084E06A3A102AF9D801A050F822F000BF85
:100EA000970F00008D0E00009D0F00008D0E0000BA
:100EB000C70F0000650F0000C70F00008D0E000077
:100EC0008D0E0000D30F0000E50E0000650F00003E
:100ED0008D0E00008D0E0000650F00008D0E0000CD
:100EE000E50E00004FF0040957E001204C3AD2B261
:100EF00000FA02F212F0626F23D19948024231D116
:100F00009848024214BF4FF0010B4FF0000B45E030
:100F10004FF0010CA2F12000C0B20CFA00F0DFF893
:100F200048C210EA0C0039D12A2A54D0252AADD162
:100F30000139ABE74B2AD8D8412A02D0453A022AD8
:100F4000A4D80AF1070A07342AF0070A24F0070494
:100F5000E5B1079B2344B34214D96FF01B0013B0D3
:100F6000BDE8F08F029A12F8012C6C2A46D10022BB
:100F7000029B934613F8023C6C2B27D14FF00809D3
:100F80004B4629E0DAE90023C4E900234FF0000BC7
:100F90000AF1080A08344FF008094B46029810F885
:100FA000012F0290002A6CD0BBF1000F7FF466AFD6
:100FB000252A01F1010001BF01464FF0010B4FF05E
:100FC00004090423EAE700224FF0000B4FF0040964
:100FD000D6E75A46F8E70246013C4C44B4FBF9F424
:100FE00009FB04F41DB1581B2044B042B5D87AB3B4
:100FF000059A5AF8048B013A059216E700229346A7
:10100000EAE7ADB1019A48326A4402F820CC02F80E
:10101000101C48B16CF07F0C02F820CC0137019A0B
:10102000013201920434B9E7049A01320492F6E7DE
:1010300008B10136F3E7039A0236002AEFD14046A1
:10104000CDE90813FFF73EFADDE908130644E6E7A9
:10105000042B08D10AF1040015B1DAF8002022604F
:10106000824604349AE70AF1070323F0070303F1E9
:10107000080A1DB1D3E90023C4E90023082308347A
:101080008CE7631BB3F5806FBFF4F1AE1DB9A6F119
:101090000804E01863E79B082A602B70039BC3B128
:1010A000049BEB70AF7037B100220AABC5F1010CA5
:1010B0000199914210D14FF0000AC5F101030DF1E1
:1010C000280902930DF1380B019B534516D1601B83
:1010D00045E7049B6B70E5E793F900E01878BEF1F3
:1010E000000F08DA0CEB040EB6453FF636AF00F001
:1010F0007F0004F8010B01330132D9E71FB199F9E0
:101100000020002A17DB039BD3B11AF80B2004F848
:10111000012B0022029B18191044B0423FF61DAF6C
:1011200099F80000414604F8010B2046049222F091
:1011300086FB049A14440AF1010A09F10109C3E784
:1011400099F80020039B55F8228045F8223040464C
:10115000FFF7B8F9421CDDE76FF00D00FFE600BFB6
:1011600000108021010000100968FF032DE9F04FF5
:1011700099B000AF04468B46C7E90C32D7F8889087
:1011800090F8028041B94578007808EB800020444F
:101190005D4520D8A0EB040B09F00103BB61E378A7
:1011A000B8F1000F0CBF4FF0000A09F0010AFB6212
:1011B00013B119F0020F17D1BAF1000F14D17B6BE4
:1011C0001BB1594620463A6B98475D46284664371E
:1011D000BD46BDE8F08F461C3046FFF773F901307D
:1011E00030440BF1010BD3E7C9F3C0033B61237813
:1011F0007B629B00FB606368FB617B6A04EB83019D
:101200007B6B002B7BD15D468844BAF1000F1ED06A
:101210000E46D7F834A0DFF87CB216F8013B54F83C
:101220002300002808BF5846FFF74CF9D7F88C3048
:1012300001304BB1D7F890309A453EBFD7F88C308B
:1012400023F81A000AF1010AB0450544E5D119F066
:10125000050F0CBF4FF0020B4FF0010B002609F0F9
:101260000209FB6A9E42B1D23B6908F1020803B34E
:1012700018F8021CF8691DF003FBD0B1C7F834D090
:101280008AB0854B6A460593FB69CDE906314FF478
:101290000073ADF82030814B42F8103F00234FF42B
:1012A00012517F4800F0A6FCD7F834D0023D013639
:1012B000D7E718F8013C54F823100846FFF760FD03
:1012C00020B1BB692BB9A5EB0B05F0E7B9F1000F15
:1012D000EDD07048002918BF0846FFF7F3F8D7F89B
:1012E0008C3053B1D7F890309A453FBFD7F88C2057
:1012F000431C22F81A300AF1010A0544D7E7BAF173
:10130000000F0FD04346102B28BF10230026BB62CE
:1013100097F828A007F14000BA6A396222F08FFAE4
:10132000396A09E0B8F1000F02D019F0040F5DD15D
:101330000026B246C7F8288001EB08037B619D1C9C
:1013400000233B6209F00203BB6009F004037B60E9
:101350003B6AFA6A934253D3637819F0020F09F09B
:1013600005090AEB03013B6214BF00237308B9F1BE
:10137000040F0CBF324600226170A270E370204659
:101380003A6BF9687B6B9847051EFFF61FAF7B6AC7
:10139000314623703B6A3A6B6370FB6A84F80280C3
:1013A000E37007F150007B6B9847061EC0F2B480D3
:1013B000FA6AFB68F86A03EB4203ABEB0301BB6A12
:1013C0003A6BC91A7B6903EB40007B6B9847002896
:1013D000C0F2A4804FF000092E443518D14561D3E6
:1013E00000213A6B08467B6B9847EFE64346102B8B
:1013F00028BF1023BB6297F8286007F150008BE7E5
:101400003B6915F8021C1BB1F8691DF039FA30BBB5
:1014100015F8013C54F823003B60FFF7B1FC3B6832
:1014200010B3BA6972B1BAF10F0F18D80AF12801D6
:1014300007F138000AF10102014401F8203C5FFA8B
:1014400082FA0CE07A6852B10F2E08D806F1280112
:1014500007F13800721C0E1806F8103CD6B23B6A31
:10146000023501333B6273E7BA68002ADBD10F2EE5
:10147000F5D806F1280007F1380C6044721C00F81A
:10148000101C07F16001023651FA82F2F6B202F83E
:10149000103CE4E7F2610200F9610200040000017F
:1014A000C048020007F1400313F8093054F823B094
:1014B00087F83F30D7F88C301BB1D7F8903099457A
:1014C00024D34FF0000801213A6B7B6B07F13F00FA
:1014D0009847061E20DB124BBBF1000F08BF9B464E
:1014E000B8F1000F06D15846FEF7ECFF00F10108F5
:1014F0001FFA88F8414658463A6B7B6B984700289C
:1015000009DB2E44351809F1010967E7D7F88C305B
:1015100033F81980D7E70646354657E6054655E6BF
:10152000F2610200014B1860704700BF24020020E6
:101530002DE9F047038B0446180716460CD5012900
:101540000CBF43F0100343F02003238386F311887C
:10155000BFF36F8FBDE8F087022903F0070700F0A3
:10156000A380D4F81490218BB9F1000F2DDA002557
:10157000D4F80080C4E9005521F0070141F00101D1
:10158000218301F0070ABA4502D0A368002B5DD180
:10159000B8F1000F01D1002D76D0002341F00801F1
:1015A000218386F31188BFF36F8F002B50D0A16881
:1015B00000294DD00E684B46524620464F68B8472A
:1015C000002E45D031463668F5E701F007035A1F73
:1015D000012A4FF000051ED821F00701062BD4F890
:1015E000008089B2C4E900550BD1B8F1000F06D0D4
:1015F0004346628B013262831B68002BF9D141F0B4
:101600000201204621831DF005FC00250028B8D0EA
:1016100041F02001B4E7042BA846B2D121F0070124
:1016200089B2204621831DF0F5FBEFE7218B23696A
:1016300021F007015D6841F0040146E0218B236938
:1016400021F007019D6841F005013EE00123A5E777
:10165000B8F1000F08D041464B4652462046D8F814
:1016600000801DF006FCF3E715B120461A49A84793
:10167000EFF31186202383F31288BFF36F8F218B42
:1016800021F0080189B22183CA0605D521F0100393
:10169000238301F0070764E78B067FF557AF21F03E
:1016A0002003238301F0070720461DF0B3FB042825
:1016B000BCD00528C2D003287FF448AF2369218B12
:1016C0001D6821F0070141F006014FF0000889B2C2
:1016D000C146218355E700BF9DEE01002DE9F0478B
:1016E000044607464FF00109DFF8488094FAA4F554
:1016F000B5FA85F509FA05FA2E0108EB05152B7BDD
:1017000024EA0A0463B158F806301B696BB94644F1
:10171000736804222846196827EA0A071DF0B8FCF6
:10172000002CE3D13846BDE8F087284698470028CA
:10173000F6D1ECE74049020010B5002288B00E490E
:101740000E4820F09EFF002200230024CDE906234E
:101750000E234FF44072CDE90334CDE90144084B28
:101760000849009408481AF05DF90849064820F035
:1017700038FE204608B010BD91170000E80C00208C
:10178000A51A0000883A002060080020B862020014
:10179000014819F0E5BD00BF000700202DE9F04722
:1017A0008146214888461DF058FC0646002838D15D
:1017B000054601271D4CDFF878A0544505D3B9F143
:1017C000000F2BD12846BDE8F087237B7BB123682F
:1017D000DB680BB12046984763689F7123681B69DB
:1017E00043B963680422204619681DF051FC013694
:1017F0001034E2E7204698470028F2D007FA06F3B3
:101800001D43F4E72846FFF769FF0546B8F1000FCE
:1018100004D040F23910002120F0A8FE002DF1D1B3
:10182000D0E70025CEE700BF101900204049020094
:1018300050490200014B53F8200070477C4A0200D7
:1018400008B530B1044A1060084600F03DFC0020A5
:1018500008BD6FF01500FBE72802002010B5044C0E
:10186000237813B9034819F07BFD0123237010BDC1
:101870003E3900200007002010B5044609481DF03D
:10188000ECFB3CB1084BD3E8EF1F0139C3E8E21F82
:10189000002AF8D105481AF091FEBDE8104004482E
:1018A00019F05EBD081900200C190020E80C00207A
:1018B000000700200022044BD3E8EF0FC3E8E12F1C
:1018C0000029F9D1704700BF0819002070B5FFF753
:1018D000F1FF0646074C084DAC4200D370BD63686B
:1018E0005B792BB123685B6813B13146204698477A
:1018F0001034F1E7404902005049020010B5044C91
:10190000044920461DF0FBF8034B1C6010BD00BFCE
:101910005C060020684A02000019002010B500246F
:101920000B4B0C491C700C4B0C481C600C4B1C6086
:10193000FFF786FFFFF7E2FF0A4B0B498B4200D30C
:1019400010BD586822110132027110331034F5E7CE
:101950003F39002040420F000819002057F00100D5
:101960000C190020404902005049020001460022A3
:10197000002301481DF0E4B85C06002001481DF07A
:101980007CB900BF5C060020024B014618681DF0C0
:10199000D3B900BF0019002001481DF008BA00BFEC
:1019A0005C060020F8B5284B1B78002B4AD0FFF7C7
:1019B000E5FF0546002842D1244B254C1B68002B2F
:1019C00019DD20F017FE4FF47A76A0FB060747F6E4
:1019D0001222002306FB0171FEF752FDD4E900320A
:1019E000C01A40F2E93361EB0201984271F1000143
:1019F00001D3FFF76BFFD4E9003213F57A7342F19C
:101A00000002C4E90032EDB1BDE8F840FFF7C4BF01
:101A100063685B7923B12368294620461B68984791
:101A20001034B442F4D32846FFF7AEFF094BD3E895
:101A3000EF1F0139C3E8E21F002ABDD0F7E7064CCB
:101A4000064EEEE70020F8BD3E39002008190020C0
:101A5000E00C00200C19002040490200504902000F
:101A600070B50D4D297861B90120FFF797FE0B4C39
:101A70000B4EB44206D3FFF795FF0028FBD101239C
:101A80002B7070BD63685B791BB1236820469B682F
:101A900098471034EDE700BF3F390020404902006D
:101AA0005049020000212DE9F8430846FFF776FE71
:101AB000044638B340F21B6600271AF0CDFA1A4BE1
:101AC000186030B1194B1B68092B02DD184819F05A
:101AD00047FC0025DFF85C9044B12046FFF7FEFD8F
:101AE000044618B94FF0FF364FF0FF37FFF75AFFA3
:101AF000804628B9B5B90E4832463B4619F064FC19
:101B00004546E9E74FF0FF364FF0FF37D5E72B6842
:101B10009B691BB1002228461146984710354D4558
:101B2000F5D3E8E7044DFAE7041900200C1900206A
:101B300000070020504902004049020013B5184830
:101B40001DF08BFA174B1B7873B1EFF31184202330
:101B500083F31288BFF36F8FFFF724FF84F311889C
:101B6000BFF36F8F02B010BD0F4B1B68002BF9D075
:101B700050B9002200230D48CDE9002347F6122278
:101B800000231AF0F5FCEDE70928EBD107481AF01D
:101B900015FD074802B0BDE8104019F0E1BB00BFD9
:101BA0000C1900203F39002004190020E80C002007
:101BB0000007002010B5064B04461B6898472146D5
:101BC000A06004481DF03AF8BDE81040FFF7B6BF2A
:101BD000280200205C060020044A054B9B1AB1EB4A
:101BE000D30F34BF52F83100002070472048020064
:101BF000404902002DE9F04F8FB0C1F34A2604AFEF
:101C000090460D46B8607B600C0D002E5FD04FF003
:101C100000090A234FF0040B07F1140AFE60C7E91C
:101C20000799C7F824900093CDF808B0CDF804A028
:101C300007F11C034A464046F968FFF797FAB0F5EA
:101C4000006F03461CD36C46D8F804308AB0244990
:101C500004AACDE9091340F2FF730B934FF400730C
:101C6000ADF830301F4B42F8103F4FF412514B4645
:101C70001D48FFF7BFFFA5462C37BD46BDE8F08FD6
:101C8000C0F30A0604F11700184420F0070080088A
:101C90003B60FFF76BFE044680B13B6800F110012A
:101CA000C7E908390A23F961CDE901AB0093404641
:101CB0000E4AF96807F11C03FFF758FA66F353253B
:101CC0002A4620467B68B9681DF002FAD4E704F181
:101CD000170020F007008008FFF748FE0446EDE7F4
:101CE000CD62020004000001D8480200A3F0010008
:101CF0002DE9F04F87B00546DDE91069DDE912787E
:101D00008A4614469B46BFB110213B464A460020F6
:101D1000CDF80080CDF81480FFF75CF8B0F5006FC7
:101D200001460BD340F2FF730221184A184807B04E
:101D3000BDE8F04F1DF025BA3946384604F00703D8
:101D400005F00704E40044EA831444EA402444EA2A
:101D5000065406F11700084420F00700800803919C
:101D6000FFF704FE054640B13FB13B464A460399A2
:101D7000CDF800801030FFF72DF85B462246514623
:101D8000284607B0BDE8F04F1DF0A2B90C63020071
:101D9000D8480200406820B1034BC01A40F3CF007E
:101DA00070474FF0FF307047204802000EB403B573
:101DB00003AB53F8042B01460448019301F072F879
:101DC00002B05DF804EB03B0704700BFE1F1010021
:101DD000CA0605D48B064CBF02490349FFF7E6BF8C
:101DE000704700BF45630200446302002DE9F04FD5
:101DF0008BB0CDE90623DDE918A9179B9DF8588023
:101E000004460D461A9F0593B8F1000F00F0DA80E2
:101E1000814B07F0020B13F80830089307F4807326
:101E200009931DF033F90246002800F09780204600
:101E30007A49FFF7BBFF0646BBF1000F09D017F048
:101E4000440F40F08D802A4620467549FFF7AEFFCB
:101E5000064407F0010353B1724B204653F8282083
:101E6000714B7249002A08BF1A46FFF79FFF17F40B
:101E7000807307F00803079D18BF0025002B00F0B2
:101E80009C806B4B204653F828206A49FFF78EFF51
:101E90008346069B2BB11A4620466749FFF786FF0B
:101EA000834475B1089B002B00F08A806349644B22
:101EB000B8F1040F18BF19462A462046FFF776FFEF
:101EC00083446048B344059B1BB122465E491CF025
:101ED000A6FCB9F1000F2DD04E463946102E2046F3
:101EE00028BF10260025FFF773FFAB4571DC0025E6
:101EF0002B4620461AF803205449FFF757FF0135B7
:101F0000102D6CD1002520465149FFF74FFF2B467D
:101F10001AF803202046A2F120035F2B28BF2E22AF
:101F20004C49FFF743FF0135102D66D1B9EB060987
:101F3000B244D1D1B8F1000F0AD0FB0704D5204636
:101F4000394A3A49FFF732FF39462046FFF740FF4A
:101F500020460BB0BDE8F04F1DF035B906466BE7E3
:101F60003D4B186800283FF473AF3C4B4FF47A7B2D
:101F70001B684FF03C0CB5FBF3F5B5FBF0F14FF4EB
:101F8000616300FB11550BFB05F5B1FBF3F2B5FBEB
:101F9000F0FE03FB121100FB1E55B1FBFCF30BFB23
:101FA00005F5B5FBF0F50CFB131120460091CDE9CA
:101FB00001E52B49FFF7FAFE4AE707F0080B68E74F
:101FC0001F4979E7079BC346012B0CBF1D482548D5
:101FD00079E720462449FFF7E9FE013585E76907DF
:101FE00003D120462049FFF7E1FEAE422B4680D8C0
:101FF00020461E49FFF7DAFE81E76A0703D1204633
:102000001949FFF7D3FEAE422B4681D82046164928
:10201000FFF7CCFE87E700BFBF85020055630200D3
:10202000596302008C4A020047630200A36D02005C
:10203000A04A02007E630200846302004C63020037
:1020400050630200E1F10100A52E00008863020048
:1020500092630200946302001819002014190020F2
:10206000626302000FF20100906302008E630200BF
:1020700042F20F7373B58B4228BF0B4605680446C6
:10208000052168460D4A1BF0B9FE064663682846DE
:102090000B225B680A491DF088F86368324669467E
:1020A00028465B681DF081F863681B2228465B6840
:1020B00004491DF07AF802B070BD00BF70690200DB
:1020C000B385020097850200002201230749884258
:1020D00007D8002A08BF0123054A1360054B186082
:1020E0007047012240085B00F1E700BF40420F004B
:1020F00014190020181900202DE9F34143680DF14F
:1021000007011C68104865681DF0E4F830B99DF8B7
:102110000710012902D10C4800F030F801232B757B
:1021200025682F68D5E90136D3E9004824B96B68E2
:102130001C6002B0BDE8F081214630464246B847F7
:10214000241A0644F2E700BFF83D0200F8B50D4638
:102150000446064F4618B44201D12846F8BD14F88B
:10216000011BBB6801485B689847F4E7F83D020033
:10217000014B036000207047E84A020070B5C46953
:102180000D4694B31D4A2379565CB34230D01C4AA5
:10219000525C9A422FD1A3689847002810DA022D8A
:1021A0000CD0032D0BD110F1860F07D0D4E8EF3FF0
:1021B00043F00203C4E8E23F002AF6E7267170BD4F
:1021C000022D26710FD1D4E8EF3F23F00403C4E8B9
:1021D000E23F002AF7D1D4E8EF3F23F00203C4E83E
:1021E000E23F002AF7D10020E9E76FF05700E6E769
:1021F0006FF07700E3E76FF08500E0E7C885020045
:10220000C485020010B54FF42814DFF820C086B052
:10221000CDE904C40824029404AC0194BDF8204024
:1022200000941EF0A8FC06B010BD00BF18002800E6
:1022300008B50348034A0021121A1DF0C3F808BD6F
:1022400030080020883A0020074808B5074A0849A6
:10225000121A1DF0B9F8BDE808400648064A0749B9
:10226000121A1DF0B1B800BF000000202C08002099
:102270005089020000000020000000205089020068
:102280002DE9F04780460C4600AF002936D0D1E951
:102290000012E9468AB06D46A3684FF0050A6E4603
:1022A0001F48CDE90723CDE9050146F810AF00230B
:1022B00032464FF421511B48FFF79CFCD4E903122E
:1022C000CD466369AD461848C5E90723C5E9050150
:1022D000C5F810A0002332464FF421511148FFF7F2
:1022E00089FCCD46E3690121104A0E481CF049FFE4
:1022F000A36901210E4A0B481CF043FFB8F1010FFE
:1023000007D1EFF305830B4A41460648103B1CF00A
:1023100038FF2146404618F051FDBD46BDE8F08724
:10232000F0630200084902001F6402004E640200CC
:102330005D6402008B64020030BFFFF7FDBF00BF89
:1023400010B5244C244925481DF04BF8A36A990187
:102350003ED5224822491DF044F81E20A36ADA0126
:1023600004D51E481F491DF03CF81F20194CA36AD4
:10237000DB0204D519481C491DF033F80220A36A7A
:102380001C0304D5154819491DF02BF82120114CC8
:10239000A36A590304D5114815491DF022F82220DB
:1023A000A36A9A0304D50D4812491DF01AF8232098
:1023B000084CA36ADB0304D508480F491DF011F847
:1023C0002420A36A6FEA03436FEA1343A36210BD9C
:1023D0001D20C3E700ED00E09E64020008490200F2
:1023E000B6640200C9640200E36402000D650200E5
:1023F0002B650200506502006A65020070B5064652
:102400000D46294C29492A481CF0EBFFA36ADB063C
:1024100047D5274827491CF0E4FF1120A36A1C0771
:1024200004D5234824491CF0DCFF12201E4CA36A6B
:10243000990712D521491E481CF0D3FF636BA26A8D
:10244000120609D501211E4A19481CF09AFE1EB138
:10245000A36A23F08003A3621320134CA36ADE0750
:1024600004D5134817491CF0BCFF1420A36A9C062E
:1024700004D50F4814491CF0B4FF15200A4B9A6A82
:10248000D10658BF9A6A9A6A920642BF5A6A22F4E3
:1024900000525A629A6A42F0FF029A6200232B703D
:1024A00070BD1020BAE700BF00ED00E095650200A6
:1024B00008490200AB650200DE650200F16502001A
:1024C000096602001F6602003E66020070B50646FD
:1024D0000D46284C284929481CF083FFA36AD904DB
:1024E0003CD5264826491CF07CFF1720A36A1A0514
:1024F00004D5224823491CF074FF18201D4CA36A00
:102500009B0512D51D4820491CF06BFFA36BA26AE6
:10251000100409D501211D4A18481CF032FE1EB1D5
:10252000A36A23F40043A3621920124CA36A59053D
:1025300004D5124816491CF054FF1A20A36ADA0584
:102540000ED50E4813491CF04CFF1B20094A936A14
:1025500043F47F43936200232B7070BD1620C5E7C0
:10256000A36A9B04F2D505480B491CF03AFF1C20D6
:10257000ECE700BF00ED00E06D66020008490200D4
:1025800083660200DE65020094660200AD6602000A
:10259000C2660200DD6602003E6602002DE9F041DF
:1025A0008AB0694B4FF000085E6800AFC6F30804BC
:1025B00088F31188BFF36F8F02F07F43B3F17F4F31
:1025C0000FD04FF0000845460023FB71E31E092B96
:1025D00000F29980DFE803F0148F928C9797979719
:1025E0009795150708D5530704D4584958481CF047
:1025F000F8FEE6E70D46E7E705464FF00108E3E79A
:10260000544953481CF0EDFE00234F4EFB71F46A11
:1026100014F0020405D050494D481CF0E2FE00249D
:1026200006E0F36A002B26DA4C4949481CF0D9FE33
:10263000FB79E3B907F1080205F120061346286883
:102640006968083503C3B5421A46F7D17B6AB8F109
:10265000000F75D0C3F3080222B96FEA53236FEA63
:1026600043237B62204607F10801FFF709FE283764
:10267000BD46BDE8F081F46A14F08044D8D03849F2
:1026800033481CF0AEFE7369AA6943F4807373612A
:10269000BFF34F8FBFF36F8F736932F8022C23F4AF
:1026A00080737361BFF34F8FBFF36F8F4DF602736B
:1026B0009A4207D12B6801212A4A25481CF061FD66
:1026C0002C68B5E7B36ADBB22BB10120F91DFFF727
:1026D00095FE0446ACE7B46A14F47F4404D00120AC
:1026E000F91DFFF7F3FEF4E7B36AB3F5803F9FD31C
:1026F000FFF726FEEDE70020F91DE8E70020F91DB1
:10270000EFE7194988E7194A16F4F87F184B6E4627
:1027100008BF13468AB0174A103CCDE905234FF491
:1027200000736A46ADF82030134B079442F8103F0F
:1027300000234FF411510648FFF75CFAB5466EE7E7
:102740006FF308038DE700BF00ED00E02367020090
:10275000084902004E6702006567020086670200B2
:1027600094670200B3670200CF670200F5660200BB
:102770000A670200F367020004000001064B5A6971
:1027800042F010025A615A6942F480625A615A69F1
:1027900022F008025A61704700ED00E0EFF3088074
:1027A000EFF3098101B57246FFF7F8FE01BD00BFE6
:1027B0000B4880F3088817F0F7FA202080F311887F
:1027C00008484FF40061401880F30988EFF3148043
:1027D0000221084380F31488BFF36F8F00F06AF87A
:1027E000D0620020905100201EF0040F0CBFEFF3C8
:1027F0000880EFF30980816911F8021C0229FFD0DB
:1028000001B572461CF0E2FD01BD00BF00B2002818
:1028100007DB01234109034A00F01F00834042F80F
:102820002130704700E100E000B200280CDB0122FB
:102830000649430900F01F008240203341F823205D
:10284000BFF34F8FBFF36F8F704700BF00E100E011
:10285000054B420953F82220012300F01F0003FA20
:1028600000F01040704700BF00E100E000B2002817
:10287000ACBF00F16040074B01F101014FEA41118B
:10288000ABBF00F5614000F00F0080F80013195451
:10289000704700BF14ED00E0044B054A23F07F03AE
:1028A0009360BFF34F8FBFF36F8F7047000000003E
:1028B00000ED00E008B5FFF7EFFF0B4AD2F88830D3
:1028C00023F47003C2F88830EFF3148323F0040379
:1028D00083F31488BFF36F8FFFF7AAFCFFF7B4FCF4
:1028E0001CF0B1FD18F08CFB00ED00E042F8203C3C
:1028F000009B0B4942F81C3C019B21F0010142F86E
:10290000183C029B42F8081C42F8143C4FF08073BC
:1029100042F8043C0023203A02654367704700BF39
:10292000B1F3010000B50B4B0E4698601546436E9F
:1029300083F30B882C4686F309880020034B9847C5
:102940002046002100220023014C204701F4010011
:10295000B1F30100583100201022014B1A61704779
:1029600000ED00E0054B5A699B689A421FBF044A7C
:10297000536843F080535360704700BF58310020C4
:1029800000ED00E0084B9B6883420BD1EFF3058319
:1029900043B1064B5A6842F080525A605A6A22F498
:1029A00000425A621FF022BD5831002000ED00E0C5
:1029B00013498A684FF030001044EFF3098C80E827
:1029C000F01F202080F31288BFF36F8F0D4F4FF060
:1029D00000664A698A603E60506F0023536780F347
:1029E000118802F1300090E8F01F8CF3098802F1A1
:1029F000000004B51CF0FDFCBDE804407047000079
:102A00005831002004ED00E008B5EFF30583064AD5
:102A1000103B02EBC30152F8330049688847BDE818
:102A20000840FFF79FBF00BFB83E02001FB501215D
:102A3000084B094A094800F021F90023054A03938D
:102A4000074B0121019301A8D31A029300F020F94A
:102A500005B000BD0000042000000020744B0200FF
:102A6000300800200A7A0B6810B562F304031C4694
:102A7000CB68520923F01F0343EA4203044A43F0A0
:102A80000103C2F89800C2F89C40C2F8A03010BD03
:102A900000ED00E010B50A4BD3F89030C3F30723E4
:102AA000013B984208D901210346064A06481CF01A
:102AB00068FB6FF0150010BDFFF7D4FFFBE700BF08
:102AC00000ED00E00A680200F04802002DE9F04F36
:102AD000144607464FF0000987B0594D019100F1A7
:102AE0000408019B994527DAD7F804B0BBF1000F21
:102AF00045D0BBF11F0F17D91BF01F0F14D158F889
:102B000004AC1AF01F0F0FD150461CF0AAFC064669
:102B10000BEB0A0001381CF0A4FC864210D06FF0C9
:102B20001506484A334601E04B46474A01214748CB
:102B30001CF027FB6FF01504204607B0BDE8F08FAE
:102B400016F1160FEDD0B442EBDDC5F89860D5F85C
:102B50009C00C5F89860D5F8A030796843F01F0B49
:102B600058F8043C20F01F001944984201F1FF3A44
:102B70001DD1D34509D13946F0B21CF07BFC09F1D7
:102B800001090C3708F10C08ABE7C5F89860D5F8D7
:102B90009C30E0B263F30401C5F89C1039461CF088
:102BA00069FC10F1160F0446C6D00134E7E7013B7B
:102BB000D345E0B223F01F03C5F8986008D1D5F8DB
:102BC000A020394602F01F021343C5F8A030E6E703
:102BD000D5F8A01001F01F010B43C5F8A03039460D
:102BE0001CF048FC10F1160FA4D0C5F89860D5F879
:102BF0009C109DF810300BF1FF3B61F304038DF83E
:102C00001030D5F8A0100130490861F347138DF852
:102C10001030796858F8043CC0B20B44029323F09A
:102C20001F035B44A3EB0A0323F01F0302A90593D0
:102C3000FFF730FF10F1160F3FF47CAF441C9EE706
:102C400000ED00E05668020030680200F048020023
:102C50000522044BC3F89420BFF34F8FBFF36F8F4F
:102C6000704700BF00ED00E0BFF35F8F0022024B12
:102C7000C3F89420704700BF00ED00E010B5034C8E
:102C80002278FFF723FF207010BD00BF41390020DC
:102C90002DE9F04F294C05464FF00008A1464FF0B2
:102CA000140A85B0DFF898B0264E0191019B984533
:102CB00018DA6B68002B3CD029680846CDE902136E
:102CC0001CF0CFFBDDE902130746581801381CF051
:102CD000C8FB874209D014236FF0150203FB08F3E9
:102CE00049F8032005B0BDE8F08F17F1160F2760F3
:102CF000F8D09BF80030BB42F4DD0AFB0891C6F81F
:102D00009870C6F89870D6F89C000B7B60F30403AB
:102D10000B73D6F8A000400860F347130B73D6F886
:102D20009C3023F01F036360D6F8A03023F01F030C
:102D3000236108F1010814340C35B7E7401900206D
:102D40004139002000ED00E0F0B55249524DD1F874
:102D500090302C68C3F307239C4287B000F2968022
:102D60000020FFF781FF4D4BC1F8C030844215D1E0
:102D70004B4D01A82C70FFF7FBF900260446B44226
:102D800013D100202B784349D1F89020C2F30722B9
:102D9000934275DBFFF75CFF002047E0696801EBB9
:102DA0000011FFF75FFE0130E0E70199300101EB10
:102DB0000613DA686FF31302B2F1807F50D00AD89D
:102DC000B2F5001F34D0B2F5800F3DD0B2F5801FB0
:102DD00012D00136D3E7B2F1006F41D0B2F1805F7B
:102DE000F7D15A689B680958013B22F01F00034441
:102DF00023F01F03012031E05A689B680958013B0A
:102E000022F01F0003440120074623F01F0340EA7D
:102E10004710CDE902218DF8100002A9287805930A
:102E2000FFF738FE002827DA6FF0150007B0F0BD75
:102E30005A689B680958013B22F01F00034402278F
:102E4000012023F01F03E2E75A689B680958013B01
:102E500022F01F000344062023F01F030027D6E7BB
:102E60005A689B680958013B22F01F00034403275E
:102E7000012023F01F03CAE72B7801332B70A8E74A
:102E8000C1F89830C1F8A00001337DE74FF0FF3062
:102E9000CCE700BF00ED00E0804B0200AAFF440039
:102EA00041390020F0B587B007460E461446002190
:102EB000102268461D4620F0E9FC02238DF80230FE
:102EC000054B2A4621466846CDE9047601931BF05E
:102ED0005DF807B0F0BD00BFA7F4010008B5024BD4
:102EE0001B689847002008BD54190020034B044A72
:102EF0001860937843F002039370704754190020D0
:102F00004C02002008B50649064821F00701C1F12E
:102F1000005202F580221BF04CFC002008BD00BFCF
:102F2000477E0020581900204FF0FF324FF0FF334A
:102F3000014818F021B900BF5C020020014818F0D8
:102F40008BB900BF5C02002038B50546FFF7ECFFE7
:102F50002A46082106481BF0BBFB044620B91DB1D8
:102F60001CF0A7FA0C230360FFF7E8FF204638BDEA
:102F70005819002010B50446FFF7D6FF2146034834
:102F8000FDF772FEBDE81040FFF7D8BF58190020CA
:102F9000014B9868603070475831002070B5416926
:102FA0000446867A0A4D59B1437ADB0706D42423B6
:102FB00003FB0653DB691B689B689847002363612A
:102FC0002420214600FB0650BDE870401FF0A7B842
:102FD000300700202422024B02FB0030704700BF64
:102FE000300700202421827A054B01FB02331A6A44
:102FF0001B7D801A1B3323F00303B0FBF3F07047F3
:103000003007002038B52424827A064B04FB0233B3
:10301000DB69D3E901240C601568FFF7E3FF04FBCB
:10302000005038BD300700202DE9FF4D05466846A9
:1030300092469B4603911FF0DFFADDE90067EFF34C
:103040001188202383F31288BFF36F8F6B8A002BC4
:1030500043D02A8A9A4227D900220023284618F012
:103060004BF9044600B388F31188BFF36F8F039BBD
:10307000002B42D032463B4668461FF0E2FA24213C
:10308000A27A264B204601FB0233DB6903A91B68A9
:103090001D68DDE90023A8470546606170BB204636
:1030A000FFF77CFF2C4624E0698A4B1E6B8288F375
:1030B0001188BFF36F8F2B7D2A8A2C6A1B3323F074
:1030C0000303521A02FB0344144B154AEB1A9B10DC
:1030D0005343A3722B7DE372C9E788F31188BFF3D2
:1030E0006F8F52465B46284618F006F904460028C2
:1030F000BDD1204604B0BDE8F08D636101230025F9
:103100002381039B29466382E27A656004F11800FB
:1031100020F0BCFB63692582E360EAE7300700200A
:10312000398EE338F8B5002424260F4D00B9F8BDD8
:10313000476800F10802D2E8EF3F591EC2E8EC1FD1
:10314000BCF1000FF7D1DBB2012BF0D1837AC46060
:1031500006FB035344609B6913B198473846E5E783
:10316000FFF71CFFFAE700BF3007002008B5254A2B
:10317000254B1A6015F096FF4FF47A612348D0F87A
:103180002436C3F30802C3F309434B4342F21071E0
:1031900082F48072883201FB02334FF4FA215B0023
:1031A000B3FBF1F201FB12331949B3F57A3F28BFA3
:1031B0000132C1F80429D0F820364FF47A60C3F305
:1031C0000802C3F30943434342F6041082F48072B9
:1031D00002F2172200FB02334FF47A701B0AB3FB92
:1031E000F0F200FB12330020B3F5FA7F4FF0010339
:1031F00028BF0132C1F81C27C1F80009C1F8003608
:1032000008BD00BF0020A1070C06002000C0FF0081
:103210000000125048B1054B054A1B68B3FBF2F39E
:103220005843044B43F00103184770470C06002035
:1032300040420F00C049020070B50B7892B00646BC
:103240000C4607AD032B31D8DFE803F0022A2C2E01
:1032500019492846FDF72EF905956378174A049316
:10326000A3781E210393E3780AA80293237910AD73
:10327000019363790093A3791AF0C0FD32460AAB3B
:103280001C4603CCAC4210605160234602F1080298
:10329000F6D1206810603046A388938012B070BDCC
:1032A0000749D6E70749D4E70749D2E70A21284664
:1032B000064A1AF0A3FDCFE7A3680200C568020022
:1032C000AA680200B1680200BB680200F081020037
:1032D0000D4B402928BF402170B51D460B4C4618A8
:1032E000B04204D1002305F81130074870BD0278C0
:1032F0001209A25C03F8022B10F8012B02F00F0256
:10330000A25C03F8012CEBE742390020E6850200BD
:1033100010B50024094B86B009480393CDE9044455
:103320001FF003F803AB00934FF4AF620A23054983
:10333000034818F033FA204606B010BDEF680200CB
:10334000200D0020883D00200146014818F066BA93
:10335000200D0020014601481EF0BCBF200D0020BA
:1033600030B50378012B11D0022B1FD06BB90A4660
:10337000134B03F1100453F8045BA34242F8045BBF
:10338000F9D143881A0A8A70CB7030BD0A460C4BBB
:1033900003F1100453F8045BA34242F8045BF9D133
:1033A00043681A0C180E08704A70EBE700F110031E
:1033B000013913F80129984201F8012FF9D1E4E706
:1033C000F785020010B51CF004FA1FF004F804465B
:1033D00008B918F01DFE064BD3E8AF3F0BB10A2029
:1033E00098471CB9BDE8104018F026BE10BD00BFBC
:1033F0006419002038B5044608481CF081F80546D9
:1034000050B1601EC0B21F2896BF054B0021195C49
:1034100005F10C001CF0F3F8284638BDE407002045
:10342000078602000F2810B50CD80D280CD90A48C1
:103430001CF066F8044618B104210C301CF0DFF8CB
:10344000204610BD1328F2D009B10448F0E702204D
:10345000BDE81040FFF7CEBF080800207807002025
:1034600005280CD0A0F10E030C2B0AD8064B23FA2A
:1034700000F000F00100C0F10200C0B2704703206C
:1034800070470220704700BF00C0080410B5002438
:1034900086B003AB00934FF480624FF0FF330549D1
:1034A0000548CDE90344059418F078F9204606B0A4
:1034B00010BD00BF00430020C00D002070B5C668DD
:1034C000337893B9B6F801400F21204602F008FE88
:1034D000F378054650B90A4A118831B96FEA0450A9
:1034E0006FEA10501080074A137070BD03730121FA
:1034F00002F012FD2846BDE8704002F0C1BC00BFDA
:1035000020380020C339002010B5084C014606229F
:1035100094F86E0003F040F938B994F86E00052273
:10352000BDE81040024903F037B910BD000000208B
:10353000CC85020070B5C3681D78B5B9B3F80160D9
:103540000F21304602F0CCFD044630B9074932461F
:10355000BDE8704006481CF0BDB9294602F0DCFC0D
:103560002046BDE8704002F08BBC70BD07690200C8
:103570008848020010B5C36801211C88204602F06B
:10358000AFFD30B905492246BDE8104004481CF0A3
:10359000A1B9BDE8104002F073BC00BF2D69020064
:1035A0008848020010B5C3680121B3F801402046E5
:1035B00002F096FD30B905492246BDE810400448A6
:1035C0001CF088B9BDE8104002F05ABC2D69020019
:1035D0008848020008B501210C301CF031F802784F
:1035E00002490348BDE808401CF074B95169020063
:1035F00088480200014608B507481BF085FF0749C7
:1036000007481EF067FE021E05DABDE808400549BE
:1036100005481CF05FB908BD34010020700300208C
:10362000600E0020736902008848020070B5C5680A
:103630000121B5F80160304602F052FD044630B970
:103640000D493246BDE870400C481CF043B92B7858
:103650003BB9D5F80330C0F89930D5F80730C0F839
:103660009D30201D4FF480311CF026F92046BDE826
:10367000704002F005BC00BF2D69020088480200BE
:103680002DE9F84FD0F80C90028A99F8001000AF9D
:103690008B00013393425DD96C468AB0CDE9073285
:1036A0006A4605232D48CDE905014FF421512C48E8
:1036B00042F8103F1CF00BF9A546BD46BDE8F88F57
:1036C00028492A4626481CF005F9013699F80030A9
:1036D0009E42F2DA09EB8603B3F801500F21284627
:1036E000B3F8038002F0FCFC04460028E8D000F1A7
:1036F000C00AB8F1000F05D065693DB91A491848EC
:103700001CF0EDF8204602F0BBFBDEE7A2692B6857
:1037100095422046636108BFA36108F1FF3802F0BB
:10372000D1FA1FFA88F817F01BFEC5F800B0236A1B
:103730006BB9C4E90755DAE8EF3F013BCAE8E23F5D
:10374000002AF8D10021204602F0C8FAD1E71D6016
:103750002562F0E70026B346B8E700BF9069020093
:1037600088480200BB690200D769020037B502EB46
:10377000C3039A4202D16FF05E0010E0144614F8C1
:10378000085B854212D10B8A54789C4209D90121E9
:103790000090074A07481BF0FDFC6FF0150003B0CE
:1037A00030BD0846536898470020F8E72246E0E716
:1037B000EE69020088480200F8B500AF06460D46E3
:1037C000FFF7D4FF5F3019D12C8AE8682146FFF754
:1037D0007FFD6D468AB00A4B6A46CDE9053640F258
:1037E0000243ADF82430074BCDE907404FF4325186
:1037F000054842F8103F1CF06AF8AD46BD46F8BDDA
:10380000106A020005000001884802002DE9F04717
:103810000C4618F0FDFBE5682A78022A4ED0042AEF
:1038200006D03C493C481CF055F86FF0150449E0BF
:10383000B4F81080B8F1020F08D84246374936482C
:103840001CF048F82046FFF76DFC3AE068783E2807
:103850003DD1B8F1030F02D131494246EFE7EB7891
:10386000012B29D10327012104F10C00D4F8149075
:103870001BF0DEFE022104F10C001BF0E1FE82468B
:1038800000783E283CD1E3681B78012B25D1032624
:1038900006232146234A9AF80000FFF78DFFB3075D
:1038A00034D56369A5EB090513FA85F5E560A4F83D
:1038B0001080012F02D104E00A2BD3D02046FFF75D
:1038C00099FE002418F0B8FB2046BDE8F087FFF70A
:1038D000C7FDC1070746F1D5C5E70A2BD7D041F28E
:1038E0006F13114A114912481AF0F8FF002383F3AD
:1038F0001188BFF36F8F0323184602DF0226C7E744
:10390000FFF7AEFDC2070646C2D4E8E72046FFF740
:1039100009FCCEE7DF6A020088480200326A020032
:103920004E6A0200744C02006E6A0200A96A02002C
:10393000C26A020010B5012104460C301BF080FE63
:103940002146BDE810400223014A0078FFF734BF4A
:10395000A44C020073B53D481BF0EBFD0446002863
:1039600071D000F10C0528461BF072FE02280246B9
:1039700003D0042845D0364903E0228A032A04D81C
:10398000344935481BF0A6FF13E0042128461BF0FC
:1039900057FEFF23428806882376238AC6F30B004E
:1039A0009A42608309D0012100922B482B4A1BF0D8
:1039B000F1FB2046FFF7B6FB12E00F2102F090FB6F
:1039C000054610B9628B2649DBE702F0B1FB2146C0
:1039D0002076320B284602F0CFF9284602F050FA42
:1039E000204BD3F8343173B31F4920481EF072FCCA
:1039F000021E28DA1E49184802B0BDE870401BF0CC
:103A000069BF022128461BF01BFE064600783E28AF
:103A100012D0FFF725FD10F002050DD140F6A143AD
:103A2000144A154915481AF059FF85F31188BFF358
:103A30006F8F0323184602DF06232146104A307891
:103A4000FFF7BAFEB5E702B070BD00BF3401002039
:103A5000886B0200F36A020088480200146B0200BF
:103A6000386B02000000002070030020600E002070
:103A7000736902006E6A02005A6B0200C26A020099
:103A8000B44C020010B5012104460C301BF0D8FDE7
:103A90002146BDE810400823014A0078FFF78CBE9C
:103AA000E44C0200F8B50121044600AF0C301BF0D5
:103AB000C7FD0678002321463046104AFFF756FE20
:103AC0005F3019D1258AE0682946FFF701FC6C4672
:103AD0008AB00B4B6A46CDE9053640F20243ADF899
:103AE0002430084BCDE907504FF43251064842F8D4
:103AF000103F1BF0ECFEA546BD46F8BD244D02006C
:103B00009C6B02000500000188480200C3681B7816
:103B10000221024A02481BF034BB00BFCE6B0200F8
:103B2000884802002DE9F74F81460F46924600284B
:103B300000F081800023DFF80481D8E8EF4FC8E867
:103B4000E23F002AF9D13CB94A463D493D4803B01D
:103B5000BDE8F04F1BF0BEBE2046FFF743FA4FF022
:103B60000C0B394D26460BFB005043884B451BD0B0
:103B70002046FFF737FA0BFB0050438801210093E2
:103B8000324A4B462F481BF005FBD8E8EF3FC8E808
:103B9000E26F002AF9D1002B4DD01E46304603B00B
:103BA000BDE8F04FFFF7BEBAA2450AD020461BF091
:103BB000A2FCBAF81020DAF80C1004F10C001BF08B
:103BC00015FD2046FFF70EFA4FF00C0808FB0050D9
:103BD00043689BB197B92046FFF704FA012108FB1F
:103BE00000504268536803F01F00814010685B0971
:103BF00000EB8300137AD3B11BF05EFE2046FFF783
:103C0000F1F94FF00C0808FB00508368002BC5D079
:103C10002046FFF7E7F908FB00F02F542046FFF796
:103C2000E1F908FB0055A86817F09AFBB6E7C9430D
:103C30001BF059FEE2E703B0BDE8F08F3001002031
:103C4000F66B020088480200681900201E6C020012
:103C500073B5C5680121B5F80160304602F040FA3D
:103C6000044638B932463B493B4802B0BDE8704093
:103C70001BF030BE2B78061D1A2B19D1C378012BEF
:103C800050D14FF4804130461BF016FE42040FD451
:103C9000D4F88C3069460093D4F8943020460193D0
:103CA00003F0AEF8204602B0BDE8704002F0E8B87C
:103CB0002B78BBBB40F2E242B5F8033027495343AF
:103CC000C4F88830B5F80520A4F89020B5F807208E
:103CD000A4F89220A3F5EA520C3A8A4204D90221B0
:103CE0001F4A1D481BF04DFAB4F89030B3F5FA7F27
:103CF00004D302211B4A18481BF043FA40F67641D0
:103D0000B4F89230A3F10A0292B28A4204D9022195
:103D1000154A11481BF035FA6FF4805130461BF0FC
:103D2000E2FD13E0D6E8AF3FDB04F5D52B78202B7E
:103D3000F2D194F89830002BEED0013B84F8983003
:103D40000A4A002304F1400017F092FD204602F0D9
:103D5000BFFBA7E72D6902008848020095F03C00F0
:103D6000516C0200786C02009F6C02005A620200E3
:103D7000B0B53C28044600AF19D101F099FA6FF4B0
:103D8000807110301BF0AFFD0020FFF7BDFB054632
:103D900028B9124912481BF0A2FDBD46B0BD0473FC
:103DA000002102F0B9F8284602F06AF8F5E76D46FE
:103DB0008AB00C4B6A46CDE905300B4B4FF41251DB
:103DC000079340F20133ADF82030084B044842F825
:103DD000103F1BF07CFDAD46DFE700BFCB6C02005F
:103DE00088480200EC6C02004663020004000001F7
:103DF000054BD3E8AF2F02F00B02D3E8EF1FC3E867
:103E0000E02F0028F9D17047D400002010B5C1E997
:103E100000239DF808300C460B72FFF7E3F80C22E4
:103E2000024B02FB00335C6010BD00BF681900202C
:103E3000F8B502460B4610481BF062FB0446C0B1C1
:103E400004210C301BF0C1FB2046FFF7CBF80C27F8
:103E500000260A4D07FB005046802046FFF7C2F8B7
:103E600007FB005086602046FFF7BCF807FB0055B3
:103E70006E602046F8BD00BFC00700206819002012
:103E800029289ABF014B185C09207047318602002F
:103E900070B5C3680F21B3F801601D78304602F099
:103EA0001FF9044630B919493246BDE87040184838
:103EB0001BF010BD65B12846FFF7E2FF2946024618
:103EC000204602F0C3FB2046BDE8704001F0D8BF99
:103ED0008378012B07D106F089FA20461BF0D4FC29
:103EE000002808BF05252846FFF7CAFF29460246D5
:103EF000204602F0ABFB002DE5D0064904481BF03C
:103F0000EEFC052120461BF06CFFDCE70769020090
:103F100088480200086D0200F8B5C6680F21B6F89F
:103F200001703578384602F0DBF8044630B91F4995
:103F30003A46BDE8F8401E481BF0CCBC65B12846A7
:103F4000FFF79EFF29460246204602F07FFB2046EF
:103F5000BDE8F84001F094BFF278C37A934205D1EE
:103F60000221144A12481BF00CF9F0E78378C27260
:103F7000012B08D10AB106F039FA20461BF084FC67
:103F8000002808BF05252846FFF77AFF2946024684
:103F9000204602F05BFB002DD9D0074904481BF0F6
:103FA0009EFC052120461BF01CFFD0E7076902009C
:103FB000884802002E6D0200086D020011289ABF89
:103FC000024B53F820000248704700BFF04B02003C
:103FD0005D6D0200034B0146D3F84C018268926884
:103FE000104700BF000000202DE9F04F91B00421E0
:103FF00000AF49481BF060FC6E4688B0474B6A46EC
:104000000593474B4FF4E65106934FF40073ADF818
:104010001C30444B444842F8103F1BF058FCB54656
:10402000424C434BE179434D07F12008012998BFE9
:104030001D4640462146FFF7FFF88AB06A463E4BD0
:10404000CDF81C80CDE905353C4B4FF42351089346
:104050003B4B354842F8103F1BF039FC0125B54673
:104060002646DFF8E080DFF8E090E3799D423ADB16
:1040700094F86F206E461046FFF7A0FFB4F8721058
:10408000B4F876308CB0314DCDE90721CDE905503B
:104090006A464FF4007509932D4BADF828504FF444
:1040A000535142F8103F20481BF011FCB54694F8DC
:1040B00070201046FFF782FFB4F874308AB0CDE963
:1040C00007236A46234B2449ADF82450CDE9051057
:1040D0004FF43351144842F8103F1BF0F8FB4437BB
:1040E000BD46BDE8F08F073631463846FFF7A4F8E5
:1040F000EA468AB040F201336A46CDE90585079762
:10410000ADF820304FF41351074842F8109F1BF0D0
:10411000DEFB0135D546A8E7D4000020696D02001A
:104120007B6D0200030000018848020000000020AF
:1041300046630200656D0200866D02000002010305
:1041400004000002956D020004000001A66D02004B
:104150000600000105000001E46D02000048704700
:10416000F5600200014902481EF0B4B86003002067
:10417000C00D002070B506460C4639B1CB684A69BF
:104180009B1A032B0ED86FF0150509E04FF0FF3096
:104190004FF0FF31FFF74CFE044618B96FF0680589
:1041A000284670BD2046FEF71DFF0C22154BA518B2
:1041B00002FB0033032128465E801BF028FA0680AC
:1041C000237C0121033B837028461BF028FA40F62C
:1041D00035439E420ED12046FFF7FCFE05460028DF
:1041E000DED00949024609481BF074FB2046FEF761
:1041F00099FFD5E7214606481DF07FFF0025FFF710
:10420000B1FFCDE7681900200B6E0200884802005C
:104210003C0100202DE9F04784B0804691460C46D1
:1042200000AF71B94FF0FF304FF0FF31FFF700FEE4
:10423000044660B96FF0680528461037BD46BDE8F2
:10424000F087887AFEF7C6FE344B984260D101228F
:10425000002138461DF086FF2046FEF7C3FE0C23E2
:104260002F4E03FB0060876020461BF078F9014663
:104270004046FFF77FFF054618B12046FEF752FF84
:10428000DAE700233846274A17F09EF8824690B1B5
:1042900040F2E313244A254925481AF01FFB5246F1
:1042A000414624481AF01AFB85F31188BFF36F8F3B
:1042B0000323184602DF2046FEF794FE0C235843E2
:1042C000365CFEB16D468AB01B4B6A46CDE90538B7
:1042D0001A4B0796089340F20243ADF82430184B6E
:1042E0004FF43251174842F8103F093E1BF0EFFAE5
:1042F0002046AD46F6B2FEF715FF092E0BD8124B3D
:104300009D5799E7B9F1000FB7D0C9F8004093E77E
:104310006FF0150590E76FF004058DE7C0070020EA
:1043200068190020B4C404006E6A02002D6E0200F9
:10433000C26A0200366E02007B6E02004663020013
:1043400005000001884802002786020073B5064672
:104350000D4642F22F00002101AAFFF75BFF044641
:1043600030B1144914481BF0BAFA204602B070BDAF
:104370000198C368B3F801203280B3F803302B8072
:10438000FEF7D0FE3388A3F11B02E02A04D90221F4
:104390000A4A09481AF0F5FE44F248112B88A3F5A1
:1043A000A47292B28A42E0D90221054A02481AF068
:1043B000E8FEDAE79A6E020088480200BA6E020050
:1043C000DF6E02002DE9F0478CB0002605465B4BFE
:1043D000B0F80190198849F47042914204BF1E80E0
:1043E000574B00AF08BF1E7800F0D6FBEB7805F105
:1043F0000408012B08BF534B404614BF002493F818
:104400006E401BF0E2F94146B8B34FF0010A07F1E4
:1044100008001BF0CFF9D5F81130C7F80130B5F816
:104420001530A7F80530EB78012B05D107F108000E
:10443000FFF76AF80446A8BB07F11004414620467E
:10444000FEF7FAFE6D4688B03F4B6A46CDE905346B
:104450004FF40073ADF81C303C4B4FF4E2513C4834
:1044600042F8103F1BF033FA1321AD4648461BF0CB
:104470009AFA3037BD46BDE8F08720461BF0D4FBE2
:104480000346006895F804A0B8609A889B7968682C
:10449000BA81BB73B8F8042098F806303860BA8047
:1044A000BB71C0E70346B5F8012023F8702BBA7B37
:1044B000B868B98920679A7140F2E2429980B5F8EC
:1044C000173053430022C4F88830B5F81930A4F8E7
:1044D0009030B5F81B30A4F89230EB782273012BA2
:1044E000E3701AD187F800A0BA88BB793868A4F8BD
:1044F0007B2084F87D30C4F8770000F0D9FE237A61
:104500001049C3EBC3035A18CB58C4F87E309388C4
:10451000A4F88230937984F884300721204601F092
:10452000FBFC26B101212046267301F0F5FC204654
:1045300001F03AFE204601F0A3FC9AE72038002063
:10454000C339002000000020026F020003000001B8
:104550008848020000B5C36889B0187820B109B056
:104560005DF804EBFFF704BCB3F801208DF8000000
:10457000ADF80120DA788DF80320B3F80B20ADF800
:104580001720B3F80D20ADF81920B3F80F20ADF8BF
:104590001B205A7C8DF81D20586801901A899B7A3F
:1045A000ADF808208DF80A30074B68461A689B88DA
:1045B000CDF80B20ADF80F30CDF81120ADF8153047
:1045C000FFF700FF09B000BDE085020010B5FBF762
:1045D00083FF034B1B6813B1BDE81040184710BDA3
:1045E0008C1900202DE9F341304D0746D5F84C01D8
:1045F0001DF05AFC48B92E492E481BF070F96FF097
:104600001204204602B0BDE8F0816FF0020105F10E
:10461000D4001BF068F901211BF04EF910EA0104E7
:1046200041D1254B1F600A4605F590701DF09AFD9B
:10463000224E05F59E701DF032FD30461DF075FED0
:1046400030466FF007034FF496621D49009417F04F
:10465000A5F8D6F880001B491DF0C3FED5F84C0123
:104660000669D6F80080B8F1000F14D1164B3360FC
:1046700083681B689847044638B1C6F80080134920
:1046800022460C481BF026F9BBE73FB902B0BDE853
:10469000F041FBF721BF6FF07704F0E705F1C400AC
:1046A00017F076F8ADE76FF07704AAE70000002076
:1046B0007F700200884802008C190020600E0020E4
:1046C00000470020977002000D380000A070020023
:1046D000F0B5C56801212F8887B0B8B201F000FDA0
:1046E000064638B926492748BAB207B0BDE8F040B7
:1046F0001BF0F0B802ACD5F80220D5F806300194D2
:10470000698900911CF089FC40B34FF0FF304FF0F5
:10471000FF31FFF78DFB054640B91B4919481BF0D7
:10472000DEF8304601F0ACFB07B0F0BD12210C30D2
:104730001AF056FF0346224623F8027B144603CCA8
:10474000596006A98C421860224603F10803F5D18E
:10475000294642F21A00FFF70DFDE2E74FF0FF3065
:104760004FF0FF31FFF764FB04460028D5D002214B
:104770000C301AF035FF2146078042F21B00EAE7B1
:104780002D69020088480200BC70020070B5064620
:104790000D464FF0FF304FF0FF31FFF749FB044665
:1047A00028B9BDE87040084908481BF098B80321B3
:1047B0000C301AF015FF068085702146BDE8704068
:1047C00042F22100FFF7D6BCD370020088480200F5
:1047D00073B5C368D9789A781D8842EA0122ADF88A
:1047E000002059791A79A8B242EA0122ADF80220D4
:1047F000D9799A7942EA0122ADF804201A7A5B7AD3
:10480000012142EA0323ADF8063001F069FC0646B7
:1048100050B91D491D48AAB21BF05CF80221A8B28C
:10482000FFF7B4FF02B070BD694601F0A5FE38B9CC
:104830001E21A8B2FFF7AAFF304601F021FBF1E7E5
:104840004FF0FF304FF0FF31FFF7F2FA0446002837
:10485000F2D00E210C301AF0C3FE00230580C0F800
:104860000A30BDF8003021464380BDF80230838015
:10487000BDF80430C380BDF80630038142F2200049
:10488000FFF778FCD8E700BF2D69020088480200D6
:1048900038B5042104460C301AF0D2FE4578017870
:1048A00022464088FFF73EF935B1044816F058FD1E
:1048B000BDE83840FFF756BC38BD00BF20010020DE
:1048C000B0B50446032100AF0C301AF0B9FEE2681F
:1048D000B0F80130117840F63542934216D16C465B
:1048E0008AB0114B6A46CDE90531104B4FF4125195
:1048F000079340F20133ADF820300D4B0D4842F8DC
:10490000103F1AF0E4FFA546BD46B0BD057822462B
:104910001846FFF707F9002DF6D0074816F020FDDE
:10492000FFF720FCF0E700BFED70020046630200D5
:1049300004000001884802002001002038B517F06B
:1049400067FB304DD5F83C31002B57D000220023B7
:1049500005F5907016F038FD00284FD10022002395
:1049600005F59E7016F0C8FC044668B940F6B143E0
:10497000254A2649264819F0B1FF84F31188BFF370
:104980006F8F0323184602DFD5F8303173B1214908
:1049900021481AF0A4FF0022204BD3E8EF0FC3E810
:1049A000E12F0029F9D108B1FEF7BCFB20461AF02F
:1049B000D6FDC5F830012046FFF70CFB0246B8B122
:1049C000174915481AF086FF164816F0C9FC20460C
:1049D000FEF708FB0C22144B1F2102FB003022467D
:1049E0004088FFF79FF82046FEF79CFBFFF7BAFBD5
:1049F000FFF7B8FBBDE8384017F01EBB01F0E4FB41
:104A0000F8E700BF000000206E6A0200FB680200A9
:104A1000C26A0200257102008848020030010020AD
:104A20000B6E0200200100206819002070B54FF0C5
:104A3000FF320D464FF0FF3300210646FEF7F2FC31
:104A4000044660B91A230A4A0A490B4819F046FF7E
:104A500084F31188BFF36F8F0323184602DF02210E
:104A600004F10C001AF0BCFD06704570204670BDC4
:104A700065720200FB680200C26A0200F8B50746D0
:104A80000024094DEE79E3B29E4202D86FF0010096
:104A900006E0294638461BF008F8073508B12046DD
:104AA000F8BD0134EFE700BF0000002073B50446F5
:104AB0000E4679B1304613491AF0F7FF054648B95A
:104AC00031461148C4EBC40420441AF0F6FF2846CE
:104AD00002B070BD68461AF05FFE05460028F6D1A8
:104AE0006846FFF7CBFF0028F4DA0748C4EBC4049C
:104AF000694620441AF0E1FF002EE8D00146304616
:104B0000E3E700BFD38502000000002070B5174D19
:104B10000622294606461EF0C1FE0446D8B14FF0D3
:104B2000FF304FF0FF31FFF783F90446D0B1062282
:104B300031460C301AF05AFD2146002242F205009F
:104B4000FFF768FB044640B110F10D0F03D108498F
:104B500008481AF0F8FF204670BD30682860B38816
:104B6000AB80F8E76FF06804F5E700BF680000204D
:104B7000A272020090480200064BD3E8EFCF4CF43B
:104B8000806CC3E8E2CF002AF7D1037A194301729F
:104B9000704700BFD4000020084BD3E8EF2F22F469
:104BA0008061C3E8E01F0028F7D1530504D5002237
:104BB0000220034905F000BD704700BFD40000206B
:104BC00087FC0100002307B50449CDE900036A46CC
:104BD000022005F0F1FC019803B000BDA7FB010025
:104BE000F7B5054670B14C4C94F8122194F8133186
:104BF0000AB19A4208D2013384F813312B7A43F078
:104C000004032B7203B0F0BD00210222084601F01C
:104C1000C3FD064648B128460121FFF7ADFF3046E7
:104C200003B0BDE8F04001F02BB901463B4800F06D
:104C300039FB94F8133173B130461AF088FF50B144
:104C4000374938481AF07FFF0021374803B0BDE8E4
:104C5000F04000F027BB94F8132194F812319A42E7
:104C600019D132492F481AF06EFF002242F2290072
:104C70001146FFF7CFFA20B12D492A481AF05FFFFD
:104C8000E2E794F81331013384F813312B7A43F0BF
:104C900004032B72D8E72A466F1C394612F82E0BF4
:104CA0001AF012FF064620B122491E481AF047FFAB
:104CB00010E094F81331013384F813312B7A43F068
:104CC00004032B7294F8A7305B0707D41A491548E0
:104CD0001AF039FF01201AF03AFFB5E73946684665
:104CE0001AF0EBFE01234FF0FF304FF0FF318DF84B
:104CF0000730FFF79DF8044660B1082269460C3082
:104D00001AF074FC3246214642F24E00FFF782FA56
:104D10000028DFD00949C8E70000002005FC010099
:104D2000B17202009048020081FB0100D6720200BD
:104D300007730200277302004773020071730200B9
:104D4000F8B5054600B33A4C94F8122194F81331A3
:104D500092B10132934210DC00210222084601F098
:104D60001BFD064688B128460221FFF705FF3046A5
:104D7000BDE8F84001F084B813B1013B84F8133169
:104D80002B7A23F004032B72F8BD0146294800F06A
:104D900089FA30461AF0DBFE064688B10121034647
:104DA000254A26481AF0EDF994F8133113B1012081
:104DB0001AF0CDFEBDE8F8400021214800F072BA9B
:104DC00094F8133194F812219A420CD2013B84F8E2
:104DD00013312B7A024623F00403022019492B7267
:104DE00005F0EAFBE0E74FF0FF304FF0FF31FFF74F
:104DF0001FF8074668B107210C301AF0F1FB691C57
:104E00001AF05BFE3246394642F22800FFF702FAFA
:104E100020B10D4909481AF092FEC5E794F8133104
:104E2000013B84F813312B7A23F004032B72BBE788
:104E30000000002005FC01008C7302009048020075
:104E400081FB010029FB0100B973020070B5044623
:104E500021BB30B324491AF028FE10BB2046FFF7CF
:104E60000DFE002802DB6FF0770070BD237853B988
:104E70001E48C279002AF6D121461AF01EFE0123EF
:104E8000C3711046F1E7012B04D1A37903F0C003ED
:104E9000C02B06D0164917481AF051FE6FF01500C6
:104EA000E3E7124DEB79012B1BD005F1D403D3E8D6
:104EB000AF3FDB0707D4002CF0D020460A491AF098
:104EC000F4FD0028EAD1EE792146731C3046EB71DF
:104ED000FFF7ECFD08B93046C7E7EB79013BEB7112
:104EE000C3E76FF00B00C0E7D3850200000000208D
:104EF000DE730200904802002DE9F341044638B900
:104F00001A491B481AF01FFE002002B0BDE8F081CC
:104F1000002141F2090001AAFFF77CF9074608B118
:104F20001449EEE7019D0622D5F80C80124908F1DC
:104F300001001EF0B3FC30B10622104908F1010057
:104F40001EF0ACFC18B92846FEF7ECF8DCE7D8F800
:104F500001302846C4F80130B8F805302770A4F8AD
:104F60000530FEF7DFF80120CFE700BF0C74020028
:104F70009048020025740200E0850200DA850200F4
:104F800007B56846FFF7B8FF044BD87118B16946FA
:104F90000020FFF78BFD03B000BD00BF0000002024
:104FA000F0B5314E89B0F479002C55D196F8C27025
:104FB00017F0010711D12D492D481AF0C4FD3C46C8
:104FC000F471162500240127F379E0B283422FD82B
:104FD000002B41D0002009B0F0BD6A4621464FF6B3
:104FE0000940FFF717F920B1224921481AF0ABFD1B
:104FF000E6E7DDF800E0DEF80C506C788CB1AB1C15
:1050000002AA12359446186859680833ACE80300C0
:10501000AB426246F6D11868CCF800009B88ACF829
:1050200004307046FEF77EF8002CC8D11249DCE748
:1050300008AB05FB003353F8182C33F8143C6946D1
:10504000CDF80120ADF805308DF80070FFF72EFD8A
:105050000028C0D10134B7E70021084609B0BDE8F7
:10506000F040FFF7F3BE00BF0000002043740200D1
:10507000904802006F7402008F7402002DE9F04125
:1050800084460E4690461D4640B13BB1310310D5D3
:10509000720707D5264927481AF051FD6FF0150011
:1050A000BDE8F0811AF0D4FD0028F9D101232B705E
:1050B000F6E7B307047822D01F492AB1B70603D513
:1050C00091F8D830580630D5C4EBC4040F5D012FD9
:1050D00008D10134604621441AF0B2FD0028DFD126
:1050E0002F7001E0002FFBD0B8F1000F05D0B20601
:1050F00042BF2B7843F002032B700020D0E77307E8
:1051000010D50D49C4EBC4040F5D012F07D1013444
:1051100021441AF095FD0028C2D12F70E7E7002F37
:10512000E5D1FAE71AF094FDC0E76FF08500B7E724
:10513000B8740200904802000000002038B50F4DFE
:10514000EB79CBB9FFF71CFF044628B10C490D4899
:105150001AF0F5FC204638BDEB79002BFAD1FFF7A9
:105160001FFF04460028F1D1681CFFF7CFFC04465E
:105170000028EFD00449EAE70024EBE70000002014
:10518000D774020090480200F67402002DE9F74F30
:10519000894601904FF0FF314FF0FF30FEF748FE97
:1051A000054600284ED020210C301AF019FA0026AE
:1051B0008046202200211EF069FB3346D9F80040CA
:1051C00008F10107D9F80420964224D294F801A0EE
:1051D000981C00EB0A0CBCF11F0F21785FFA80FBD2
:1051E00011D80AF1010C07F803C00133DBB2F954FE
:1051F0006168524638441EF022FB0BEB0A03DBB217
:1052000001360834DEE709290FD11C2B0DD80821FF
:10521000CBF11F0AE5E700222946019888F8003003
:1052200003B0BDE8F04FFEF7F5BF0121074A08487B
:1052300019F09FFF2846FDF775FF6FF0150003B0CA
:10524000BDE8F08F6FF06800F9E700BF1975020044
:1052500020480200F7B5CDE90001694642F2080096
:1052600016461D469DF82070FFF790FF044610B1CA
:10527000204603B0F0BD4FB9094BD3E8EF1F41F012
:105280000401C3E8E21F002AF2D0F6E7694642F2C1
:105290000900CDE90065FFF779FF0028ECD0E8E7C9
:1052A0002800002003460148184700BF18000020CE
:1052B00000487047180000202DE9F04F89B00546DE
:1052C0008946CDE90223D0F810809F4FD7E8AF3F41
:1052D0005A0740F193814468630506D4D0F810A0C2
:1052E000BAF1000F10D0A6070ED16FF015040023FD
:1052F00009F1010109F10400029A9A4240F0878104
:10530000204609B0BDE8F08F904E2878F3798342AB
:10531000EBD9C0EBC00007228D4930441EF0BEFA25
:105320000028E2D0A00706D196F86F30082B02D8EB
:10533000AB689F2BD9D914F0300F00F0B280BAF1CE
:10534000000FD2D0E10600F1B08004F46034B4F56F
:10535000603FCAD028461AF092FC83460028C4D089
:105360007C4BD3E8AF3FDA05C3F3002A00F1498153
:10537000D7E8AF3F5B0501D5FFF70EFC0023CDE971
:105380000533CDF81B30AB686A68ADF81030EB68B8
:1053900012F4004FADF8123014BF0623072312F4A5
:1053A000803F03F0050118BF0B4612F4003F03F0E5
:1053B000030118BF0B468DF81D30D7E8EF3F23F4EB
:1053C0008073C7E8E23F002AF7D12B78B8F10002DA
:1053D000337686F86E3018BF012269685E480DF199
:1053E0001503FFF74BFE0446002880D15B4BB8F154
:1053F000000F67D02A69116847F8B31C918899801B
:1054000092799A716B689C0762D0B8F1000F5BD0FB
:1054100013F0100F0CBF012304238DF814302B69F7
:105420001A68CDF816209A88ADF81A209B798DF865
:105430001C304FF0FF304FF0FF31FEF7F9FC04460F
:10544000002800F0E1800F2204A90C301AF0CEF8F9
:105450002146002242F20600FEF7DCFE0446002848
:105460007FF445AFB8F1000F3ED0686810F003003C
:1054700046D10646012138481AF015FC044600289A
:1054800074D00121364A374819F073FE002E3FF4DC
:105490002EAF3046002100F03FFD304600F0F0FC1A
:1054A00025E7BAF1000F7FF450AFD5E902239A4205
:1054B0003FF61BAF1F2A7FF618AFB3F5804F7FF67C
:1054C00044AF12E7224A96E78DF81480DA46B0E737
:1054D000980501D4039B1BB102238DF81430F5E726
:1054E00003238DF81430A4E74846DDE90212129B2D
:1054F000CDF800A0FFF7AEFE04460028B5D0F6E6D2
:10550000347E07221249154886F86E401EF0C6F90F
:1055100050B92046144901F0C1F8064600286AD067
:10552000052100F0F9FCA5E720460C4901F0FAF846
:1055300000287FF4DAAE307E084901F0AFF8064665
:10554000002858D00621ECE7D400002000000020FD
:10555000D385020028000020180000202100002030
:105560003275020020480200CC85020016B1304698
:1055700000F086FC6B6813F0030F324B1FD0D3E8AA
:10558000EF2F42F40072C3E8E12F0029F7D1BAF1FE
:10559000000F1DD0D3E8EF2F42F48062C3E8E12F63
:1055A0000029F7D16A6851071BD5D3E8EF1F41F4F2
:1055B0008051C3E8E21F002A3FF499AEF5E7D3E833
:1055C000EF2F22F40072C3E8E12F0029DFD0F6E7C5
:1055D000D3E8EF2F22F48062C3E8E12F0029E1D065
:1055E000F6E7D3E8EF1F21F48051C3E8E21F002A59
:1055F0003FF47DAEF5E76FF00B0478E66FF00A0438
:1056000075E66FF0770472E66FF068046FE619F8DC
:105610003320012A09D111F83320012A05D150F88D
:10562000332012B11278D20701D4013364E606495F
:1056300006481CF080FE0023054A044816F050F985
:105640005EE600BF28000020C556000030000020A4
:105650001C4E0E0010B517481AF04DFB164CD4E83E
:10566000AF3FDA05C3F3002022D5D4E8AF3F9B0556
:1056700015D507221149E01F1EF010F9034614F852
:10568000100C93B905220E4901F086F8044630B19A
:105690000021017300F040FC204600F0F1FBBDE862
:1056A0001040002103481AF0FEBA0622E11FEBE782
:1056B00010BD00BF1800002028000020D385020084
:1056C000CC85020010B5FFF7C5FF034630B1BDE839
:1056D00010400221024A034819F053BD10BD00BF1B
:1056E0004D7502002048020070B59AB014220021C6
:1056F00004A81EF0CBF847F21213ADF80C304FF4AB
:10570000807344F20102ADF80E30374B3749CDE9D2
:10571000052303A801AB20221DF033FA0346E0B1B4
:10572000334A0121334819F02CFD1F25324BD3E8B1
:10573000EF1F21F00101C3E8E21F002AF7D12F4E2D
:1057400016F066FC34680CB1043C3FD10023C6E976
:10575000003316F071FC1AB070BD02AB4122019803
:1057600009A91DF0E4F9034608B1254AD9E7254AFD
:105770000DF125030DF1650153F8040B8B4242F83E
:10578000040BF9D102AB20221F4901981DF079F9D1
:10579000034608B11D4AC4E701981DF02AF90546E1
:1057A00010B11B4A0346BCE716491A481AF0A6FA7C
:1057B000194820311AF0A2FA184BD3E8EF1F41F034
:1057C0001001C3E8E21F002AB0D0F6E7002D114D0A
:1057D00018BF002523680BB1284698476468002C41
:1057E000B4D0043CF6E700BF000002099B8602002B
:1057F0007375020078480200901900209819002063
:105800008F750200E4390020C4390020B27502000F
:10581000D6750200243A0020443A0020D40000202B
:1058200030B5A7B01422002108A81EF02FF80423D9
:105830003D22002116A815931EF028F847F21213F6
:10584000ADF81C304FF4807344F20102ADF81E3005
:10585000284B2949CDE9092307A805AB20221DF0D3
:1058600090F90346E0B1254A0121254819F089FC49
:105870006FF0040416F0CCFB224B1D6865B10020CC
:105880001860214BD3E8EF1F21F00201C3E8E21FAB
:10589000002AF7D144B3A84716F0CEFB27B030BD9D
:1058A0001A4B0DF15502194603F1400053F8044B11
:1058B000834242F8044BF9D106AB029320230D48F2
:1058C000CDE9001315AA412305991DF0A9FA034655
:1058D00008B10F4AC8E705981DF08BF80446002868
:1058E000C8D00C4A0346BFE70DA808491AF006FACB
:1058F0000DA8D0E7000002099B860200F6750200A1
:10590000784802009419002090190020E439002002
:105910002C76020048760200402208B503491DF0AB
:10592000BDFFB0FA80F0400908BD00BF5B860200F1
:1059300010B598B004461422002102A81DF0A6FF5D
:1059400044F21213ADF804304FF480734FF48042E8
:10595000ADF80630144B2146CDE9032304230DF1A5
:105960001D008DF81C301AF0C9F904F120010DF169
:105970003D001AF0C3F96B46412207A901A81DF0AA
:1059800000F9044601A81DF093FA2CB900981DF007
:1059900030F8012018B010BD044823460121044A04
:1059A00019F0EFFB0020F5E700000209784802003B
:1059B0006576020010B5002834D01D4A136823B163
:1059C000043B984231D05B68F9E71A4BD3E8AF1F2C
:1059D000890707D518480221184A19F0CAFB6FF049
:1059E0000F0010BD1468011D44605068116000B9BB
:1059F0005160D3E8EF2F42F00101C3E8E01F002817
:105A0000F7D1D30701D50020EBE70D4BD3E8EF1F0B
:105A100021F01001C3E8E21F002AF7D10948FDF781
:105A200099FCF0E76FF01500DBE76FF07700D8E73F
:105A30009819002090190020784802008976020009
:105A4000D400002090030020044BD3E8AF3F13F0B4
:105A5000100F034808BF0020704700BFD40000208B
:105A6000243A002070B51A4A054613688B4228D0A4
:105A7000184BD3E8AF3FDC0626D5136813B16FF09F
:105A80000F0070BD144BD3E8AF0FC007F7D4D3E8B5
:105A9000EF0F40F00204C3E8E64F002EF7D110F0FC
:105AA0000204ECD111600D4829461AF027F90C4880
:105AB00005F120011AF022F90A48FDF74BFC2046B7
:105AC000DFE76FF07700DCE76FF07C00D9E700BF1D
:105AD00094190020D400002090190020E4390020FF
:105AE000043A00208003002070B505460B4B1C686B
:105AF00044B154F81C3C1C3C13B12846297B984700
:105B0000E469F5E7064C074EB44200D370BD236844
:105B100013B12846297B98472034F5E7D419002093
:105B2000E84702000848020010B50446FDF75AFA9B
:105B3000044901EB0011204619F087FEBDE8104032
:105B4000FEF710BBA0190020002370B50546D1E96F
:105B500001460748C1E901331CF0CFFA3CB1314698
:105B600028462346BDE870406FF06D02184770BDAF
:105B70002007002037B5437B0446072B3FD1051D86
:105B80004FF4806128461AF0E0F8410537D4D5E893
:105B9000AF3FDA0326D5E37823B90221194A1A4820
:105BA0001AF0D1F8637B072B29D1184B93F8D83022
:105BB0009B0624D519F0C9FE08B30DF1060101A812
:105BC000FEF7C4FBD8B92046BDF80620BDF8041086
:105BD00019F028FF034690B101210D4A0A481AF036
:105BE000B2F80CE0204619F002FF034620B1012173
:105BF000084A05481AF0A7F8637B072BCBD003B0FF
:105C000030BD00BFD87602003848020000000020F6
:105C1000F1760200B776020070B505460022002337
:105C20000E4815F0D1FBB8B90D4B1C6834B154F8CF
:105C3000143C1C3C03B19847E469F7E7094C0A4E51
:105C4000B44204D32846BDE8704015F0A1BDA36856
:105C500003B198472034F3E770BD00BF1007002060
:105C6000D4190020E8470200084802002DE9F0415D
:105C7000044620270025EFF3118287F31288BFF333
:105C80006F8FE16929B1206A0B688142E36108BF27
:105C9000236282F31188BFF36F8F71B1D1E901687C
:105CA0000748C1E901551CF028FA1EB100224146FF
:105CB0002046B047FEF756FADDE7BDE8F08100BFA9
:105CC000200700200448B0F8FC3000F58070002B5D
:105CD00008BF0020704700BF0000002030B5044618
:105CE0000D4689B016F0B8F90B4BD3F880208242EC
:105CF00005D1204609B0BDE83040FFF7B7BF1846D0
:105D000004F124011CF0E6FA25B1694604F12400EF
:105D10001CF0F0FA09B030BDB817002038B50022E9
:105D200004468A4202D10024204638BD012004F1F5
:105D3000C803D3E8EF5F002D04D1C3E8EC0FBCF13A
:105D4000000FF6D102D0D0340244EAE7002CEAD0AA
:105D5000C822002120461DF099FD04F140000449AD
:105D60001CF0E9FA034904F124001CF098FADBE77F
:105D7000FD68000061FD0100F7B516460D460121E2
:105D80000446FFF7ABFF012E23D0022E52D1236928
:105D90003BB135480121354A19F0EBF9204619F09D
:105DA000FDFF25612269138A012B5AD9D268128816
:105DB000043292B2934254D343D9012100922A482B
:105DC0002B4A19F0E7F9204603B0BDE8F04019F07E
:105DD000E5BF206940B9274A3146234819F0C9F97F
:105DE000204619F0DBFF01E02A8A2AB9284603B0D1
:105DF000BDE8F040FDF796B9018A438A47695B1A0E
:105E0000C168C91B5B1A9A420CD91B4A3146164815
:105E100019F0AFF900222046216900F0C5FF0023E8
:105E20002361E3E7E9680C3019F0E0FB2846FDF751
:105E300079F9B7E701213346104A0B4819F083FF7F
:105E4000CEE7002204F11003D3E8EF1FC3E8E02FF0
:105E50000028F9D10122204603B0BDE8F04000F04F
:105E6000A3BF03B0F0BD00BF384802000D770200A9
:105E70008D7702002A770200487702006F770200D0
:105E800008B500F1C803D3E8EF2F013AC3E8E12FCA
:105E90000029F8D1AAB90B4B984212D303F1D002D2
:105EA00090420ED2C01AD023B0FBF3F203FB1200D3
:105EB00038B9054815F054FABDE80840034815F014
:105EC00067BC08BD000F002010070020B0030020B1
:105ED00010B5044619F071FF16F09AF80C4B04F156
:105EE000BC01D3F8143143B90A4819F011FF16F078
:105EF000A3F8BDE81040FEF735B9994201D01B6800
:105F0000F1E716F099F82046FFF7BAFFF1E700BF76
:105F10000000002014010020F8B5457B04468D42A6
:105F20000E4600AF1CD1082D98BF544B6C4694BF51
:105F300053F82530524B88B0524ACDE905234FF42F
:105F400000736A46ADF81C304F4B42F8103F0023F7
:105F50004FF4E4514D48FBF74DFEA546BD46F8BD54
:105F600041730DB919F029FF637B082B00F2828081
:105F700001A252F823F000BFC55F00001B600000C3
:105F80005D5F00005D5F00005D5F00005D5F000021
:105F90005D5F00009D5F00005D5F00000023C4E9BD
:105FA0000D33E378012BD9D1A378394A012B08BFEF
:105FB000032304F1400008BF84F89830002315F053
:105FC00057FCCBE7082DC9D8DFE805F02005171CE2
:105FD0001C1C1720200004F140001CF0B7F901211F
:105FE0002046FFF77BFE204619F0D8FE0022002352
:105FF00004F1400015F074FCB0E7237B13B1204698
:10600000FFF772FD2046FFF73BFFA7E73346214A23
:1060100002211E4819F097FEA0E7237B3E2B0FD1EB
:106020006D4688B01C4B6A46CDE90534032342F81F
:10603000103F00234FF4C4511448FBF7DBFDAD467D
:10604000164D05F58076616911B9FEF78BF885E785
:10605000A2690B68914208BFA36120466361FFF704
:1060600073FDB5F8FC30002B14BF3046002015F04E
:1060700077F9E8E70A4A3346CAE700BF384D02001D
:10608000A8770200B277020003000001384802003E
:106090005A620200C3770200DA7702000000002093
:1060A00001780200F8B5074608480D46164619F073
:1060B00084FE044648B183781F4202D03146A84787
:1060C0002046BDE8F840FFF7DBBEF8BD000F00201A
:1060D000002201200149FFF7E5BF00BF755B00000A
:1060E00070B505460F480E4619F067FE044660B1CC
:1060F000427B012A02D0073A012A03D82388AB4207
:1061000005D02046FFF7BCFE0024204670BDA378D2
:106110001E42FAD102212B46034A044819F013FE0D
:10612000EFE700BF000F00201D7802003848020092
:10613000034BC01A034B00115843C0B2704700BF55
:10614000000F0020C54EECC4F8B51D4652EA050309
:1061500006460F4614460DD015F07EFF0E4BD3F8C1
:106160008030834206D1002402210C4A0C4819F0E9
:1061700000F825460B4922462B46002E14BF304618
:10618000084619F0BDF9044618B1791D0C3019F014
:106190001CFA2046F8BD00BFB81700203478020072
:1061A000384802003007002010B50446054815F0B5
:1061B000EFFA204600F054FD2046BDE81040FFF7FE
:1061C00093BC00BFA00300202DE9F04F002387B04F
:1061D00000AFFB607B61B24B5A8A12B91B68002B7F
:1061E00040D0B04DD5F814311C461BB154F8BC3921
:1061F00003B1BC3B0026AC49002C33D0B5F8FC20E1
:10620000002A00F06381D5F808215AB904F1BC06D0
:10621000002B00F0A880D3F8BC2002B1BC3A1C4689
:106220001346E9E70A68002AF0D0D4F8A820002A2B
:10623000ECD0D4F8AC20002AE8D0D4F8B020002A62
:10624000E4D0637B072B11D12046904770B104F155
:10625000C003D3E8AF3F022B08DC204619F0ADFDA8
:106260000446F8B91C37BD46BDE8F08FD4F8BC3001
:1062700004F1BC02002E6ED1D5F81811C5F8143106
:106280008A4201D1C5F8183100232046C4F8BC3039
:10629000D4F8B030984728B1637B072B02D1204651
:1062A000FFF716FE637B072B40F00D812046D4F8E4
:1062B000A830B5F8FC1007F1100298478146002875
:1062C00000F0E480B5F8FC203B699A4208D301460F
:1062D000D4F8AC60204607F1140307F10C02B04774
:1062E0007B69D7F80C803B60B9F81030002B00F0C8
:1062F000D4804846D7F810A019F0BDFA786000287D
:1063000040F0DE80B5F8FC30DFF8A0B1002B14BF00
:10631000584600200022002315F056F868B90022E4
:106320000023614814F0E8FF0646F0B9B5F8FC30E8
:10633000834218BF584615F013F86FF00B05484616
:10634000FCF7F0FEB8F1000F00F08B802A462046E3
:106350003968C04785E03360D5F818319A4208BFE4
:10636000C5F8186190E71A4659E73B68C0F8048001
:106370008360B5F8FCB00022DA454FF000034FF01F
:106380000001474898BF1FFA8AFBFCF74DFE804684
:1063900050B1FCF727FE464B5A4603EB0013494623
:1063A000404619F02EFA8046B5F8FC3094F8C490B7
:1063B0009A4584BF01237B607B6898BF09F102097D
:1063C00084F8C43004F1C00ADAE8EF3F0133CAE8C8
:1063D000E23F002AF8D104F1140B3146584619F077
:1063E00097FCA378012B55D108F10C031846042122
:1063F0007B6019F00CF9228829F0020942EA09327F
:106400000280B8F810200221043A4280786819F01E
:1064100006F94046FDF7DEFD8146002853D0DAE854
:10642000EF3F013BCAE8E23F002AF8D13146584627
:1064300019F099FC1F4A4B4601211F4819F083FCB3
:106440004046FCF76FFE20463146FFF77DFBB5F86E
:10645000FC301648002B08BF002014F081FF6FF0BD
:1064600004056E4688B0154B6A46CDE90535042310
:10647000079442F8103F4FF401510F480023FBF7F7
:10648000B9FB1321B546204619F0ABFC2046FFF7B7
:10649000F7FCE7E66FF01509C1E76FF079054EE705
:1064A0009C070020000000202007002000010020A1
:1064B000A01900200B6E0200384802005D7802002F
:1064C0006FF004053BE7FDF74DFEDFE79368FFDE65
:1064D00040F2E2432DE9F041D0F888600446B6FB73
:1064E000F3F6031DB6B2D3E8AF2F92041BD5B0F874
:1064F0008C20B24217D8B0F88E20B24213D3B0F835
:106500009010B0F8942091420DD1B0F89210B0F8EC
:106510009620914207D1D3E8EF1F21F40051C3E840
:10652000E21F002AF7D1114B1D6865B155F80C7CAC
:106530001C3D37B131462046B4F89230B4F8902073
:10654000B847ED69F1E70A4DDFF82880454501D3EA
:10655000BDE8F0812F6937B131462046B4F892305A
:10656000B4F89020B8472035F0E700BFD4190020D8
:10657000E8470200084802002DE9F04106460846B7
:106580000C4619F0E4F9054610B92846BDE8F0813B
:10659000134B1F6887B157F8103C1C3F0BB9FF69BC
:1065A000F8E72146304698470028EFD0204619F0FA
:1065B000CEF90028F3D1E9E70A4FDFF82C804745F0
:1065C000E3D2FB680BB92037F9E7214630469847FC
:1065D0000028DBD0204619F0BAF90028F3D1D5E71E
:1065E000D4190020E8470200084802002DE9F041D4
:1065F000C37805468BB900F17E06114B1C687CB14F
:106600001C3C05F1700763691BB13A4631462846C8
:106610009847E46924B11C3CF5E700F17706ECE704
:10662000084C094FBC4201D3BDE8F081636923B136
:106630003146284605F1700298472034F2E700BF42
:10664000D4190020E847020008480200F8B5437A50
:1066500005468372164619F004FD0D4B1C684CB1BB
:1066600054F8043C1C3C1BB132462846697A9847D2
:10667000E469F4E7074C084FBC4200D3F8BDA369B6
:106680001BB132462846697A98472034F4E700BFA8
:10669000D4190020E84702000848020038B5054632
:1066A0000C460F480121FFF739FBC0B10572236882
:1066B0000367A388A0F87430A37980F876300123AB
:1066C000437283728370074BC0F8A830064BC0F842
:1066D000AC30064BC0F8B030054BC0F88C3038BD3C
:1066E000000F0020616B000031FD010025FD01005D
:1066F0001800280070B5054609480E4619F05DFBE4
:10670000044658B18378012B05D13246294619F049
:10671000D9FB18B92046FFF7B3FB0024204670BD13
:10672000000F0020F0B589B000AF0E46FFF7E2FF82
:10673000044610B331463846FCF77EFD637B6E4657
:10674000082B96BF0E4A0F4B52F823308AB00E4AE0
:10675000CDE90773CDE905246A460C4B09930C4B30
:1067600042F8103F00234FF442510A48FBF742FA27
:106770002046B546FFF784FB01202437BD46F0BD17
:10678000384D0200A877020080780200010302045D
:106790000500000238480200F8B505460F480E46CD
:1067A000174619F00AFB044650B18378012B04D137
:1067B00066B9637BBB4205D02046FFF761FB00242E
:1067C0002046F8BD237AAB42FAD0F5E73246294697
:1067D00019F078FB0028ECD1EEE700BF000F002095
:1067E00070B58B780646012B0C4692B042D191F8D9
:1067F000703007AD032B37D8DFE803F002303234B6
:106800001E492846F9F756FE059594F871301E2169
:10681000049394F872301A4A039394F873300AA8D8
:10682000029394F87430019394F87530009394F8BF
:10683000763017F0E3FA32460AAB10AD1C4603CCB3
:10684000AC4210605160234602F10802F6D1206884
:1068500010603046A388938012B070BD0949D0E71C
:106860000949CEE70949CCE70A212846084A17F02A
:10687000C5FAC9E700238DF82830DCE7A3680200D9
:10688000C5680200AA680200B1680200BB68020085
:10689000F081020038B5044608460D4619F057F855
:1068A00038B3154B93F8D830990707D4E37873B110
:1068B00029462046BDE8384000F0A2BA94F8993045
:1068C0009A07F3D5231DD3E8AF3F5B04EED42946E6
:1068D000204619F017FB58B92B88A4F88C306B8828
:1068E000A4F88E30AB88A4F89430EB88A4F89630E6
:1068F00038BD6FF01500FBE700000020F7B510F879
:10690000333C054623BB403819F04EFB344B1C6822
:1069100054B154F8183C1C3C23B115F8341CA5F1B3
:1069200040009847E469F3E72E4C2F4FBC4206D352
:10693000A5F1400003B0BDE8F040FFF7A1BA6368DD
:1069400023B115F8341CA5F1400098472034EDE739
:1069500010F83E3C012B40D1A0F13C04D4E8EF3FBD
:1069600023F40052C4E8E12F0029F7D1990420D57F
:10697000EB6C694600936B6DA5F140000193FFF746
:1069800089FF034678B9D4E8EF3F23F48053C4E885
:10699000E23F002AF7D14FF40061204603B0BDE882
:1069A000F04019F0D2B9114A0221114819F0CBF97F
:1069B000F1E74FF428130F4A6946A5F14000CDE9ED
:1069C0000023FFF767FF034628B94FF480512046A4
:1069D00019F0BBF9DFE7084AE6E703B0F0BD00BFF6
:1069E000D4190020E847020008480200B9780200E4
:1069F0003848020018002800DE78020038B50E483A
:106A00001BF04DFB00240D4D29460B4801341BF0B3
:106A100074FB032C05F10C05F6D119F0CFFE02F042
:106A2000F3FA044628B903F08FFD044608B919F0BB
:106A30005DFB204638BD00BF20070020B0190020B4
:106A400098B50E4A00AF13682BB90D485060184630
:106A50000A60BD4698BD6C4688B00A4B6A46CDE9CF
:106A60000530032342F8103F074800234FF4C2517A
:106A7000FBF7C0F86FF00B00A546EAE7E819002025
:106A8000844D020091790200A04802002DE9F041F6
:106A90001D4652EA050306460F46144610D015F06F
:106AA000DBFA094BD3F88030834215BF224600221F
:106AB0002B4600233046391DBDE8F041FFF744BBAB
:106AC00000221346F6E700BFB8170020F8B50F46BE
:106AD00000210546164600234FF224420846FFF7E0
:106AE000D5FF044638B901212B46074A074818F05C
:106AF00048FB2046F8BD04210C3018F071FD0570EC
:106B000047704680F5E700BFB8790200A048020050
:106B100070B5056804461E4615B96FF07F0070BD5C
:106B20006B7B072BF9D10B7A012B07D001210A4A85
:106B30000A4818F026FB6FF01500F0E7CB7A072B18
:106B4000F9D98A61CE6130301BF0D7FA204619F0AE
:106B500002FA0020E3E700BFE0790200A04802004B
:106B60002DE9F84F88469146D0F8B44000AF4CB1BB
:106B7000403C236B6BB104F1300A50461BF0E0FA45
:106B8000054660B9FDF7EEFA00263046BD46BDE881
:106B9000F88F2068B43019F0FDF9246CE7E718F09D
:106BA0006AFE80B16C4688B02A4B6A46CDE905354D
:106BB000032342F8103F00234FF4C2512648FBF74D
:106BC00019F8A546E0E7284618F0C9FC656C0646AA
:106BD0009DB9A38C058A403B9BB23F2B03D8238DE4
:106BE0009D4228BF1D46042106F10C0018F00FFD40
:106BF0000580A38C043543806564A8451FD3B6F88F
:106C000010B0AB4506D100220023504614F074FBAF
:106C1000FCF788FAA38CA3F140023F2A06D8AB45C3
:106C20001ABF002213460D4AF361B2612068B430E6
:106C300019F0B0F9236B13B1204619F08CF9636C8D
:106C40009845C9F800302CBF0023A3EB0803636408
:106C50009BE700BFF8790200A04802009F000200F5
:106C6000F7B504460026234D234FBD4201D303B0A0
:106C7000F0BD2988204619F009FA6B68019001A936
:106C80002046984700282FDB01982B888382838435
:106C900000F11003D3E8EF2FC3E8E16F0029F9D129
:106CA000066446648660A26B00F10803F2B9C4E989
:106CB0000D330460C66030301BF0F1F90198436871
:106CC0001B6803B19847019B1033D3E8EF1F41F0D5
:106CD0000101C3E8E21F002AF7D101984368DB698C
:106CE00013B100F1100198470835BEE71360A363A4
:106CF000DFE700BFD0470200E847020073B50B8A08
:106D00000646032B0D4607D8214A0121214818F0D9
:106D100030FA002002B070BD042105F10C0018F01B
:106D20008FFC2B8A428804469A4206D000921A4A67
:106D30000121184818F02EFAEBE743780BB9174AEF
:106D4000E3E70378012BE4D0132B06D1022AE0D02D
:106D5000022300931346124AEAE70221114A0D4822
:106D600018F00FFA6178022201203568FFF7AEFEB5
:106D700004460028CDD002210C3018F031FC00234D
:106D8000214603704370284619F096F9C1E700BF09
:106D9000107A0200A04802002E7A02004F7A020008
:106DA000707A02009B7A020038B50B8A0546032BE5
:106DB0000C4609D801210F4A0F4818F0DAF920468D
:106DC000BDE83840FCF7AEB9042104F10C0018F01E
:106DD00037FC4188284619F080F930B9074A0B463C
:106DE0000548022118F0CDF9E9E7436821465B69BF
:106DF0009847E4E7C37A0200A0480200E07A020064
:106E000070B5134A0C4611780646013111F0FF01A6
:106E10000ABF01230B461946137012200822FFF700
:106E200055FE054688B108210C3018F0D9FB23889F
:106E30002946038063884380A3888380E388C380D6
:106E40003046BDE8704019F037B96FF00B0070BDE7
:106E5000643A0020232823D81C2804D8431E1A2B68
:106E60000DD906207047A0F11D03062B20D8DFE8BE
:106E700003F004251F100B1F1D0005207047012380
:106E80000F4A83401A400AB1022070470D4A1A4047
:106E90000AB1012070471B2814BF06200320704749
:106EA00000F07F03522B03D100207047032070476E
:106EB00010F0400F14BF00200620704704207047D8
:106EC000AAAA8A025455450108B5EFF3118120237F
:106ED00083F31288BFF36F8F002303600F4B5A6850
:106EE000C2B9C3E9000081F31188BFF36F8F0C486A
:106EF00014F04EFC031E0CDA01210A4A0A4818F06D
:106F000040F9002383F31188BFF36F8F03231846E2
:106F100002DF08BD10605860E5E700BF301A0020AE
:106F2000E80300201C7B020028480200094B011FD7
:106F30009A680948914204BF00229A601A6A9142F5
:106F400004BF00221A629A6B914204BF00229A6326
:106F50001AF0E7BF381A0020B40600202DE9F74FD9
:106F6000804608460C46FCF73DF8182343432C4E58
:106F70000546F21891680191E16808F14C00D0E8EB
:106F8000AF0FC00709D42749274819F0AAF96FF0B5
:106F90001509484603B0BDE8F08FE068007810712D
:106FA0000022F2500B78D22B0FD1D8F800302146B6
:106FB00018681AF0B1F8814638B11C491A4819F01E
:106FC00090F92046FCF7AEF8E3E7182303FB0563CE
:106FD000E768D4F814B0B4F810A0C3F80880002310
:106FE00021461A4608F10400FFF792FD8146002869
:106FF000CFD010F1690FA7EB0B0703D10C490A485A
:1070000019F06FF96269019B12FA87F7182255434C
:107010007219E760A4F810A0936046F80590B8E7ED
:10702000381A0020457B0200284802005F7B0200DE
:10703000727B020010B5044600F14803D3E8EF1F4D
:1070400041F00101C3E8E21F002AF7D1201F19F027
:10705000CCF804F1640004491BF06DF92068BDE828
:10706000104001F055BF00BF8980000073B50E4687
:10707000438D418B01328B4228BF0B469A42054615
:1070800009D9022100921C481C4A18F083F80024F8
:10709000204602B070BD3046FFF7DCFE6FF01403EF
:1070A000034113F001030ED014F0D6FF144BD3F8B4
:1070B000803083421DD0134B1B681A1A18BF4FF043
:1070C000FF32134600E0104A00211048FFF7DEFCB3
:1070D00004460028DCD0FBF785FF18220C4B012169
:1070E00002FB003304F10C009D6018F079FA067081
:1070F000CEE70022E5E700BF28480200957B0200AA
:10710000B8170020801A00201C4E0E0054070020E3
:10711000381A00202DE9F04106460D4690461F46DC
:10712000C9B104220121FFF7A1FF044628B9BDE837
:10713000F0410A490A4819F0D4B804210C3018F07B
:107140004FFA0570A0F80180C77021463046BDE8AF
:10715000F04119F0CAB8BDE8F08100BFBA7B020067
:1071600028480200F0B51D4603680E460039044663
:1071700018BF012187B01868174619F0F6FD48B905
:1071800004F14C0019F016F900280CBF1220002061
:1071900007B0F0BD002D40D01822002168461CF039
:1071A00075FB67B1002213212046FFF75FFF0190B6
:1071B00028B91B481B4919F094F81120E8E7236807
:1071C00029461B68284600930023ADF812300C9B1B
:1071D000154A0393BDF834308DF80860ADF81030CF
:1071E00001238DF814306B4619F08DF89DF814309A
:1071F00063B14FB10198FBF795FF2A46314620460F
:107200009DF81430FFF786FF0020C1E7019900299F
:10721000FAD0204619F069F8F6E70120B8E700BF78
:1072200028480200D77B02006F0202002DE9F341DB
:107230000B8A04460E463BB929492A4819F051F8F1
:10724000002002B0BDE8F0810568012106F10C00C4
:1072500018F0F6F96B7B0746072BF1D154F8043C84
:10726000002BEDD0002203781F4D043C15F83200AE
:107270004FEAC208984205EBC20114D1328A48781D
:10728000904226D90121009316481346174A17F059
:1072900081FF04234544AA78012AD1D1002BCFD005
:1072A0000022397811E001320C2ADFD1104A022184
:1072B0000C4817F066FF39780846FFF7CBFD21220E
:1072C000C24012F00102BBD106232046FFF722FF85
:1072D000B6E74B682046314698470346DAE700BFD9
:1072E000F07B020028480200AC4D0200257C020021
:1072F0000B7C0200F8B5124A0746002311480E46DF
:1073000018F0FEF8044638B9012133460E4A0F48FA
:1073100017F037FF2046F8BD09210C3018F055F959
:107320002046FBF75FFE1822094B012102FB0033C8
:1073300004F10C009F6018F053F90670EAE700BFF3
:107340001C4E0E0054070020B879020028480200A5
:10735000381A00202DE9F0410C7C0546043CE4B2CB
:10736000022C08468CB001D0102C6FD104210C30B7
:1073700018F066F90DF1080806884788011D2246B5
:10738000404618F0E9F9002862D0002E3DD0002FC9
:107390003CD0B74239D300244FF42053404601A9D2
:1073A0008DF80440ADF8063018F0A9F9002838D15E
:1073B0001422002107A81CF069FA11212846FFF7C2
:1073C00099FF099000283FD001210C30CDE90758E2
:1073D00018F006F94FF000080A90394680F800804E
:1073E00007AB30461B4ACDF82C8018F08CFF0A9B67
:1073F00009991C7824BB0846FBF794FE0A23324601
:1074000010212846FFF786FE07E0374601233A465B
:1074100010212846FFF77EFE002420460CB0BDE870
:10742000F08142F60103404607A98DF81C40ADF8F3
:107430001E3018F064F90028BAD010233246E7E76E
:10744000284618F052FFE7E71124E6E70424E4E7B2
:107450000E24E2E7B97900002DE9FF4103680446F4
:107460000E461868012119F080FC50B904F14C0057
:1074700018F0A0FF002814BF0020122004B0BDE8BF
:10748000F0811022002168461CF000FA21212046DC
:10749000FFF730FF029038B34FF00108009406F177
:1074A0000C07338A012B04D82046029918F01DFFDF
:1074B00018E0384618F0D4F86B4601460B4A0546EA
:1074C0008DF80C8018F01FFF9DF80C30002BE8D0D1
:1074D0000298FBF727FE2A46202120469DF80C3013
:1074E000FFF718FE0020C9E71120C7E7D305020007
:1074F0002DE9FF41036804460E461868012119F082
:1075000034FC50B904F14C0018F054FF002814BFAB
:107510000020122004B0BDE8F0811022002168464E
:107520001CF0B4F90F212046FFF7E4FE029038B3B7
:107530004FF00108009406F10C07338A012B04D8A0
:107540002046029918F0D1FE18E0384618F088F865
:107550006B4601460B4A05468DF80C8018F0D3FEA9
:107560009DF80C30002BE8D00298FBF7DBFD2A4693
:107570000E2120469DF80C30FFF7CCFD0020C9E716
:107580001120C7E75F060200F0B51E4603680546F6
:107590000F4685B001211868144619F0E6FB50B972
:1075A00005F14C0018F006FF002814BF0024122437
:1075B000204605B0F0BD76B31022002168461CF0CD
:1075C00065F921462846FFF795FE029008B3BDF8FD
:1075D00028303146ADF80430012330468DF80C30A8
:1075E0000E4A6B46009518F08EFE9DF80C400299ED
:1075F0005CB10846FBF796FD3246394628469DF8B1
:107600000C30FFF787FD0024D2E7284618F06DFE06
:10761000CEE71124CCE70124CAE700BF5F060200D1
:107620002DE9F0410C7C0546043CE4B2022C0846EE
:107630008CB001D0102C7AD104210C3018F000F855
:107640000DF1040806884788011D2246404618F0BF
:1076500083F800286DD06EB36FB3BE422AD80121E3
:10766000686819F082FB044680BB42F602038DF87D
:10767000000069464046ADF8023018F040F828B3E3
:1076800042F60303404606A98DF81840ADF81A30BB
:1076900018F035F8D0B1012E03D14FF6FF739F4299
:1076A00014D005F14C0018F085FE002814BF00240A
:1076B000122407E0374601233A4608212846FFF7FF
:1076C00029FD002420460CB0BDE8F08118220021DD
:1076D0000DEB02001CF0DAF809212846FFF70AFE3C
:1076E000089010B301210C30CDE9065817F078FF4F
:1076F0004FF000080A230990394680F800800E4AAE
:107700008DF82C30304606AB18F0FDFD9DF82C406E
:10771000089934B10846FBF705FD32469DF82C3038
:10772000CBE7284618F0E1FDCCE71124CAE7042492
:10773000C8E70E24C6E700BF717A00002DE9F043C8
:1077400088460446062187B008F10C0017F078FF40
:107750000588D5B14688CEB1B54216D800238288B7
:107760008DF800308DF804304FF42053684601A99D
:10777000D8F80C90ADF80220ADF8063017F0BFFF36
:10778000074670B10A232A4602E02E4601233246FC
:1077900006212046FFF7BEFC0026304607B0BDE8B4
:1077A000F0830146142201A8B8F810801CF06EF88E
:1077B00007212046FFF79EFD0290D8B10A233146EB
:1077C0008DF8153028460C4A01ABCDE903790194B8
:1077D0008DF8148018F097FD9DF8156002992EB170
:1077E0000846FBF79FFC9DF81530CCE7204618F0C3
:1077F0007CFDD2E71126D0E7697800007FB5CB6821
:1078000004461D8885B15E887EB1B5420CD8102231
:10781000002168461CF03AF805212046FFF76AFD72
:10782000019058B9112007E02E4601233246042169
:107830002046FFF76FFC002004B070BD6B46314658
:107840002846084A009418F05EFDDDE901132BB9C3
:107850000846FBF767FC0A232A46E8E7204618F0AB
:1078600044FDE8E7330102002DE9F04342F601034D
:10787000002591B0166880460F4600680BA9D6F81F
:10788000049014468DF82C50ADF82E3017F037FFC9
:1078900000286AD04FF42053D8F800000BA98DF8C7
:1078A0002C50ADF82E3017F02AFF38B1A3681BB169
:1078B0005A88BA4200D25F80012035E061680846EC
:1078C00018F01FFC728D738B9A4294BFC0EB0200BC
:1078D000C0EB0300032826D9084617F047FE0546EB
:1078E0006168084618F00DFC6B8A2A8AA3EB020C2B
:1078F0006B69EA68D21AACEB0203B6F81AC0728D53
:10790000944594BFC0EB0C00C0EB0200834228BF3B
:10791000034683B9887AFBF75DFB0022002317F04A
:10792000EFFD054618B9002011B0BDE8F08301460F
:10793000606817F02CFE00230093D8F80460102331
:107940004146484602AAB047061E0EDB227CE0688C
:10795000B24226D001460BA817F0FEFE40B9237CA8
:10796000124A0221124817F00CFC0023A360A3E77F
:10797000F2B202A906A817F0EFFE10B90D4A33467D
:10798000EFE706A90BA817F0BAFE0028EDD1607446
:10799000042105F10C0017F023FEA0600780A36806
:1079A00089E702A91BF07AFFEFE700BF447C0200E1
:1079B00028480200637C02002DE9FF414FF00008D7
:1079C0004FF4205305460E46006802A91446176876
:1079D0008DF80880ADF80A3017F091FEA0B142F69C
:1079E0000103286803A98DF80C80ADF80E3017F05C
:1079F00086FE48B123691BB15A88B24238BF5E8007
:107A0000012004B0BDE8F0816168286817F077FEB6
:107A100010B100232361F3E7E368A0681A786AB124
:107A2000B7F81AC0798D038A8C4594BFC3EB0C0359
:107A3000C3EB0103934201DA0020E2E704210C309A
:107A400017F0CEFD20610680236929465E80074B32
:107A50000194009338460023A26818F033FD0028F3
:107A6000EADB2069003818BF0120CAE74F02020094
:107A70002DE9F347176805468A460068516816469F
:107A8000D7F8049017F03BFE804600284BD1952292
:107A90002946484619F0F1F80446307548B1F368B4
:107AA0001C7814B1444686F81480204602B0BDE824
:107AB000F0872946484619F0A0F910B90823337514
:107AC000F3E7B068347517F051FD02210C3017F060
:107AD00087FD164B3061A0F800A000930196234665
:107AE00029463846B26818F0EDFC002806DA10F591
:107AF000807F94BF0E2040423075D6E73369002B5B
:107B0000D3D0B06818F0FDFA7B8B7A8D9A4294BF7F
:107B1000C0EB0200C0EB0300F3681B78984294BFEF
:107B200000240124C1E70124BFE700BF13010200C4
:107B30002DE9F04182B000AF0446884600220023C0
:107B400039463A4813F0EAFA0546B0B16D4688B0B6
:107B5000374B6A46CDE90534032342F8103F002332
:107B60004FF4C2513348FAF745F8AD466FF00B06B3
:107B700030460837BD46BDE8F08114F06DFA2E4B53
:107B800024221860294638681BF080FE3B680022DA
:107B90001C603C680023C4E90155C4E90755274827
:107BA000391D7D6013F0BAFA064688B123686C4629
:107BB00088B0234ACDE905236A46032342F8103FE3
:107BC0004FF4C4512B461B48FAF714F8A546CDE7ED
:107BD0000146A02278681BF059FE7868194B836033
:107BE00054301AF05CFA7B684C33D3E8EF2FC3E8CB
:107BF000E16F0029F9D17B681C60E3697D681BB9DE
:107C000004F10C001AF04BFAE26905F19803C5F88B
:107C10009820226AE36102B9236217227B685A85A1
:107C20005A830433C8F80030A2E700BF980600204A
:107C3000827C020028480200801A0020B40600203E
:107C4000A77C0200C003002010B5437B072B07D0A0
:107C500002210F4A0F4817F08CFA0024204610BD6D
:107C6000042118F03AFA044620B90B49094818F0E3
:107C700038FBF3E700F14803D3E8AF3FDB0704D458
:107C80000649044818F02DFBE7E750F8044CE5E7F7
:107C9000CC7C020028480200DA7C0200457B02000E
:107CA0002DE9F04F85B000AF7860EFF31186202307
:107CB00083F31288BFF36F8F584C204618F017FAE1
:107CC00023680546FB6086F31188BFF36F8F002899
:107CD0005FD0FBF787F9182202FB00F35049C81860
:107CE00051F8039003690021D0E90246BB6090F887
:107CF0000480B0F806B01BF0C9FDA87AFBF76AF95A
:107D00006969824651B16A7AD00705D4DAF81C2035
:107D1000284612689268904700226A6129465046B8
:107D20001AF0FDF9B8F1000F0DD064B1236853B11A
:107D30001B6843B1B9F1000F2FD001214B46394ADE
:107D4000394817F01EFAFB681BB3002079681AF057
:107D5000C1FA00281DDA6C468AB0344B6A46059396
:107D6000334BCDE906304FF40073ADF82030314B82
:107D700042F8103F00234FF411512B48F9F73AFF16
:107D80000023A54683F31188BFF36F8F03231846A2
:107D900002DF1437BD46BDE8F08F4046FFF75AF8C2
:107DA0000546201D18F08DFC052DCCD801A353F8F5
:107DB00025F000BFF77D0000CD7D0000477D00006D
:107DC000F77D0000477D0000CD7D000004F14C03ED
:107DD000D3E8AF3FDA0704D41749134818F081FA03
:107DE000B1E7236D002BAED00023144A04F16800E4
:107DF00013F076FDA7E754F84C3B1D68D4E8AF3F7D
:107E0000DB07E9D5002E9ED0002403E02846B968A0
:107E1000B0470134A3B25B45F8D394E7301A002091
:107E2000381A0020F57C020028480200147D020068
:107E3000BB86020004000001457B02001C4E0E00C0
:107E4000F8B50F461646FFF7FFFE68B1C469204635
:107E50001CB150F8984904B1983C731C30B9022108
:107E60000E4A0F4817F08DF90020F8BD458B428D62
:107E7000954228BF15469D4204D24CB9254620465E
:107E80002C46EBE732463946BDE8F840FFF7EEB83E
:107E9000D4F89850002DF2D0983DF0E72F7D0200E5
:107EA00028480200002337B505460C46019314F01C
:107EB000D3F80E4B1B68834204D00D4BD3F88030AF
:107EC000834201D100252C4601A92A4623460948B0
:107ED00013F024F9014630B91C2201981BF0D6FC9E
:107EE000019803B030BD0020FBE700BF801A0020DE
:107EF000B8170020D006002010B50022044600F17B
:107F00000803D3E8EF0FC3E8E12F0029F9D108B146
:107F1000FBF708F92146BDE8104001481AF001B806
:107F2000D00600202DE9F743044668301E460F4670
:107F300090461AF00BFA236D53B90221144A1548E2
:107F400017F017F9204603B0BDE8F04300F084B8FD
:107F5000114A93424FF0000217D05D685A60206DBD
:107F6000D0F81890FFF7C8FF00232068236518F0A9
:107F7000D9FB3DB12068CDF8009043463A463146E2
:107F80000068A84703B0BDE8F0831546ECE700BFE2
:107F90004A7D020028480200841A0020F7B550F8F4
:107FA000044C0546002C52D000F1940104F11C0051
:107FB00018F0E7F90022002305F1500013F09CF9B6
:107FC000014650BBEB6C2BB102466FF06703281FD4
:107FD000FFF7A8FF002345F8043C05F14803D3E868
:107FE000EF1F21F00101C3E8E21F002AF7D1E36986
:107FF0006BBB0022002304F10C0013F07DF978B96B
:10800000666886B921461348266019F08AFF2868F9
:1080100003B0BDE8F04000F0D3BFFBF783F8C9E739
:10802000FBF780F8E5E7A26833689642636008BF13
:10803000A36077683FB1B3696FF0670100930023D5
:1080400020681A46B8473046FFF756FFD8E703B016
:10805000F0BD00BF9806002010B504460430FFF7BD
:108060009DFF1321606817F0BCFE034630B1BDE8E8
:1080700010400121024A034817F083B810BD00BF29
:10808000617D020028480200F0B589B0044654F82A
:10809000683D00AF38461968FEF7A2FB6E4688B00F
:1080A0000B4B6A46CDE905374FF40073ADF81C3031
:1080B000084B42F8103F00234FF4E2510648F9F70D
:1080C00099FD2046B546FFF7C7FF2437BD46F0BDF2
:1080D0007F7D0200030000012848020070B550F8BF
:1080E000043C0446002B3CD0051F39B1C36C002B67
:1080F00037D01B7CDA0734D505231CE006683046F0
:1081000000F04AFF737A012B2BD0E46C4CB3237C34
:10811000DB0726D5E368002BEED028466269617C38
:10812000FEF7A4FF064668B9637C01210D4A0E489C
:1081300017F027F80E2300222846BDE870401146AC
:10814000FFF7F0BEE368D4E90512984718B130464E
:10815000FAF7E8FFEEE731462846FEF7FFFE002873
:10816000F5D170BDAB7D020028480200F8B51D4670
:108170000F461646FAF736FF1823044C03FB00405F
:108180000123C0E90376C3800575F8BD381A0020C5
:1081900008B51AF0EAFD38B101210346034A044844
:1081A00016F0EFFF6FF0040008BD00BFD27D0200A3
:1081B00080480200F8B5074600260A4C2546621C96
:1081C0005FB91046084918F0E9FB10B9103416B130
:1081D00005462846F8BD0126F0E73846217817F015
:1081E00071FEF2E7B81A0020D385020070B50E4C7C
:1081F000054623780E46834203D1601C18F0CEFB5F
:1082000080B9237BAB4201D0002070BD31460748C6
:1082100018F0C4FB0028F7D001235B4203F00C03E5
:10822000E018F2E70023F8E7263800203338002072
:10823000F8B507464C1C01F11505661E67B12246CC
:10824000384614F8011C17F03DFE18B90A34AC4248
:10825000F3D106463046F8BD2046024918F09EFB91
:10826000F3E700BFD3850200024608B50749013095
:1082700018F0A7FB00230C3202F8043CD2E8EF1FF1
:10828000C2E8E03F0028F9D108BD00BFD385020055
:10829000F8B5154607460E461C46FFF7A7FF0246EF
:1082A00080B91249FFF7A2FF024630B9BDE8F84095
:1082B00001210F4A0F4816F05CBF314600F8017BE0
:1082C00018F07FFB138923B9518921B91581548195
:1082D000F8BD9D4204D35189A142F9D29D42F6D204
:1082E00053891581A342F3D2F1E700BFD385020081
:1082F000E87D0200804802002DE9F047264B174632
:10830000826880469A4227D1C568AB8A23B300268B
:108310006C1C05F1150AB4F807309BB122463846AB
:1083200014F8011C17F0CEFDC8B9214614F8010C51
:10833000FEF7E0F930B1437B072B08BF46F001069A
:10834000FDF79EFD0A345445E5D12EB9AB69AE82E6
:1083500013B13146404698470120BDE8F087387A8E
:1083600007F1700117F016FB78B90C4B9D4202D152
:10837000384618F0BEFB2046094918F022FB0023BE
:1083800004F8013CA4F80730DCE7204607F170014F
:1083900018F017FBD6E700BFA583000010040020EB
:1083A000D38502002DE9F8431F46BDF820308146F1
:1083B0008846002B41D17B1E012B41D8CE68012F6E
:1083C00031460CBF15781588FFF732FF0446C0B957
:1083D00015B93846BDE8F8833146FFF729FF044652
:1083E00038B91A4802211A4A16F0C3FE6FF010007D
:1083F000F0E709F17001013018F0E3FA99F808305C
:108400002370F36943B12A464146484698470028FD
:10841000E0DB0138012816D82581B38AAB4203D0AE
:108420003146404618F0D4FA002DD2D10949601CDB
:1084300018F0C7FA25702581CBE76FF00600C9E771
:108440006FF00C00C6E76FF00D00C3E78048020034
:10845000077E0200D3850200F8B51F46BDF818302C
:108460000546012B164632D83B44012B3C4631DCF5
:10847000FFF7A0FE024660B9FFF79CFE024640B936
:108480000221174A174816F074FE6FF010042046B8
:10849000F8BD8FB10023117A21FA03F0C70703D585
:1084A0003078D840C00718D50133032BF4D1337886
:1084B00003F0070319431172501C05F1700118F005
:1084C00080FA2B7A1046137018F039FBDFE76FF053
:1084D0000604DCE76FF00C04D9E76FF01204D6E76E
:1084E000217E02008048020010B504461149D1E8FF
:1084F000EF3F23F00203C1E8E23F002AF7D108462C
:1085000018F0F6F9C20705D500220023A1F13000CA
:1085100013F0E6F9204618F0AAF950B12046FFF70B
:1085200049FE30B1037ADB0703D5BDE8104018F0EF
:1085300006BB10BD80100020012110B5144818F0B2
:1085400035FAC30722D40221114818F02FFA084047
:1085500007D11049104B0A88104CA34211D300B127
:108560000A800F490F4819F0E6FE40F23912002345
:108570000C48FAF7E9FEBDE810400B490B4819F02A
:10858000DABE9888083302440120E6E710BD00BF38
:10859000D81A00203E380020084802002048020077
:1085A00021880000E00F0020898B0000501000207F
:1085B0002DE9F04130B3078A3FB901244FF0140C84
:1085C000114ADFF848E0724503D33B461846BDE840
:1085D000F081D2E90065B04204D36B1E0CFB03634B
:1085E00098420DD963191C460832ECE70CFB016870
:1085F0004045EBD0013163188D429BB2F6D1F2E7D2
:108600000021F8E70346E1E708480200204802009D
:108610002DE9F74F9A464FF6FF73BDF8305080466C
:10862000002D08BF1D46234B91461B8800918342B5
:108630003AD203B0BDE8F08F73682344434531D28A
:108640009CB208361C4B9E42F6D3F2E74846895846
:10865000019317F054F8019B88B101340137A4B29B
:108660007368BB42EDD9009B9C42E2D84445F4D3E9
:108670000BFB07F231688B18B9F1000FE6D1BAF1A4
:10868000000F0BD1013D1846ADB221460E9A0D9B4D
:108690009847002DCDD00028DFD1CAE7DA6892458F
:1086A000DBD1EFE70027DBE701244FF0140B034E8B
:1086B000C8E700BF3E3800202048020008480200FA
:1086C00010B59EB01022002168461BF0DFF814227E
:1086D00000210DEB02001BF0D9F84FF41053ADF858
:1086E000103080231022ADF812304FF48063284CF4
:1086F0006946CDE906340DEB02001CAB1AF041FAD5
:10870000034630B1234A0121234816F03AFD1EB03A
:1087100010BD014648220AA81BF0B8F822461C9951
:108720000AA81AF01FFB034660B101211B4A1A4830
:1087300016F027FD1C981AF05CF903460028E6D0D5
:10874000174AE0E74FF6FF710120164A0AAB18F00E
:1087500075FA1022144904AB0AA81AF01EFB04464D
:108760001C981AF046F914B1104A2346CBE721466B
:108770000D4B03F11002187812F8014D0131082950
:1087800003F8014B1070F6D1094818F00FF9BEE755
:108790000002C0034D7E020080480200767E020087
:1087A000947E0200F7080200D00F0020AA7E02008B
:1087B000801000202DE9F04116490746A1F1300054
:1087C00014461D46BDF8186019F0D7FD124818F080
:1087D0008FF8000701D4FFF773FF3846FFF7EAFC74
:1087E00068B1037AD9070AD500F10C03184618F0CE
:1087F0007FF8C20703D40221184618F0D7F81023D7
:108800003246069329462046BDE8F041034B18F056
:1088100004B900BF1010002080100020D00F0020ED
:1088200008B5054818F064F8030703D4BDE808400C
:10883000FFF746BF08BD00BF80100020002307B52A
:108840000193FFF7B5FE411C89B20846034A01AB0C
:1088500018F0F4F9019803B000BD00BFB30802009E
:108860002DE9F04387B0437B8046072B0C46154625
:108870004FF0000002AF40F0A28042F603033873CD
:1088800007F10C012068FB8116F039FF064600282D
:1088900035D1D4F80490B9F1000F05D101214A4A2D
:1088A0004A4816F066FC89E001232146009007F152
:1088B0000802C847031E11DA6D4688B009930423E5
:1088C000434ACDE9072402AA42F8103F4FF4015170
:1088D00033463E48F9F78EF9AD466FE0012B05D0DF
:1088E00001213C4A394816F04CFC67E03B7A03F022
:1088F0003003002B62D02046FFF7A0FF0446002380
:1089000020683B7342F6021307F10C01FB8116F05D
:10891000F6FE18B12046FFF791FF0446002642F606
:108920000219206839463E70A7F8029016F0E7FE5B
:10893000E0B142F603032068391D3E71FB8016F05A
:10894000DEFE98B14FF42053206807F108013E7213
:108950007B8116F0D4FE48B142F60103206807F18E
:108960000C013E73FB8116F0CAFE08BB0023206891
:108970003B7342F6021307F10C01FB8116F0BFFEB8
:108980000646D8B9D4F80490B9F1000F86D0022376
:1089900000902146404607F10C02C847031E8BDBBE
:1089A000022B9DD1BB891D4214BF0120002006E08F
:1089B0002046FFF743FF04460028B2D100201437B9
:1089C000BD46BDE8F08300BFC07E020080480200C3
:1089D000D47E0200FA7E02002DE9F843154688464F
:1089E00094226968074618F048F90646002843D1E2
:1089F000022238466968FFF733FF00283FD0002184
:108A00002048B5F81490FFF74DFA044620B96FF0EE
:108A10000B052846BDE8F8831D211B4B09F1020216
:108A200041744261C660436085613846FFF708FAC9
:108A3000814618B92046FFF75FFAE8E7012332467E
:108A40003146FFF793FBA98A09F10C00023116F0B9
:108A5000C7FD20F8028BAA8A29691AF0F0FE214688
:108A60003846C4F8089017F0E5FE05460028D0D037
:108A70002046FFF741FACCE74FF0FF35C9E76FF02A
:108A80001505C6E71C4E0E00B908020070B5054674
:108A90008AB03A4817F02CFF42070C4667D515B14B
:108AA0006B7B072B66D1666830460596FFF780FD25
:108AB0002268ADF8180032B305A9029130490023AD
:108AC0000191012100914FF6FF710593FFF7A0FD81
:108AD000059E1EB96FF001000AB070BD66600023EC
:108AE00030688DF8103042F6030304A9ADF8123057
:108AF00016F005FE70B90598C3689B799B0605D4EE
:108B00006FF01500E8E70028E9D1E3E718F04FF827
:108B1000ADF81800059818F09BF860600028EFD0B9
:108B2000BDF818003DB10123014622462846A37531
:108B3000FFF752FFD0E76FF07F0307930223ADF8F2
:108B4000203042F60213ADF8123005ABA575029342
:108B50000C4B4FF6FF710193012304AA00932B469F
:108B600009948DF81050FFF753FD0798B4E76FF0A4
:108B70000A00B1E76FF07F00AEE700BFD40000202D
:108B8000E9080200FD8D0000034613B550F8082CDB
:108B9000A0F12001019200F13004D4E8EF2F22F07F
:108BA0000102C4E8E02F0028F7D10D4A002043F865
:108BB0001C2C0C4A23F8080C43F8182C01AA43F883
:108BC000102C042223F8060C23F80C2CFFF75EFF70
:108BD00018B90221204617F0E9FE02B010BD00BF0F
:108BE000484E0200E98400002DE9F84F91463D4BC4
:108BF000826806469A4200AF70D1D0F80C80D9F84E
:108C0000004008F1010508F1150AB5F80730F3B185
:108C10002A46204615F8011C17F054F9B8B14FF454
:108C200095723146204618F028F830B3032812D147
:108C3000EB4688B06A462C4BCDE9053642F8100F5A
:108C400000234FF4C4512948F8F7D4FFDD460A3514
:108C5000554543D0D9E7052820460CBF4FF0030BFC
:108C60004FF0020B17F028F9834506D999F8043024
:108C70005B45ECD289F804B0E9E74146304617F08D
:108C8000A7FE1B4B984529D1207A04F17001FFF70C
:108C9000ADFA054610B303890BB94389F3B12046F9
:108CA000FDF746FA2A89134B134923F820206A89D5
:108CB00003EB80035A80182202FB00110B6104238E
:108CC0000E4A20464A600E4A8B828A60FFF7DEFE1B
:108CD00020B101210B4A054816F04BFA0120BD4690
:108CE000BDE8F88FA5830000137F020080480200D2
:108CF0001004002022380020A01A0020484E020054
:108D0000470B0200277F020070B504468AB038483E
:108D100017F0EEFD42070D4663D514B1637B072BB8
:108D200062D16E6830460596FFF742FC2A68ADF8BE
:108D3000180032B305A902912E49002301910121A7
:108D400000914FF6FF710593FFF762FC059E1EB977
:108D50006FF001000AB070BD6E60002330688DF8BE
:108D6000103042F6030304A9ADF8123016F0C7FC28
:108D700070B90598C3689B79DB0605D46FF01500C0
:108D8000E8E70028E9D1E3E717F011FFADF8180094
:108D9000059817F05DFF68600028EFD0BDF8180057
:108DA0002CB101462A46204617F0A8FFD2E76FF003
:108DB0007F0342F6021207930123ADF8122005AAA1
:108DC00002920D4AADF82030CDE900324FF6FF7126
:108DD000234604AA09958DF81040FFF719FC07985F
:108DE000B8E76FF00A00B5E76FF07F00B2E700BFA9
:108DF000D4000020E9080200FD8D00002DE9F84FA5
:108E000014463F4B826882469A4204D04FF00108D4
:108E10004046BDE8F88FD0F80C903A4B994518D1F0
:108E20000026394D2846394917F0B8FD78B9072290
:108E3000294615F8010CFDF7AFFC28BB236929462C
:108E40001A6915F8010C53881288FFF721FA0C35BE
:108E5000C6B109F1010609F1150BB6F80720A3897F
:108E60009A420BD1314616F8010CFDF743FC074638
:108E700020B1437B072B0AD0FDF702F80A365E4586
:108E8000C4D0EAE70126CDE7FCF7FAFFDFE7D9F81F
:108E9000203023B15146984708B93846ECE7942270
:108EA0005146384617F0E9FE80460028F5D1A389DF
:108EB000022B15D1B6F807309A0713D53846226928
:108EC000A188FFF789FD054618B92269937D013312
:108ED00093753846FCF7D4FF002DA560CEDA97E7EE
:108EE000012B01D00025F4E7B6F80730DB07F9D5F0
:108EF00038462269A18817F001FF0546E9E700BF5F
:108F0000A58300001004002027380020D38502002C
:108F100013B50446009001204FF6FF716B460C4AD2
:108F20008DF8040017F08AFE204616F0C5FF9DF864
:108F30000410884209D2204616F08DFF034620B166
:108F40000221044A044816F01CF902B010BD00BF0B
:108F5000E98B0000447F0200804802002DE9F041C7
:108F60000C4B06461B680F46904683B153F80449E4
:108F700004B1043C1B681BB1424639463046984751
:108F80002CB1656805B1043D23462C46F2E7BDE8E7
:108F9000F08100BFDC1A002013B5044600900120C8
:108FA0006B46064A4FF6FF718DF8040017F046FE37
:108FB0000021204617F0D9FE02B010BDE98B000059
:108FC00070B5044603464FF6FF7101200D4A17F0B5
:108FD00035FE2046FFF7EEF8054688B1207A04F109
:108FE000700116F0D7FC20B92846BDE87040FFF7A5
:108FF0003BB904F17001681CBDE8704017F0E1BC9A
:1090000070BD00BFF98200007FB54FF420520023ED
:10901000ADF8162004AA0292094A0120CDE90032D7
:109020004FF6FF7105AA04938DF81430FFF7F0FA9C
:10903000049B012B14BF6FF01500002007B000BD8A
:10904000030E0200014608B5034817F0F1FE0028A0
:10905000024808BF002008BD8C10002088100020A6
:10906000084B00F5B4701A68074BD0E8EF1F99421F
:1090700004D1C0E8EC2FBCF1000FF6D1D0E8AF0F5F
:10908000704700BFE41900208810002008B5FFF7E2
:10909000E7FFE8B1036883B1426872B182680AB140
:1090A000042008BD0C4A1278002AF9D042688AB917
:1090B000934214BF10460320F3E7074A1278002AB0
:1090C000F4D0002BF2D08268002AEFD00120E8E72C
:1090D0000320E6E70220E4E7653A002010B5062108
:1090E00016F0FBFF044630B90121044A044816F08B
:1090F00040F8204610BDA0F1EC04FAE7787F0200AA
:10910000B048020038B50546EC2200211AF0BEFB3B
:10911000102105F127000CF029FF044648B905216C
:10912000284617F0CCFEFCF78FFC034B1860204656
:1091300038BD0824FBE700BFE41A002070B5041D09
:109140000E462046042117F073FE68B1002200216C
:1091500000230846FDF79AFC054638B9042120464D
:1091600017F0ADFE284670BD034AF0E701210C3030
:1091700016F036FA0670F5E71C4E0E0038B50446B8
:109180000D494C3019F0D7F8A4F1EC0017F0BFFEF0
:109190000A4A04F17C03D3E8EF1FC3E8E02F00285C
:1091A000F9D14FF0FF338034D4E8EF2FC4E8E13F2A
:1091B0000029F9D138BD00BFB1A3000088100020FC
:1091C00038B505460821043017F079FE084905F145
:1091D0005700FCF747FC48B10821281D17F062FE34
:1091E00004480121044A15F0C4FF082038BD00BF1F
:1091F0001F110200B0480200937F0200002370B5E7
:109200001A460446EC300D46FDF782FC58B1693031
:1092100004D10121084A094815F0ABFF2846BDE8F2
:109220007040F9F77FBF04F59C700023BDE87040E3
:10923000034A12F055BB00BF727B0200B048020027
:109240001C4E0E0073B5047A0546022C23D844B197
:1092500090F8DC30D0F8D840DC4004F0010444F051
:10926000800403212846FFF769FF0646D8B1102184
:109270000C3016F0B5F9009012482346006805F14D
:10928000270205F1570118F00AF8044680B130466C
:10929000F9F748FF07E0032C08D0012123460A4ACA
:1092A0000A4815F06EFF082002B070BD0024D8E710
:1092B00031462846FFF7A2FF281D214617F0F2FD90
:1092C0002046F1E7E41A0020AC7F0200B04802001B
:1092D00070B504460D4686B0FFF7C2FE04F13702B2
:1092E0001146EB68064603F1100053F8045B834215
:1092F00041F8045BF9D1237A052B00F29A80DFE86C
:1093000003F017242403986C02AB4D4900930968BD
:1093100004F1270304F1570001F01CFA60BB0A2195
:10932000201D17F0CCFDB3680299D4F8EC009847E3
:109330000D21204617F0C3FD1021201D17F0BFFDA1
:10934000204617F0FFFD054617E094F8DC10D4F82E
:10935000D83002ADCB403A4903F0010300950968CB
:1093600043F0800304F1570017F099FF40B1012149
:10937000344A354815F0FDFE0825284606B070BD74
:109380001022294604F117001AF088FA08B10425C2
:10939000F3E70321204617F092FD17F0D3FD0546B1
:1093A0000028E9D194F8DC300133DBB2142B84F8C7
:1093B000DC3008D120460D2117F081FD1021201D41
:1093C00017F07DFDD9E7102104F127000CF0CEFD48
:1093D000003818BF0120C500CFE7102104F1270095
:1093E0000CF0C4FD0028C7D10EB90225C5E7F3680B
:1093F000002BFAD0154BE27A1B8812F0010FADF862
:109400000830A37C08BF0320DB0703D5002814BF66
:109410000120022000258DF809000C21201DC4E93F
:10942000385517F04CFDF368D4F8EC0002A99847C2
:10943000A3E70121064A044815F0A3FE9CE700BFFC
:10944000E41A0020C87F0200B048020080490200F0
:10945000AC7F02002DE9F047044690B00CAD10221D
:10946000002128461AF012FA237A052B32D8DFE8B9
:1094700003F0060303063121D4F8D8300C93D4F856
:10948000EC3004F1470204F1C707CDE9017203F1A2
:109490007E020092773304F1270204F1370104F1D0
:1094A000970001F0F1F8F0B1474A0121474815F063
:1094B00060FE14E0D4F8E430002BE0D02E4603F137
:1094C0001007324618685968083303C2BB42164673
:1094D000F7D1D4E701213E4A3C4815F052FE08205E
:1094E00010B0BDE8F087D4F8EC3008AE03F1770295
:1094F0007E33019304F111030292009338462B4608
:10950000039604F1370204F1270117F0ECFE08B1CD
:10951000304ACAE7237A052B0ED1D4F8E01021B3E4
:109520000B46AC4601F1100E6246186859680833C4
:1095300003C273459446F7D1D4F8EC300DF1100A0C
:1095400003F17E027733019304F10A030292009340
:1095500038462B46CDF80CA004F1270204F1370160
:1095600017F0C1FE30B11C4A9FE7102228461AF0BE
:109570008DF9E1E71022514604F1B7001AF08EF997
:10958000F8B90D212046FFF7D9FD07460028A6D0DF
:1095900010210C3016F024F832460346164603CE4E
:1095A000AE4218605960324603F10803F6D13946DD
:1095B0002046FFF723FE201D012117F080FC00202C
:1095C0008EE70B208CE700BFE17F0200B04802006D
:1095D000AC7F0200F67F02001980020070B5CC68F3
:1095E00005460B21043017F05DFC234605F11702F8
:1095F00004F1100153F8040B8B4242F8040BF9D12B
:109600002B7A012B09D0022B13D12846042117F005
:1096100056FCBDE87040FFF715BE0A21281D17F063
:1096200007FC0028F1D0281D002117F048FC00207D
:1096300070BD03480121034A15F0A3FD0820F7E798
:10964000B0480200AC7F020098B50F4A00AFD2F8D4
:10965000EC3033B90D48EC32506018460A60BD4614
:1096600098BD6C4688B00A4B6A46CDE905300323A5
:1096700042F8103F074800234FF4C251F8F7BAFAF6
:109680006FF00B00A546EAE788100020C04E0200EC
:109690003D800200B04802002DE9F04188B0064646
:1096A0000B4600AF0D21043017F0C2FB90B3DC680D
:1096B000D6F8EC30022003F170084246197A17F010
:1096C000AAFD0546E0B941463846F9F7B5FD6E46B4
:1096D00088B0134B6A46CDE905374FF40073ADF8F7
:1096E0001C30104B42F8103F0F482B464FF4E2510C
:1096F000F8F780FA0820B5462037BD46BDE8F0816E
:1097000022462E3504F1100352F8041B9A4245F804
:10971000041BF9D13046092117F0D1FB0020EBE7FB
:109720006280020003000001B0480200F7B5044661
:10973000FFF796FC0E210646201D17F079FB78B93D
:109740004D4B2022196804F157001AF0A7F838B9D8
:1097500002214A4A4A4815F00CFD082003B0F0BD2A
:109760000C212046FFF7EAFC07460028F5D04021EF
:109770000C3015F035FF02463F4B1B6803F120010A
:1097800053F804CB8B4242F804CBF9D1203003F1DB
:10979000200253F8041B934240F8041BF9D13946C8
:1097A0002046FFF72BFD237A052B5DD8DFE803F079
:1097B00003491A035C590421204617F080FBFFF788
:1097C00041FD0028C9D1201D072117F078FB082092
:1097D000FFF738FC00284DD1204603B0BDE8F0402B
:1097E000FFF7EEBC2046D4F8EC70FFF739FC0421FB
:1097F0004FF0FF3306460DEB010001930CF0B6FB72
:109800000028AAD1019B1F4A84F8DC00B3FBF2F1C7
:1098100002FB11330193C4F8D83056B1336843B119
:109820000B21201D17F04BFB38463368D4F8D810B5
:1098300098470321204617F042FB0E2117F03FFB0B
:10984000C1E72046032117F03AFB0E2117F037FB42
:10985000201D0A2117F033FB7368D4F8EC009847F9
:10986000B1E704212046E9E70121074A044815F041
:1098700088FC72E7002071E7E41A00207C80020077
:10988000B048020040420F00AC7F020070B50546B0
:109890000E4605F15704FFF7E3FB2246F36803F198
:1098A000200153F8040B8B4242F8040BF9D105F167
:1098B000770203F1200153F8040B8B4242F8040BAA
:1098C000F9D12046FCF728F8F0B103211C4A1D48C5
:1098D00015F04FFC281D0E2117F0F1FAD5F8EC40D9
:1098E000D4F8A40038B9207A04F1700100F03AFEEF
:1098F000C4F8A40098B1438A03F024037BB1437CED
:109900009B070CD4032070BD2046FCF711F830B93A
:109910000C4802210C4A15F02CFC0B20F3E70B4BF2
:109920001C682CB9281D062117F0C9FA2046EAE761
:109930002846FFF7FBFE003818BF0120C000E2E711
:1099400097800200B0480200B8800200E41A0020AC
:1099500038B5144B05461B78EBB101F00F042846CF
:10996000FFF794FB104B03281B780CBF04F00B048B
:1099700044F0040405F5B670D0E8EF2F013203D1AE
:10998000C0E8E13F0029F7D1D0E8AF3F33B144F060
:109990000104E0B238BD01F00704E0E704F0FE0086
:1099A000F8E700BF653A002041060020F8B50D46F3
:1099B0000446D0F8EC70FFF753FBED68EB78102B02
:1099C00001D00620F8BDD7F8A430002B5AD00F21C3
:1099D000201D17F02DFA20B92046FFF793FB002831
:1099E00059D1012363722B682046C4F80A30AB8832
:1099F000E38102232374A978FFF7AAFFE0742046CD
:109A0000FFF744FB1023607423752B7903F00303E5
:109A100063756B7903F00103A375E37C1E073CD4E7
:109A20000521201D17F004FA002844D0574B1B785D
:109A3000A374E37C990606D5AB789A0603D5142166
:109A4000201D17F03CFAE37CDB0736D5AB78DE0748
:109A500033D50D21201D17F032FAA37D032184F8A0
:109A6000E830637D201D84F8E93017F028FA237B65
:109A7000E17C03EA0102100723D42D78042D27D9B5
:109A8000002331E0387A07F1700100F06BFDC7F870
:109A9000A40000289BD1082094E7AB781807BFD515
:109AA0000521201D17F00BFA637D03F00203637597
:109AB0000023A375B4E7364BB9E700236375A3759C
:109AC000CBE7E27AA07C0243D207D6D505230BE090
:109AD0000B4313F0040307D02046FFF7D7FA2D4BB2
:109AE00005EB85052B441B5C23722046D7F8A41098
:109AF00017F0A4F908B9032064E7D4F8EC309B7A96
:109B0000032B33D022D8013B012BC4D80521201DC3
:109B100017F08EF90028EED00C21204617F0CFF96F
:109B20000221FFF70BFB05460028B4D006210C30BC
:109B300015F056FDD4F8113029460360B4F81530FD
:109B400083802046FFF75AFB00203BE7042BA2D17D
:109B5000237D627B934228BF1346102B7FF431AFE5
:109B60000521201D17F064F90028C4D0237A002BAA
:109B7000C1D00521201D17F05BF90028C6D1237A3A
:109B8000013BDBB2012BC1D8B5E700BF673A00202B
:109B9000663A0020F78602002DE9F041C7780446B6
:109BA000012F04D06FF015042046BDE8F081FFF7C7
:109BB00095FA0546002800F0A7800421043017F02C
:109BC00037F9002840F0A3800321281D17F030F951
:109BD00010B16FF00F04E7E73946281D17F028F998
:109BE0000028F6D12846FFF73BFAD5F8EC300746B7
:109BF0009B7A032B43D033D8013B012B49D90F214A
:109C0000201D17F015F90028CCD1D4F8A40090B984
:109C100004F170073A462020217A00F0DDFCC4F8F8
:109C2000A40040B93A460420217A00F0D5FCC4F8DB
:109C3000A4000028B6D0438A03F02403002BB1D03F
:109C4000A37A022B25D9427CD207ABD5032B20D097
:109C50000269324B9343A5D1037C102BA2D118E0AB
:109C6000042BCCD12846FFF711FA032804D1002F8A
:109C7000C5D0FB68002BC2D0294B1B7807E02846D3
:109C8000FFF704FA032804D1002FB8D0FB68002B9B
:109C9000B5D0D4F8A4303BB9207A04F1700100F0BB
:109CA00061FCC4F8A400A8B32846FFF72BFA0446C9
:109CB00010B16FF0680477E70B212846FFF73EFAF2
:109CC00007460028F5D001210C3015F089FC092148
:109CD00080462846FFF73CFE2346224688F80000CF
:109CE000394605F1EC00FCF713FF044618B138467D
:109CF000F9F718FA58E7281D0F2117F0E0F80121AD
:109D0000284617F0DCF84FE76FF07F044CE76FF060
:109D1000040449E76FF00B0446E700BF0001200090
:109D2000653A0020F8B5D0F8EC400646D4F8A430E7
:109D3000051D002B3FD10221364A374815F019FA8C
:109D40000721364B5F5CD4F8A4306BB11B7C23B188
:109D50000221284617F06CF830B1D4F8A40017F0AF
:109D60006EFA0023C4F8A4300221284617F060F8E8
:109D700048B9072F94BF2A4B1F213A46204698BF67
:109D8000D95DFCF763FC0321284617F051F888B32E
:109D9000244B1B6873B353F80C5905B10C3D5B6839
:109DA00013B139462046984725B3EA6802B10C3A08
:109DB0002B461546F3E7B9B90D21284617F038F8B8
:109DC000184B07461B68ABB153F80C5905B10C3D55
:109DD0001B6813B13946204698475DB1EA6802B165
:109DE0000C3A2B461546F3E70139C9B20E29A8D91A
:109DF0000927A8E7304617F08AF8637B072B08D1BC
:109E0000627AA37A9A4204D02046BDE8F840FFF770
:109E1000C3BEF8BDD4800200B0480200E88602004C
:109E2000D7860200DC190020F8B505460F4604303D
:109E3000022116F0FDFF10B195F8E820B2B1002420
:109E40000321281D16F0F4FFB0B139462846FFF76C
:109E500069FFF4B102211C481C4A15F08AF905215A
:109E6000D5F8EC0015F0BDFF0020F8BD95F8E940ED
:109E7000B4FA84F46409E3E70121281D16F0D8FF41
:109E80000028E2D10F21281D16F0D2FF0028DCD1D6
:109E9000DFE705212846FFF751F9064688B1012181
:109EA0000C3015F09DFB234607702246314605F124
:109EB000EC00FCF72DFE0028D7D03046F9F732F938
:109EC000D2E76FF06800D0E7B0480200FE800200E1
:109ED000144B10B5044618604FF0FF324FF0FF33BB
:109EE000114811F049F9114811F000FD0E4811F028
:109EF000B3F974B10E4CD4E8AF3F5B0610D5201F08
:109F0000FFF714FC60B1201F0821BDE81040FFF7E7
:109F10008BBF0221BDE81040064A074815F029B959
:109F200010BD00BFE41A00203404002048040020C3
:109F30008C10002056810200B04802002DE9F34148
:109F40000B8A0E4643B901212E4A2F4815F011F90C
:109F5000002002B0BDE8F0810121A0F1E805A0F1E8
:109F6000EC0406F10C0015F06BFB0421804628463A
:109F700016F05EFF98F8003028B1244A02212248EA
:109F800015F0FFF8E4E70E2B01D9214AF6E7214F3F
:109F900057F833204AB902211F4A1B4815F0F1F83F
:109FA00007212046FFF740FFD2E71946204616F06A
:109FB0009CFF98F8003060B902211348174A15F049
:109FC000E0F80321284616F033FF0028C0D008210E
:109FD000E7E707EBC301328A0979914208D00121F2
:109FE0000093094813460E4A15F0D4F80A21D8E721
:109FF0003146204657F83330984701460028A7D00D
:10A00000CFE700BF6F810200B04802008A810200E2
:10A01000BB810200E84E0200DD810200F7810200F0
:10A02000257C02002DE9F04F99B090F8E930D1F885
:10A030000C8023F0020380F8E930D0F8EC6098F847
:10A040000030044600AF06F17009002B3CD098F8B0
:10A05000063003F0C003C02B36D041463846F9F72E
:10A06000EBF86E4688B06C464FF4007A6D46634B51
:10A07000DFF88C81CDE90537ADF81CA045F8108FCD
:10A0800000232A464FF4E2515E4807F1200BF7F710
:10A09000B1FD4946B5465846F9F7CEF8A5465A4BA4
:10A0A000A4F81CA0C4E9053BC4F8108000232A468C
:10A0B0004FF4E2515348F7F79DFD0A25B54628466F
:10A0C0006437BD46BDE8F08F07224146484619F087
:10A0D000E5FB68B14146307A00F0C4FA054638B174
:10A0E0000146204616F0AAFE48B3284617F0A7F806
:10A0F0000D21201D16F09CFE002867D04A46022044
:10A10000317A17F088F80546D8B907F14004494676
:10A110002046F9F791F86E4688B03C4B6A46CDE987
:10A1200005344FF40073ADF81C30354B42F8103F46
:10A130004FF4E2512B463348F7F75CFDB54608254E
:10A14000BDE7F378002B3BD106F17E031878012898
:10A150002BD19A7902F0C002402A26D1D3F80120EF
:10A16000C5F83E20B3F80530A5F8423096F87030B7
:10A17000DBB196F8763003F0C003C02B15D024492C
:10A1800007F14002C7E91098BD64FBF78BFFD8F8D0
:10A1900000303046C5F80130B8F80430A5F8053075
:10A1A00098F80630EB71FCF721FA2846FAF70AFD19
:10A1B00048B10221174A134814F0DBFF03257EE75C
:10A1C00006F17703C2E72846FAF70AFD94F8E9306A
:10A1D0005B0703D50A21204616F071FE94F8E8507B
:10A1E0004DB994F8E930002B7FF469AF2946204639
:10A1F000FFF798FD63E7002561E700BF12820200C8
:10A2000003000001B0480200908202006280020058
:10A21000D70F0200268202002DE9F0410D460446C8
:10A22000D0F8EC80FEF71CFFED6806462B78012184
:10A230000F48104A271D14F0A4FF0A21384616F0D3
:10A2400054FE38B16EB920462978FFF76BFD002027
:10A25000BDE8F0810B21384616F047FE0028F1D109
:10A26000F1E73369002BEED040469847EBE700BF9B
:10A27000B0480200618202002DE9F04389B0054632
:10A28000A0F1E8060446884600AF0121304655F8A3
:10A29000EC9916F02AFE38B3B8F1000F19D003215B
:10A2A000304616F0C5FDF8B14046F9F7E9FD013832
:10A2B000C0B208288CBF0024394B4FF0020198BF70
:10A2C0001C5C304616F0FBFD21462846FFF72AFDB0
:10A2D0000AE099F80B303BB10321304616F0A8FD97
:10A2E00030B9284616F013FE2437BD46BDE8F0838A
:10A2F0000521304616F09CFDB8B114F8043C1B074C
:10A3000007D514F8033C180703D51121304616F081
:10A31000D6FD14F8043C23F0080304F8043C14F8B8
:10A32000033C23F0080304F8033C14F8033CD9076A
:10A3300014D50621284616F0C2FD0221304616F03B
:10A34000BEFD2168D1F8A46086B114F8043C002B4E
:10A35000CAD114F8031C0029C6D1B6E79A0701D563
:10A360000821E7E75B07E8D50A21E3E738467031C3
:10A37000F8F762FF6D4688B00A4B6A46CDE90537AB
:10A380004FF40073ADF81C30074B42F8103F4FF408
:10A39000E25133460548F7F72DFCAD46A4E700BF70
:10A3A000DF8602008382020003000001B048020041
:10A3B00037B5A0F59C75A0F59A74D4E8AF3FD5E801
:10A3C000AF2F012100920748074A14F0E3FE284608
:10A3D0000821FFF7A7FC0421204603B0BDE8304068
:10A3E00016F06DBDB0480200988202002DE9F043DE
:10A3F00089B000AF0446FEF771FE054680B3061D26
:10A400000321304616F014FD50B3D4F8A40008B16F
:10A4100016F015FF207A04F1700100F0A3F88046D1
:10A42000C4F8A40000BB384604F17001F8F704FF3B
:10A430006E4688B0414B6A46CDE905374FF400734C
:10A44000ADF81C303E4B42F8103F4FF4E2513D480E
:10A450004346F7F7CFFB0821B5462846FFF7E4FC53
:10A460002437BD46BDE8F0830E21304616F0E0FCEF
:10A4700028B1D4F8A420537C43F0020353742B7A00
:10A48000032B0DD8002B4DD1D4F8A420537C23F0FE
:10A4900020035374D4F8A420537C23F001030DE06F
:10A4A000053B012BF0D8D4F8A420537C43F02003C3
:10A4B0005374D4F8A420537C43F0010353742B7DD0
:10A4C000697BD4F8A4208B4228BF0B463046137416
:10A4D000052116F0ADFCD4F8A420537C48B343F01A
:10A4E00010030D213046537416F0A2FC0028B7D09B
:10A4F0002021D4F8A40016F09EFED4F8A43005F173
:10A5000047021E33573552F8041BAA4243F8041B76
:10A51000F9D10023D4F8A42053619361D4F8A42086
:10A5200093839DE70521304616F082FC0028ABD0CE
:10A53000BFE723F01003537492E700BF628002006C
:10A5400003000001B0480200012208B5034B044893
:10A550001A70FBF72FFA002008BD00BF653A0020F3
:10A5600050040020F8B5114E0746344614F8013B5C
:10A570000D46834204D10722204619F08FF980B19D
:10A5800007220B490B4819F089F960B904F8017CDE
:10A590002B682360AB88A380AB79A37140F21123B1
:10A5A000F3600248F8BD0020FCE700BFE81A002075
:10A5B000D3850200E91A002010B4064B0C46598AD4
:10A5C000014204D018461146234610BC184710BC5F
:10A5D000704700BFE81A002010B50A4C1346628A83
:10A5E000024202D022788A4201D0002010BD072208
:10A5F0001946601C19F052F900280CBF20460020B3
:10A60000F4E700BFE81A0020F8B50B780D46012BDF
:10A6100001D00020F8BD8B7903F0C003402BF8D1A6
:10A620000F4C638A9B07F4D523788342F1D104F160
:10A630003E0706223946681C19F030F908B9084867
:10A64000E8E7691C04F12E0015F030F80028E0D08E
:10A65000D5F80130C4F83E30B5F80530BB80EEE7E0
:10A66000E81A002010B5074C2378834208D107224E
:10A67000601C19F013F900280CBF2046002010BD03
:10A680000020FCE7E81A00202DE9F04384468946C3
:10A6900090462E4A9BB01D46DDE923760CAB02F1B5
:10A6A000300E1C4610685168083203C472452346B8
:10A6B000F7D11068127961462060227104A8202227
:10A6C00016F0CBFD6B462022214804A900F06EF85D
:10A6D0000446B0BB49460DF1350016F0D6FD4146A3
:10A6E0000DF1450016F0D1FD294611F8013B062277
:10A6F0000DF156008DF8553016F0AFFD2299062267
:10A7000011F8013B0DF15D008DF85C3016F0A5FDF0
:10A710003B46352268460CA900F048F8044680B94B
:10A72000384616F0A4FD012335228DF830306846F6
:10A7300033460CA900F03AF8044610B9304616F03A
:10A7400096FD20461BB0BDE8F08300BF82490200A1
:10A750001087020070B50E461D46144698B001469B
:10A76000202204A816F079FD202231460CA816F00C
:10A7700074FD294614A816F088FD2146684616F097
:10A7800084FD6B465022684604A900F00FF840B9DA
:10A79000039B054A1BBAB3FBF2F102FB11331C9A6F
:10A7A000136018B070BD00BF40420F002DE9F041AA
:10A7B0008CB080460D4616460021142207A81F467D
:10A7C00019F064F84FF41053ADF818308023ADF849
:10A7D0001A304FF44063144C1022CDE9083441463E
:10A7E00004AB06A818F0CDF9034648B10F4A10484B
:10A7F000012114F0C6FC6FF004000CB0BDE8F0813C
:10A8000005AB0293102321462A46CDE90073049834
:10A81000334618F0F8FA0446049818F0EAF8204392
:10A82000EBD0044A2346E2E70002C003E0820200C4
:10A8300040480200FC82020010B5002402F1FF3CF7
:10A840001FFA8CFC186001FB0CF300F1070E2EF0D0
:10A85000030EAEF80020C450BCF1000F11D0023A34
:10A8600092B202FB011C02FB01F36044A3EB0C0358
:10A870004FF6FF7C013A92B26245C050A0EB010056
:10A88000F8D110BD036813B11A6812B902601846F6
:10A890007047D91D21F00301B1F800C0D11D21F08E
:10A8A00003010CF1FF3CA1F800C0EFE70B6873B1A6
:10A8B000073323F003031A8801320346D1F800C09E
:10A8C00043F807CB23F003031A8008607047012286
:10A8D000F3E700BF02FB0100704700BF401A90FB86
:10A8E000F2F080B2704700BF6AB153426FEA03438F
:10A8F0006FEA134311440138CA1811F8013D91421F
:10A9000000F8013FF9D17047014402E010F8013B23
:10A910001BB98842FAD1002070470120704700BF60
:10A9200010600860704700BF03680A68934209BF5F
:10A93000002200230A6002601846704713681860FE
:10A940001368596010607047884203D01AB1436899
:10A9500013607047002070470B68834209D02AB10A
:10A96000586810601A680A6018467047002BF9D1C1
:10A97000FAE70023F8E700BF2DE9F8434FF090080D
:10A980000C270D4EDFF8349006F1200409EB080582
:10A99000294620462A1D083CFFF7C2FFB442A5F114
:10A9A0000C05F5D1043F3B1DA8F13008A4F12006A9
:10A9B000EAD1BDE8F88300BF881B0020D41B00202B
:10A9C00003468C4600B5AAB101EB4101164803EBE2
:10A9D000430E090101EB8E010144487A91F808E029
:10A9E000704504BF013008725DF804EB61461846FB
:10A9F0000EF0C6B901EB4102DFF82CE0120100EBCA
:10AA0000400302EB8303734493F80AE0DA7A724559
:10AA100000D000BD01329A720122044B5A545DF8F5
:10AA200004EB0EF0DDB900BFB01B00202C1B002092
:10AA300070B504460D4682B01AB318785978401A9A
:10AA400010F0030030D12B4A4FEA440C4FEA450E78
:10AA5000A444AE444FEA8C0C0CEB0E1C01310CF1FB
:10AA6000040C1970586819466244FFF767FF012209
:10AA7000214B294620465A550EF0B2F9002002B06B
:10AA800070BD01930EF096F9019B0028D5D02946A0
:10AA9000204601930EF080F9019B597848B9187847
:10AAA000401A10F00300CED00128E8D0013119700F
:10AAB000DDE705EB450004EB440C0E4A000100EB1A
:10AAC0008C001044867AC07A4FEA440C86424FEAE2
:10AAD000450E05D01878401A10F00300E4D1B7E70E
:10AAE0001A78521A920701D002311970D3E9020282
:10AAF0009047C3E7B01B00202C1B00202DE9F04F2E
:10AB0000DFF8589189B019F80030002B56D0002199
:10AB100003248346DFF848A1C0EB0013CDE90411FC
:10AB200000EB40079B000AEB0717039309F800109E
:10AB30000294B8460023B96A58F8240F07AA07936D
:10AB4000FFF702FF0446ACB1079D2E786A78B61A6B
:10AB500006F00306012E34D02B789A1A02F0030275
:10AB6000012A3CD1D7E9090107AAFFF7EDFE044607
:10AB7000002CE9D197F82E3097F82F209A4203D075
:10AB800087F82F300123049397F82C3097F82D2065
:10AB90009A4203D087F82D3001230593029B0C3F86
:10ABA0005D1EEBB2FF2B0293C3D1D846DDF810B087
:10ABB0000599BBF1000F01D0002944D009B0BDE8D0
:10ABC000F08F013A6A70079BD3E902029047079D14
:10ABD0002B786A789A1A02F00302012A21D0002207
:10ABE0004146B86A0193FFF7B7FE6C60019B6A7833
:10ABF0006B702B789B1A03F00303012B08D0D7E965
:10AC0000090107AAFFF7A0FE012E04469BD10EE022
:10AC1000039B6A701A1D294620465244FFF78EFE98
:10AC2000EDE707AAD7E90901FFF78EFE0446029B6C
:10AC30008BB101235946584609F80B300EF0D0F875
:10AC400009B0BDE8F08F0A464046414609B0BDE86C
:10AC5000F04F0EF095B8002C8CD0EAE72C1B0020AA
:10AC6000B01B0020034681B1002001F1FF3C53FAE4
:10AC70008CFC591E11F8013F23B15A1E01301340BC
:10AC8000C0B2FAD16145F5D170470846704700BFA0
:10AC900070B50646007EFF282ED00D4602464FF0C6
:10ACA000000ED6F800C007E09C681CF80130104682
:10ACB000FF2BA64420D01A4602EB420395424FEAEE
:10ACC00003110CEB0313EFD1A84202D11CF80120B1
:10ACD00032761CF8011000EB40000201FF29986851
:10ACE0000CF8021006D001EB41010CEB01118B684E
:10ACF00003448B60704470BD002070BD2DE9F043AB
:10AD000004462C259E46264B104605FB04335C6802
:10AD100083B004EBC10214F83170D478567804F192
:10AD2000010C5FFA8CFC674598BF4FF0000C66453C
:10AD3000BDF830802FD07646074605FB04FE084656
:10AD4000042502215468D2F80490744409F80E5086
:10AD5000A1700A996770A1600B996660E1600D9916
:10AD6000A4F810806161129921620E99A1610F9976
:10AD7000E161109961621199A16282F803C0D3E97F
:10AD800008260193904700222946019BB047A078EE
:10AD900003B0BDE8F083012003B0BDE8F08300BF3D
:10ADA000701C0020437A002B00F004812DE9F04F45
:10ADB0008B4682464668013B0268DBB287B006EBF1
:10ADC000C303019202930596029B5A6893F801907F
:10ADD0000492CDF80C90BBF1FF0F5ED000260BEB78
:10ADE0004B04019B2201DE4613F802B003EB04146E
:10ADF000FF2727709AF81830DAF80050BB4205EBAD
:10AE0000020800F0CA80D8F8081000960CE0091A71
:10AE100005D1B8F81E90F68BB14500F28680AA5C89
:10AE20001F46FF2A76D0134603EB430205EB0216BA
:10AE3000B0684FEA430C88424FEA0212E7D9009EFD
:10AE4000FF2F18BF07EB470788F8003018BF3F01F6
:10AE50006344C8F8081005EB03130CBF8AF818E028
:10AE600005F807E09A68521A9A60A3780133637074
:10AE7000002EB0D04FF00002736A3270B27013B17E
:10AE80000020B16A98476368002BA4D1736ABBF1B4
:10AE9000FF0F2362B36A6362A0D1DDE90397012546
:10AEA000029B9878484509F101022AD02C2303FB24
:10AEB00009F302995FFA82F90978FA5C494508BFFB
:10AEC0004FF00009042A07EB0306EBD196F801E0E6
:10AED00001990EEB4E0201EB02146078A178120189
:10AEE000884225D04FF00002FA54736AB57013B14E
:10AEF0000120B16A9847029B09F101029878484500
:10AF0000D4D1029B059A5870934250D0029B083BC3
:10AF1000029359E79C444FEA0C1CC8F8081088F8C3
:10AF20000020009E05F80CE09FE70146009E87E7A1
:10AF30004FF6FE70338ADAF814108342CDF80C9085
:10AF400007D04FF6FF701B1AB3FA83F35B0984F83E
:10AF50002C304FF6FD70336AA362F3686360338A66
:10AF6000834288BF0023A3837369A361B369E3604D
:10AF7000F36923610023B0686361A06073685D1AA0
:10AF80000FD40023284463614FF00003E383E37888
:10AF9000A06043F00103E3702AE7AB548AF818E09D
:10AFA00063E7CB1A9842ECD81B1A0020EBE707B0F6
:10AFB000BDE8F08F704700BF01232DE9F04F447EBC
:10AFC00091B08376002C40F0C280037EFF2B00F00E
:10AFD000BD8081460CF0ACFF99F818A0BAF1FF0FC4
:10AFE00000F0CD81D9F81430A046A0EB030BD9F8BE
:10AFF0001C30CDE904945B4594BF00230123D9F8AC
:10B00000006003930AEB4A0A06EB0A14A5684FEAAC
:10B010000A1A5D4577D8A278637816F80AA09B1AB9
:10B02000DFB2012FA84468D1A06AD4F81890002894
:10B0300000F01E810168002900F08C80039BB9F1AB
:10B04000000F00F05281002B00F07381037A5A0741
:10B0500000F06381037A23F007030372B4F81EC083
:10B06000E2780CF1010322F00102E27094F82C2046
:10B070009BB2E383002A00F0F780A28B9A4280F013
:10B08000F380A06A002800F06F81037A03F00703C1
:10B09000012B00F0E9804FF0000C4168C0F804C0BB
:10B0A000A36A1A7A6CF302021A72A278531EA37072
:10B0B000E3689C460BB3049B60695B69E278A8EB8C
:10B0C0000000184402F001022369002F40F00681BD
:10B0D000E78BCDE900233B4600226746B847039B38
:10B0E000B9F1000F18BF43F0010303934FF00003C1
:10B0F000E383E37823F00103E370BAF1FF0FABEBD6
:10B10000050B7FF47FAFDDE9049499F80B3099F8D3
:10B110000A209A4208D10132D2B2022A16BF14463E
:10B120000023234689F80B4009EB8303C3F80C8006
:10B13000D9F8244000254B46012204210320A446CF
:10B1400089F81A5011B0BDE8F04F6047847611B00D
:10B15000BDE8F08FB9F1000F00F0BE80039B002B1B
:10B160007FF478AF049BDB6943453FF673AFBAF1D8
:10B17000FF0F00F0FE80B4F81EC0CDF82090CDF88F
:10B180003890A38B616863458EBF6346ACEB0303C5
:10B190009BB20991CDE90A5B03FB0111CDF83CC0DC
:10B1A0004FF0000EA34653468446CDE90C8ACDF8F5
:10B1B0001890DDF83880DDF82490079109970E92F9
:10B1C00003EB430306EB031291681B018E44F04529
:10B1D00077D3946A9069002C6DD02468002C6AD0D3
:10B1E000D58B978B5468AF4240F2A980002C00F0B9
:10B1F000AD80B9F1000F00F0A980AA46611A04FBE6
:10B200000A11079C8C422CBF4FF0000A4FF0010A34
:10B21000BCF1000F08D0DCF800402CB1069919B938
:10B220007044A04240F2B480AF4246D8D0789BF838
:10B23000032000F0010402F00105A54205D34240BD
:10B24000D1073AD4BAF1000F37D06046DDE90C8A55
:10B250005C46DDE90A5B099FDDF83CC0002840F050
:10B260009080DDF82090FBE6A378013BA37044E7D3
:10B27000B9F1000F4ED0039B002B7FF4EFAE049B7F
:10B28000DB699845FFF4EAAEBAF1FF0F7FF473AFC4
:10B29000531EA370E3689C46002B3FF434AF049A1E
:10B2A00063695269A8EB03039818E278039923694C
:10B2B00002F001020CE7002892D1F35CFF2B7FF42F
:10B2C0007FAF6046DDE90C8A5C46DDE90A5B0E9AD9
:10B2D000002867D0DDF820900027DCE6CDE90023C8
:10B2E0004FF6FF730022E04707E763B9049BDB6971
:10B2F000984508D3BAF1FF0F3DD09623B4F81EC08D
:10B3000008930E933DE7037A4FF096095A077FF4AE
:10B31000A1AE02E04F464946C8E6A18BE28B9142BE
:10B320003FF698AE012262F302030372B4F81EC026
:10B3300096E6049BDB699845FFF488AE17E74CB9A5
:10B34000BCF1000F13D04FF0000A64E7BCF1000F0E
:10B35000F9D1B2E7B9F1000F04D0A5EB070A1FFA43
:10B360008AFA4BE7CA4653E70146A2789EE6E246D0
:10B370005CE7039F8FE64FF09609039F8BE6A0469C
:10B38000C3E60168DDF8209000293FF463AE5DE676
:10B390002146DDE90C8A5C4660460A9D099FDDF87E
:10B3A0002CB0EFE767460146DDF820907EE600BF4F
:10B3B000837E002B40F005832DE9F04F437E8BB058
:10B3C0000793002B7AD10121837AC27AD0F814B086
:10B3D0009A42417600F0F6820B44DBB2022B0ABFA0
:10B3E000079A1A4613460124837200EB8203DB6836
:10B3F00003935B444361037E81461D4606930CF034
:10B4000097FD99F80930FF2D08BF8346049008BFC7
:10B41000C9F81400002B00F0E283D9F80450013B76
:10B42000DBB205EBC30AFF23CDE908B40293D9F8D8
:10B430000030059501939AF802B09AF80310594527
:10B4400071D0DAF8048024E0082B4FD86178019A93
:10B4500001EB410702EB07167278B0783F01121A30
:10B4600012F0FF0234D1062B40D199F81B308B42E9
:10B4700069D04FF0000308F80530A370636A13B178
:10B480000020A16A98479AF802B09AF8031059452B
:10B4900049D09AF800300BF10102D2B2934208BFB2
:10B4A00000222C2303FB0BF58AF8022018F8053044
:10B4B00008EB0504042BC7D89346E8E70421446A47
:10B4C000034601220846A4460BB0BDE8F04F604792
:10B4D000052B2FD16368DBB9A368CBB9E368BBB98F
:10B4E0002369ABB9A38A9BB9A37D8BB94FF0000345
:10B4F00008F805304FF00103A370636A002BC2D037
:10B50000A16A012098479AF802B09AF80310BEE7A2
:10B51000012A25D004214B4601220846D9F82440AF
:10B52000A0478AF802B0059B9A4500F0CA80AAF1AC
:10B53000080A80E7012A00F08280062BEAD199F8F8
:10B540001B308B4295D16168D9F814208B1A40F1D9
:10B550009B80521A0399914200F29680002395E055
:10B560004846FFF795FBB060049BD9F814C0A3EBE5
:10B570000C01039B03EB010E704540F28E80A0EBA3
:10B580000E02736803B3A38AF3B1013B98B2A082A1
:10B59000D6F804E0F38B964508D30BE01FFA8BF343
:10B5A000A2EB0E02F3839645A08A03D2834203F1F5
:10B5B000FF3BF3D8834206D201339BB2F383A08AC8
:10B5C00072448342F8D3B083636802EB030EC6F87B
:10B5D00008E0A06873690344B06A736140B102680F
:10B5E00032B1D4E901329B1A4360D6F808E073699E
:10B5F000002959DB7144994260D9C91A002373614B
:10B60000B160E268B3691344B3612269934294BFA5
:10B6100000239B1AB361A37D1BB1F27863F3000290
:10B62000F270E37D13B1013B86F82C30DDE9012394
:10B63000D3557378627801330292737019E7062B41
:10B640003FF413AF4846FFF723FBB378B060737045
:10B6500099F81B2063789A427FF40BAF18F80530F5
:10B66000062B3FF470AFFF2389F81B3018F8053024
:10B67000062B3FF468AF082B3FF465AF0499D9F867
:10B6800014208B1A3FF565AF039A1344D9F81C2098
:10B690009A4288BFC9F81C30EBE6736900229E44C9
:10B6A000AEEB000070616CE7049AACEB020CF44561
:10B6B000A0D39C440021ACEB0E03A0E75B1A002151
:10B6C0009DE7DDE908B499F81850002C00F01D81C1
:10B6D000069BEB1A18BF0123FF2D08BF1C460593DC
:10B6E00061D00027049BD9F80080039ECDF810B0EC
:10B6F000A3EB0B0A019705EB450308EB0314A268C3
:10B700001B01B24200F249820199A07811440191D3
:10B710006178B61A091AD9F81C00AAEB020A82420B
:10B7200026BF4FF0FF320020801AB4F81EE028BF79
:10B7300089F81B20C9F81C00A06AA269C9B20028B8
:10B7400000F0B6800768002F00F09D80002A40F0CE
:10B750009D80022900F01B820022A26018F80320BD
:10B7600089F818206268A06A002A73D120B1027A91
:10B7700002F00702012A49D049B1012902D0BEF1E5
:10B78000000F04D0236A13B10120616A9847A278A0
:10B79000627099F81850FF2DADD1DDE90543FF2BFC
:10B7A00018BF44F00104002748460299FFF7FAFA4F
:10B7B000CDE90194D9F800B0019B187EFF2800F074
:10B7C000118204464FF0FF0800E01C4604EB4403DE
:10B7D0000BEB0315A96A1B018C4629B10A7A02F00A
:10B7E0000702012A00F0F5801BF80330A046FF2B6A
:10B7F000EBD1DDE90194002F40F0A780069B834246
:10B8000040F0A380002C00F08B80A2E03146A278AB
:10B81000A66062700498019FD9F814C000EB070B72
:10B82000BBEB0C00D4F814E04CD40844864552D24B
:10B830000021A0EB0E00616101320299D2B2A0603A
:10B8400008F803106270029599F81850FF2D7FF4E4
:10B8500052AFA2E720B1017A01F007010129D5D04A
:10B86000B4F81EC0BCF1000F39D1B4F81CC094F874
:10B870002C00614601FB0221002839D06278A4F82F
:10B880001EC0A160C6E7002A3FF466AF02297FF41C
:10B8900063AFBEF1000F7FF45FAF007A00F00700E6
:10B8A00001283FF459AFC9F81C2089F81B5053E711
:10B8B000002A3FF451AF02297FF44EAFBEF1000FD2
:10B8C000F1D049E7ACEB0B0C8C45AED3F44400202F
:10B8D000ACEB0101AFE7AEEB00010020ABE70021CC
:10B8E000A07801FB0221607094F82C000028C5D1DB
:10B8F0008A45C3D9019F11448A4500F10100FAD855
:10B90000604401971FFA80FCB8E748460299FFF7A8
:10B9100049FA99F81800069B834213D19D4211D130
:10B92000002389F8193099F81A30002B46D0D9F83D
:10B9300024404B46012203210420A4460BB0BDE85D
:10B94000F04F6047FF2800F05681069BFF2B00F068
:10B950003A81D9F8003000EB400003EB00139F68F8
:10B96000002F33D00CF0E4FA0A260446D9F814501C
:10B97000621B974202F1060116D9B9422CBF6D181D
:10B98000ED19D9F82830284698470CF0D1FAC4F1BF
:10B9900001022B1B02449A4208D9013E01D0044601
:10B9A000E4E700DE0446E1E701230793002389F87A
:10B9B000193099F81A30079A1A43B8D10BB0BDE87C
:10B9C000F08F7047079B1C46039314E589F81970A4
:10B9D000ADE7AA68002A40F02181D5F818A0BAF195
:10B9E000000F06D10A68002A00F024818C464FF02F
:10B9F000960ADCE90029914580F0DA801BF80310F3
:10BA0000FF2900F0D580A2EB090E00220198CDE9B4
:10BA10000494C069994600F19606AEEB0A000390C3
:10BA20001746104634460B46CDF820800AEB07082F
:10BA3000C64540D303EB43030BEB03118E681B0198
:10BA4000304496287DD9A0F196063E44764528BF1D
:10BA500076460AEB040296450ED3B0450CD8AA6987
:10BA6000002A00F088809CF80820120700F18380EB
:10BA7000B6EB0A0240F0AC808A6A22B1127A02F078
:10BA80000702012A6DD08A69002A6AD04968002914
:10BA900067D096320744D419AA69002A75D09CF859
:10BAA0000810AEEB0A02090700F1968000201BF88F
:10BAB0000330FF2BBAD14B46DDF81090059C914422
:10BAC000CCF804901BF803A0DDF82080BAF1FF0F3A
:10BAD000514618BF4FF0FF0E01D1B1E0014601EB16
:10BAE00041000BEB0017BE684FEA410996424FEA4E
:10BAF000001080F0A7801BF800008E46FF28A2EB04
:10BB00000602EBD1AA60B8F1FF0F00F0838008EBCA
:10BB1000480212010BF802A009EB010212011BF806
:10BB200002100BF803100BF802400222EB8B0127E6
:10BB3000013BEB839CF8083062F302038CF8083079
:10BB40003AE6AE698EB19CF8086016F0080680D01F
:10BB50008C690744963403993C448C4298BF224632
:10BB6000A4E700221BF80330A3E78A690744963252
:10BB70003A4414469AE7002C3FF47EAFA6EB0A063F
:10BB8000A642FFF479AF224695E722468EE7BEF142
:10BB9000000F7FF4E1AD96227FE6921BA26099F838
:10BBA0001830DDE90542934218BF44F00104FAE57C
:10BBB000CCF804901BF80330FF2B08BF00223FD0C5
:10BBC0000023AB60B1E70CF099F999F81800C0E6D2
:10BBD000A242FFF451AF6EE711460022BDE7FF23FA
:10BBE000029370E59946029C2FB9069BFF2B02D168
:10BBF000002C3FF495AE0CF08BF900287FF490AE4A
:10BC0000C9F81C0089F8190099F81A30002B7FF444
:10BC10008EAED3E6019A82F818A07DE700DEA96A0D
:10BC2000D5F818A08C46BAF1000F7FF4E2AE0029D7
:10BC30007FF4D8AE00DE4FF0960AD5F828C0D8E6DB
:10BC4000AA6072E7B61ABEF1FF0FBE60AA603FF4A9
:10BC50006CAF71461BF803A04FEA4E0953E700BFD3
:10BC600010B58E469DF80CC0049970BB184C22602C
:10BC7000029A84F808E06372626093B14FF02C0E70
:10BC8000013BDBB202EBC303A2F10800596013F8D9
:10BC90000829ACEB020C83420EFB02115FFA8CFC0C
:10BCA000F4D1BCF1000F10D1FF23059AC4F814C0E1
:10BCB0002262069AA4F80AC06262079AC4F81CC0FD
:10BCC000A2622376E376604610BD012010BD00BF5E
:10BCD000701C002040B9064A117EFF2901D1107264
:10BCE00070476FF00F0070476FF01500704700BF8E
:10BCF000701C00202C22084B00B502FB0033D3F847
:10BD000024E0BEF1000F06D0F446012203210220F8
:10BD10005DF804EB604700BD701C002000B5BDF865
:10BD200010C0DDF814E0CDF80CC04FF0000CCDF8D9
:10BD300010E0DDF818E0CDF814E0DDF81CE0CDF8F7
:10BD400018E0DDF820E0CDF81CE0DDF824E0CDE9D6
:10BD500008EC5DF804EBFEF7D1BF00BFBDF80CC0E6
:10BD6000CDF808C0DDF810C0CDF80CC0DDF814C067
:10BD7000CDF810C0DDF818C0CDF814C0DDF81CC037
:10BD8000CDF818C0DDF820C0CDF81CC0DDF824C007
:10BD9000CDF820C0FEF7B2BF2DE9F04704462C25B0
:10BDA0001846264B82B005FB04335C68BDF834802E
:10BDB00004EBC10E14F831709EF803409EF8016048
:10BDC00004F1010C5FFA8CFC674598BF4FF0000C42
:10BDD00066459DF838909DF844A02AD00527064670
:10BDE00005FB04F402250846DEF804100F550C4448
:10BDF00062700A9A6660A2600B9AA4F81480E260EE
:10BE00000C9A84F8169022610F9A84F817A0626247
:10BE1000109AA570A2628EF803C0D3E90825019399
:10BE2000904700220421019BA847A07802B0BDE8FA
:10BE3000F087012002B0BDE8F08700BF701C002031
:10BE400000B589B0DDF828C0DDF82CE0CDF800C0E1
:10BE50004FF0000CCDF81CC0BDF834C0CDF804E0A4
:10BE6000CDF80CC09DF838C0DDF830E0CDF810C03A
:10BE7000DDF83CC0CDF808E0CDF814C0DDF840C0D6
:10BE8000CDF818C0FFF788FF09B000BDF0B52C262B
:10BE90001A4C1F4606FB00435C6883B004EBC105E7
:10BEA00014F83100EC7895F801E004F1010C5FFA28
:10BEB0008CFC604598BF4FF0000CE6451BD04FF05E
:10BEC000070E084606FB04F102266C6804F801E040
:10BED0000C446270089AA6706762A26285F803C07B
:10BEE000D3E908250193904700220421019BA8472C
:10BEF000A07803B0F0BD012003B0F0BD701C00209D
:10BF0000F0B52C261B4C1F4606FB00435C6883B033
:10BF100004EBC10514F83100EC7895F801E004F168
:10BF2000010C5FFA8CFC604598BF4FF0000CE645B1
:10BF30001DD04FF0080E084606FB04F102266C687F
:10BF400004F801E00C446270089A67606262099A22
:10BF5000A670A26285F803C0D3E908250193904733
:10BF600000220421019BA847A07803B0F0BD012066
:10BF700003B0F0BD701C00200BF0DABF401A704710
:10BF800000210148704700BF7F410100022801D015
:10BF90000120704738B5054608461C4603F018FCDA
:10BFA00018B100232370184638BD284638BD00BF9D
:10BFB000002303700B70704710B5044682B0002058
:10BFC000019102F055FF80B9019944B9084B49B17C
:10BFD000086818608A889A80002002B010BD054B5E
:10BFE0000029F5D119609980F6E70C2002B010BD48
:10BFF000A41C00209C1C00200128024605D8044BEC
:10C000000448002A18BF184670470020704700BF38
:10C010009C1C0020A41C002001280AD8064A074BBB
:10C02000002818BF1346186808609A8818468A8046
:10C0300070470023184670479C1C0020A41C002059
:10C0400010B504460AF026FA50B90AF0AFFD60B9FF
:10C050000BF0F4F970B92046BDE810400FF080B93C
:10C0600000DE0AF0A3FD0028F2D000DE0BF0E6F9B6
:10C070000028F0D000DE2046BDE810400FF070B977
:10C08000086001480FF06CB9F42200200FF068B985
:10C090002DE9F0470B78072B84BF2B4B93F84030EA
:10C0A0009A424ED0284D5C1CE4B2914635F83320BC
:10C0B000082C8246884608BF0024002601270280FB
:10C0C00005EBC30319E0012838D012225A60072C6F
:10C0D00088F8004088BF95F84040A14523D023B29E
:10C0E000013435F83310E4B2BAF80020082C08BF48
:10C0F0000024914205EBC30315D15868B0B1FF2865
:10C10000E1D9027902F00302013A012A12D912227E
:10C110005A6003F077FB072C88F8004088BF95F839
:10C120004040A145DBD13046BDE8F08701365F6075
:10C13000F6B2CCE701360122F6B2E9E70136F6B2F3
:10C14000C5E70026EFE700BFD01C00202DE9F04135
:10C150002F4E338898424CD913F0FF0820D02D4D34
:10C160006C7D0134E4B2052C08BF00242B7DA34272
:10C1700018D02948FEF786FB074688B12748FEF706
:10C1800081FB002837D007606B7D45F8230033889A
:10C1900008F1FF30013B10F0FF086C753380E0D1EF
:10C1A000BDE8F0813388002BFAD000271C4D6C7B52
:10C1B0000134E4B2032C08BF00242B7BA342EFD050
:10C1C0001548FEF75FFB80460028E9D01348FEF7CC
:10C1D00059FBB0B1C8F80470C0F800806B7B45F81B
:10C1E000230033886C73013B9BB23380002BDFD17B
:10C1F000D6E78046B3E73846BDE8F0410649FEF78A
:10C2000055BB4046BDE8F0410349FEF74FBB00BFB8
:10C21000381D0020B42000203C1D0020901D00206F
:10C22000181D00202DE9F84300274FF005092E4B7B
:10C230002E4E181D052224213783FEF7FDFA2C4BC4
:10C2400005220821181DFEF7F7FA96F81880747E6B
:10C250000134E4B2062C08BF0024A04514D02448C1
:10C26000FEF710FB054678B11F48FEF70BFB0028D0
:10C2700034D06F600560737E46F8230009F1FF3308
:10C2800013F0FF097476E3D11A4B0822181D6421BC
:10C29000FEF7D2FA184B0A22181D0821FEF7CCFA35
:10C2A0001548FEF7EFFAA8B1144A111FFEF738FB44
:10C2B0001148FEF7E7FA78B1114A111FFEF730FB7B
:10C2C0000622104BFF201A80FFF740FFBDE8F8431D
:10C2D00008F0F4BD00DEE7E700DEEDE7284604499C
:10C2E000FEF7E4FAD0E700BFF8200020B0210020DC
:10C2F000CC200020901D00203C1D0020341D00207B
:10C300002C1D0020381D0020F0B57B4D7B4E89B0E0
:10C3100006AA04A90DF10F0004F076F80446D5E949
:10C32000000105AAFEF710FB074650B3059B002B42
:10C3300069D0187806AA04A904F07EF8059B044683
:10C34000002840D0069ABDF810101F78ADF81210E2
:10C35000079204F083F82146079ABDF8120004F012
:10C36000B1F8204604F044F8384607AA0DF112014E
:10C3700004F062F804460028EBD130680EF0F0FFBC
:10C38000C6E7002C3DD0069B9DF80F700793BDF8C3
:10C390001030ADF8123004F061F82146079ABDF86C
:10C3A000120004F08FF8204604F022F8384607AA5D
:10C3B0000DF1120104F040F804460028EBD130687A
:10C3C0000EF0CEFFA4E707931B79013B2C2B1DD861
:10C3D000DFE803F01E31701C1C1C1C1C1C1C1C1CE8
:10C3E0001C1C1C1C1C1C1C1C1C1C661E1C1C1C1C41
:10C3F0001C1C1C1C1C1C1C1C1C1C1C1C1C1C1C1C7D
:10C400001E0009B0F0BD00DE059B92E700DE7FE76D
:10C41000002239496868FEF79FFA3846384B079979
:10C4200093F84130374A0B70FEF788FA334B18689F
:10C430000EF096FF6CE700222F496868FEF78CFA31
:10C44000079884682CB12378002B52D02378013BC5
:10C450002370037B13B1012B44D000DE00232A4A52
:10C460000373537E117E0133DBB2062B08BF00231A
:10C4700099423CD00760517E42F821005376002C4F
:10C480003FF446AF2378002B7FF442AFA368002B24
:10C490003FF43EAF1D4AE0689342C9D0984737E762
:10C4A000002215496868FEF757FA3846079903F0E5
:10C4B00073FC2DE7384607A903F088FC0E490022DB
:10C4C0006868FEF749FA079900293FF421AF0B7914
:10C4D0002E2B3FF41DAF0A4B384693F84130094AE2
:10C4E0000B70A1E7019003F085FD0198B6E700DE2F
:10C4F000C5E700DEAAE700BF301D0020F0220020C3
:10C50000D01C00202C1D0020B02100208DC0000078
:10C5100000B52A4B89B018600BF0E4FC284B1A7860
:10C52000002A42D0274B0C210593274B4FF0020CD9
:10C530000493264B26480393264B00900293042332
:10C540000191254A0370037280F810C080F818C06A
:10C5500019460020FFF784FB68BB012200211F4819
:10C5600015F000FE09F014FF034610B1184609B09B
:10C5700000BDFFF757FE0AF003FB03460028F5D184
:10C5800002F032FC03460028F0D10AF04BFF0346CC
:10C590000028EBD103F0A8FB03460028E6D1079062
:10C5A000012009F02DF9079BE0E7FEF7E5F90122EC
:10C5B000034B1A70B6E700DECFE700BFF022002081
:10C5C000683A0020CD8E0100318E0100118E0100ED
:10C5D000142500200423002034250020F42200200C
:10C5E00030B585B002F006FC90BB03F083FB002859
:10C5F00033D100241C4B2046A3F8404009F000F939
:10C600001A491B4A1B4BA1F8204194829C810122AC
:10C610002146684615F0A6FD174B03202246214609
:10C62000C3F808D0FEF704FAC8B94FF0FF324FF054
:10C63000FF3368460EF0C8FE02F0E2FB88B9FFF750
:10C64000F1FD0021012005B0BDE83040FFF7B4BC8A
:10C6500000DE03F04FFB0028CBD000DEC9E700DE90
:10C66000E3E700DEEBE700BFD01C0020CC21002078
:10C67000B4200020181D00208804002008B5FFF712
:10C68000AFFF09F0BBFE00B108BDBDE80840FFF7F1
:10C6900021BB00BF2DE9F043804689462C4D2D4E2D
:10C6A00083B00023C8F8003095F8414001AAD6E9CC
:10C6B0000001FEF749F90746002834D0019B48469F
:10C6C0001A782549FFF7E4FC034690BB95F8402013
:10C6D0008DF8012095F841200DF101010DF10200C6
:10C6E0001C46FFF7D5FC44EA000212F0FF020346A5
:10C6F000F0D101990B79012B22D131467068FEF7F8
:10C700002BF938461549FEF7D1F8154A1388052B41
:10C7100013D80198013313491380FEF7C7F801209D
:10C72000FFF714FDBDE7224648460B49FFF7B0FC72
:10C730000346184603B0BDE8F08300DE1388E8E73F
:10C7400013461846C8F8001003B0BDE8F08300BFD8
:10C75000D01C0020281D0020101D00203C1D0020A2
:10C76000381D0020901D0020002300B5384985B0F9
:10C77000486803AA0393FEF7EFF8002860D0354914
:10C78000FEF794F8039A13792D2B19D8DFE803F0FC
:10C79000171818171818181818181818181818181B
:10C7A000181818181818181B17171717171718180C
:10C7B000181818181818181818181818181703B96E
:10C7C00000DE05B000BD137F3C2B1ED0537FD3B1DC
:10C7D00093681B68986D30B100221F499A650093D9
:10C7E000FEF764F8009B93F85E2022F0010283F8C4
:10C7F0005E20002002F03CFB10F0FF00E1D109F0C8
:10C8000089F805B000BD00DEF3E79168D1E9003298
:10C81000C2B100204860916FC1B902F16C0102F110
:10C82000680001930092FEF77FF8DDE900230146DE
:10C8300050B110689167009302F0B0FF009BD2E7FF
:10C8400000DE9CE700DEE4E700DEF2E700DEE4E77E
:10C85000281D00203C1D0020901D002070B504689C
:10C86000064682B00CB3344D2046037924682D2B44
:10C8700018D8DFE803F02717172717171717171708
:10C880001717171717171717171717171721342701
:10C8900027272727171717171717171717171717E8
:10C8A0001717172700DE002CDED1FF20346002B0FE
:10C8B000BDE87040FFF74ABC037F3C2B2AD01BB178
:10C8C00000DE0379002B2ED02B88052B28D80133CE
:10C8D0001A492B80FDF7EAFF002CC5D1E5E7C08897
:10C8E0000028E0D102F068FF0346F0B1D3F88820B9
:10C8F000EAB903F17C0103F178000193FEF714F823
:10C90000019BB0B1C3F88800184602F047FF002C25
:10C91000AAD1CAE70949FDF7C9FF002CA4D1C4E791
:10C9200000DE2B88D3E700DECEE700DEDEE700DEA8
:10C93000DFE700DEE6E700BF381D0020901D002085
:10C940000148FDF79FBF00BF3C1D00200149FDF7D6
:10C95000ADBF00BF3C1D00200148FDF793BF00BFE5
:10C96000901D00200149FDF7A1BF00BF901D0020D0
:10C97000034B044A93F841300B70FDF7DFBF00BF53
:10C98000D01C00202C1D002008B5064B064A93F849
:10C9900041300B70FDF7D2FF044B1868BDE808402A
:10C9A0000EF0DEBCD01C00202C1D0020F022002048
:10C9B0000B490A7B4B7B9A420AD8A3EB020C5FFA25
:10C9C0008CFC604509D89A4207D051F82200704784
:10C9D00003339B1ADBB29842F7D90020704700BF9F
:10C9E000181D0020074A117B537B8B4208D04B1C3B
:10C9F000DBB2032B08BF002352F8210013737047EA
:10CA000000207047181D002000B50D4A92F841C063
:10CA100092F840E00CF10103DBB2082B08BF0023C1
:10CA20009E4508D022F83C0002EBCC0CCCF8041058
:10CA300082F8413000BD00DE00231B80FFDE00BF16
:10CA4000D01C0020022802D00B68022B0DD000B5AC
:10CA500083B001914FF0FF324FF0FF3303480EF0E7
:10CA6000B3FC0199086803B000BD7047F4220020B0
:10CA7000044A13680BB11846704703461060184605
:10CA8000704700BFCC1C0020044A136823B19842B1
:10CA90000ABF00210023116018467047CC1C0020FB
:10CAA000014B1868704700BFCC1C0020044A136873
:10CAB0000BB118467047034610601846704700BF18
:10CAC000141D0020044A136823B198420ABF0021B4
:10CAD0000023116018467047141D0020014B186890
:10CAE000704700BF141D002070B5046884B023781F
:10CAF000EBB1054601220021684615F033FB0D4BD2
:10CB0000C4F80CD0A36023788BB100220A4B032019
:10CB100011469D60FDF78CFF38B947F612220023BD
:10CB200068460EF051FC04B070BD00DEF5E76FF012
:10CB30007700F8E78DC000007804002070B5294C1C
:10CB400086B02368002B3ED0994248D14FF0020CAA
:10CB500005AB00931646244B02460D4600200321E8
:10CB6000CDF814C0FFF792F9022803460FD0059ABA
:10CB7000022A0CD1ABB123680BB19D4225D0002D08
:10CB800014BF6FF02D006FF0770006B070BD4FF04E
:10CB9000FF334FF0FF3215480EF016FC059B002BBB
:10CBA000E9D130460393FFF79FFF226812B1954207
:10CBB000039B10D09DB90028E7D010F1780F08BF73
:10CBC000002006B070BD2160C0E700236FF0770041
:10CBD000236006B070BD23600028D6D0EDE76FF06B
:10CBE0002D00D2E7CC1C002081C00000F4220020E0
:10CBF0000B490A7D4B7D9A420AD8A3EB020C5FFADF
:10CC00008CFC604509D89A4207D051F82200704741
:10CC100005339B1ADBB29842F7D90020704700BF5A
:10CC2000B4200020074A117D537D8B4208D04B1C55
:10CC3000DBB2052B08BF002352F8210013757047A3
:10CC400000207047B420002010B582B00446019146
:10CC500003F0D4FB034620460199034A0B7002B04F
:10CC6000BDE81040FDF76ABE341D002001220020FF
:10CC70001146014BFDF7DCBE6804002010B582B000
:10CC80000446019103F0BAFB0346019920460B705C
:10CC9000054AFDF753FE012200201146034B02B066
:10CCA000BDE81040FDF7C4BE341D0020680400201C
:10CCB0002DE9F047194E1F4696F821C196F820310C
:10CCC0000CF10105EDB2092D08BF0025AB42144659
:10CCD0009DF820201DD006EB4C1CE6468046894678
:10CCE000E3682068616802F0010AA268AEE80F00FC
:10CCF0009CF81C30CCE9047823F0030343EA0A03D0
:10CD0000CCF818908CF81C3086F821516046BDE8AC
:10CD1000F0874FF0000C6046BDE8F087CC21002082
:10CD2000054890F8203190F821219A4214BF00EB79
:10CD300043100020704700BFCC21002002780B492F
:10CD4000082A91F8213184BF91F820210270934282
:10CD500009D0531CDBB2092B08BF002301EB4211A1
:10CD60000370084670470021FBE700BFCC2100207C
:10CD70002DE9F04F434E87B096F8203196F82121E7
:10CD80009A4251D04FF000090B24CB46CA46CDE958
:10CD90000499029006EB4313CDF80C901D7FD3F855
:10CDA0000080C5F34002DF6805F001053CB34AB3DB
:10CDB00096F8211196F82031994235D00133DBB233
:10CDC000092B08BF0023994286F820312CD0590145
:10CDD00006EB431382B9D868002D28D1BAF1000FB1
:10CDE0003BD0BBF1000F44D01A7F970704D1824596
:10CDF000725842D0834536D0013CE4B2CEE700DE23
:10CE0000002AD5D1204902988B6011461E4B019211
:10CE1000FDF70EFE019A0028CAD000DE96F8211117
:10CE200096F820319942C9D107B0BDE8F08F039A36
:10CE3000BAB1B9F1000F08BFB9461A7F9507DBD424
:10CE4000D207D4D5BBF1000FD6D1039A8242EBD0E2
:10CE50008145E9D0013CE4B2A0E7BA46CDF81080A4
:10CE6000EBE70397E9E705999142DDD0013CE4B295
:10CE700094E7BB46CDF81480DFE704999142B9D11D
:10CE8000D2E700BFCC21002058040020054B1A7EB9
:10CE9000597E914204D053F8220010B10C307047F3
:10CEA00000207047B021002070B5134A117E537ED8
:10CEB0008B421FD04B1CDBB2062B08BF002352F85D
:10CEC00021401376A4B10223002526682371A060B7
:10CED000256003F093FA03462146084A2370304642
:10CEE000FDF72CFD012228461146054BFDF7A0FD5C
:10CEF000204670BD0024FBE7B0210020341D002037
:10CF00006804002000B59646D0E90723D0F818C081
:10CF1000D018113084458ABF6246A0EB0C03113350
:10CF20000A60CEF8003000BD00B583B0049B93F8D2
:10CF30000AC02CF0020C83F80AC04FF0000CCDE9B7
:10CF400000CC09F0F3FB03B000BD00BF0346012095
:10CF500000B5197F83B001401A69CDE90010D3E90B
:10CF6000050109F0E3FB08B903B000BD7730FBD041
:10CF700000DEF9E7CB681A78042A02D15B78052B2A
:10CF800003D003691B6813B118470020704710B520
:10CF90000846F6F7C7F86FF07F0010BDF0B50B8AB2
:10CFA00085B0002B5CD0064601F10C000C4612F057
:10CFB0004FFB0128054623D002280AD00121034651
:10CFC0002A4A2B4812F0DDF86FF01503184605B019
:10CFD000F0BD03A9204600F0C3FF0399034679B3CF
:10CFE0003046FFF7C7FF034618B30121214A0190DD
:10CFF0001F4812F0C6F80398F6F794F8019BE5E78E
:10D00000002303A92046039300F0BCFA014607461B
:10D0100078B13046FFF7AEFF0346B0B9039D45B186
:10D02000284601F0B5FB03466B711348039915F0D0
:10D0300064F82046F6F776F80023184605B0F0BDF0
:10D040000028F6D0184605B0F0BD0C4A29460190DC
:10D05000074812F096F83846F6F764F8019BB5E7F2
:10D060000121074A024812F084F8ADE7A44F0200FC
:10D0700058480200744F0200F8250020904F02002B
:10D08000604F020008B5FFF7F9FA38B90448F5F720
:10D0900079FC0448F5F776FC002008BD00DEF5E7D2
:10D0A000F811002078120020F0B5064683B014E095
:10D0B0004FF0FF324FF0FF3300211320F6F7B2F9A3
:10D0C0000546BDF80210224601F046FB29463046CF
:10D0D000FFF750FF40BB15F0A8F90DF1020101A8C0
:10D0E000FFF7D8FA04460028E2D1019BA3B1FFF76D
:10D0F0003BFB019F384601F04BFB019D78716B793A
:10D10000032B02D12B79182B10D02946174814F085
:10D11000F4FF019B002BE0D14FF0FF324FF0FF33C3
:10D1200013480EF051F9D8E700DED4E721464FF05E
:10D13000FF324FF0FF330520EF88F6F773F904460E
:10D140000246394605F11C0000F08EFF384600F01B
:10D15000ADFF3CB121463046FFF70CFF20B9204619
:10D16000F5F7E0FF019DD0E700DEF8E7F8250020A5
:10D1700008260020F0B5054689B0244814F08FFF3A
:10D180004FF0FF320021224814F0ECFF2048FFF757
:10D19000BFF90446002830D101F010FB002600271B
:10D1A0006FF0090C4FF4E072CDE90667CDE9014458
:10D1B000184B194904940095CDF80CC017480EF08F
:10D1C00031FC1749154815F00CF96FF0070C4FF4B6
:10D1D0006072CDE90667CDE90144124B124904940F
:10D1E0000095CDF80CC011480EF01CFC10490F48FA
:10D1F00015F0F7F8204609B0F0BD012103460D4AAD
:10D200000D4811F0BEFF204609B0F0BDF825002002
:10D2100008260020A9D00000504C0020F811002062
:10D22000D84F02003DD20000104E0020781200209E
:10D23000E84F0200B84F020058480200F0B5064619
:10D24000002783B04FF0FF324FF0FF3335480EF028
:10D2500053F80028F6D043790190042B36D8002BE0
:10D260004AD0022B4FD04FF0FF334FF0FF32022055
:10D27000F6F7C0F80446019B002C4ED01846214614
:10D2800000F050FF019B01A81F60FFF7E7FA20465E
:10D2900012F065F905462146002012F08AF92B8A22
:10D2A0000446012B0ED933691B6843B12946304629
:10D2B000984738B915F0B9F8002CE8D1C2E72846EC
:10D2C000F5F730FF2846F5F72DFFF3E7052B13D1CF
:10D2D0004FF0FF334FF0FF320820F6F78BF804468B
:10D2E0000198214600F0EAFE019B01A81F60FFF7AC
:10D2F000B5FA002CCBD1A5E700DE019B01A81F6089
:10D30000FFF7ACFA9EE70023002201210020F6F788
:10D3100089F80446019B002CB0D101A81C60FFF7DE
:10D320009DFA8FE7F825002008B50EF071FE05483C
:10D3300014F0BDFE034814F0B2FEBDE808400EF044
:10D340007BBE00BFF8250020DFF874C0DCF804C005
:10D350001CF0005F06D0DFF86CC0DCF800C01CF0E9
:10D36000080F00D1704770B503F10C0482B0019032
:10D370000E4620460221154612F032F940F63E4391
:10D3800001210380204612F02BF904230B210370A6
:10D39000204612F025F9019AA0F80150027032B12E
:10D3A0000023C0F80330C0F8073002B070BD7268C7
:10D3B000B368C0F80320C0F8073002B070BD00BFEA
:10D3C000580100205001002030B50138154689B0C1
:10D3D00011280AD8DFE800F025425909096B097FB6
:10D3E000A9BD090909090909090D6FF0150009B05E
:10D3F00030BDCB68DA789978188807F04BFD5E4B22
:10D4000004460121188812F02CFB034601210C3040
:10D41000019312F0E5F8019B04702B60002009B025
:10D4200030BD554B0D21188812F01BFB0D212860D3
:10D430000C3012F0D5F800234FF4806C04216322E5
:10D44000DFF838E10370C0F801E0A0F805C0C17151
:10D45000037242728372C3720373DFE7464B41214A
:10D46000188812F0FEFA412128600C3012F0B8F84A
:10D4700000213E22019000F8031B16F007FA40F24B
:10D48000A732019BA3F80120C8E73B4B092118886C
:10D4900012F0E7FA092128600C3012F0A1F80022FE
:10D4A000034603F8012BC0F801205A60B6E7C968AB
:10D4B0000020FEF781FD304B0121188812F0D1FACF
:10D4C000034601210C30019312F08AF80022019BDF
:10D4D00002702B60A2E7DFF8A8C003ACBCE80F0025
:10D4E0000FC4DFF894E0DCF80030BEF80000132130
:10D4F000238012F0B6FA132128600C3012F070F875
:10D5000000238446054624880CF8013B0DF10C0EDF
:10D51000BEE80F00C5F80100CCF80410CCF80820D4
:10D52000CCF80C30ACF8104078E7134B1821188871
:10D5300012F097FA182128600C3012F051F80022EE
:10D540000190012100F8022B0AF050FC019B587059
:10D5500064E7094B2121188812F083FA2121286001
:10D560000C3012F03DF800230146013001F8113B68
:10D570000AF08CFC52E700BF403800200200050092
:10D580001C500200002270B5038A8EB0022B099253
:10D5900040F22481044603210C3012F051F8228A13
:10D5A00083789A42C0F023810188C74AC1F385235A
:10D5B000082B118088B2C1F309020DD8D3B1013B09
:10D5C000072B17D8DFE813F0FC001600D800BE00C8
:10D5D0001600160016001C003F2B0BD121461046EA
:10D5E00009AAFFF7F1FE163018BF099C40F0E5804C
:10D5F000B54B188801210EB0BDE8704012F043BA57
:10D60000511E4D29F6D801A353F821F03BDB000051
:10D61000CDDB00007DDB0000F5D5000073DB0000F2
:10D620004FDB000063DC000057DC00004BDC000037
:10D6300041DC0000F5D50000F5D50000F5D500006F
:10D64000F5D500001DDC000001DC0000F9DB000066
:10D65000F1DB00005BDE0000F5D5000029DE0000F4
:10D6600017DE0000D1DD0000AFDD0000F5D50000C1
:10D67000A5DD000075DD000053DD0000F5D50000DC
:10D68000F5D50000F5D5000029DD00000DDD000016
:10D69000DFDC0000A7DC00009BDC0000F5D500000B
:10D6A000F5D500008DDC000085DC00007FDC00008B
:10D6B000B1DA00007BDA000045DA00003BDA000056
:10D6C0002BDA0000DFD90000D5DA0000A5D9000070
:10D6D00055D90000F5D50000F5D50000F5D50000BE
:10D6E000F5D50000F5D50000F5D50000F5D5000012
:10D6F000F5D50000F5D50000F5D50000F5D5000002
:10D70000F5D50000F5D50000F5D50000F5D50000F1
:10D71000F5D50000F5D50000F5D50000F5D50000E1
:10D72000F5D50000F5D50000F5D50000F5D50000D1
:10D73000F5D5000031D90000F5D50000F5D5000081
:10D7400031DB0000511E08293FF654AF01A353F806
:10D7500021F000BF99D8000045D800001DD8000076
:10D76000F5D50000F5D50000F5D50000F5D5000091
:10D77000F5D50000FBD70000632A00F0CD8300F24E
:10D780007F83032A00F0B0802D2A00F0AB83012AAA
:10D790007FF430AFE1684D4B08684C681860114663
:10D7A00040F6014004925C6012F05BF901210446EE
:10D7B0000C3011F015FF0023037020460EB070BD31
:10D7C000062A00F06A831D2A7FF414AFE3681888E4
:10D7D00002F042F93C4B014618880CE701213C4A13
:10D7E0003C4811F0C6FC002420460EB070BD01215B
:10D7F000394A384811F0BDFCF5E7072141F209002C
:10D8000012F02FF9072104460C3011F0E9FE014611
:10D81000002001F8010BFEF7FFFBCEE7092141F2E2
:10D82000030012F01EF9092104460C3011F0D8FE55
:10D8300000220346602103F8012BC0F801205A6042
:10D840004171BAE7412141F2020012F00AF9412187
:10D8500004460C3011F0C4FE00213F22049000F871
:10D86000021B16F013F84FF40A71049B0422C02027
:10D870004FF0200CA3F80F104FF490619871DA72FA
:10D880001648DA75164A83F801C0C3F81A00C3F8BF
:10D890002120A3F8271090E7092141F2010012F09E
:10D8A000E0F8092104460C3011F09AFE00234FF4F1
:10D8B00050610D22DFF82CC08370C0F805C00180D4
:10D8C000C370027179E700BF403800205801002082
:10D8D000305002005048020048500200F7C3F70ED3
:10D8E00030F0F97FF105FFFF00200021C64A4FF01C
:10D8F000FF3441F6FF75C2E900011F200021C34B30
:10D90000C3E90045C24BC3E90001FEF769FEC14B04
:10D910000121188812F0A5F8012104460C3011F0FD
:10D920005FFE0023BC4A03701360FFF7FDFC44E771
:10D93000032142F24B0012F094F8032104460C300C
:10D9400011F04EFE00230146013001F8023BFEF7C4
:10D950002FFB32E7E2689478D178E30744BF41F0C7
:10D960000301D170A6071088B2F805C0137940F101
:10D97000DB8243F00303137143EA0102032A40F000
:10D98000E1824D0700F0D9820CF1FF321CF0030C4C
:10D9900002F0010208BF624602F00AF99D4B0146FF
:10D9A000188828E6E3681A78D10749BF0721587814
:10D9B00008465970920749BF0722997811469A7014
:10D9C00002F0ECF8934A05460121108812F049F85C
:10D9D000012104460C3011F003FE0570EDE609212B
:10D9E00042F22F0012F03DF8092104460C3011F0EC
:10D9F000F7FD05460AAB0DF1220208A90DF11E0044
:10DA000002F09EF80022BDF81E30A5F80130BDF8E6
:10DA10002030A5F80330BDF82230A5F80530BDF858
:10DA200028302A70A5F80730C7E6E368188807F0A1
:10DA30008DFE784B01211888B6E6E368187807F068
:10DA40006FFEBFE7E368072118680A909A889B7900
:10DA500042F22C008DF82E30ADF82C2012F001F897
:10DA6000072104460C3011F0BBFD411C04900AA8AC
:10DA700007F024FE049B18709FE6E36807211868EE
:10DA80000A909A889B7942F22B008DF82E30ADF8DF
:10DA90002C2011F0E6FF072104460C3011F0A0FD08
:10DAA000411C04900AA807F0CBFD049B187084E683
:10DAB000022142F22A0011F0D4FF022104460C3068
:10DAC00011F08EFD049007F087FC0022049B587033
:10DAD0001A7072E6E36805211B8842F230001D4689
:10DAE00011F0BFFF052104460C3011F079FD021D35
:10DAF000C11C0490A8B202F031F8049BDA781870C7
:10DB00001879002A92FAA2F290FAA0F1B2FA82F2FF
:10DB100008BF4FF0FF320028B1FA81F108BF4FF083
:10DB2000FF3101320131A3F80150DA70197144E676
:10DB3000E068C17907F014FE44E7012142F20100D8
:10DB4000E268334B14685268C3E900422CE6E4688B
:10DB500094F80EC0A379627921792088CDF808C0A5
:10DB600094F80DC00734CDF804C0009401F06CF8AF
:10DB700028E7E1680120FEF71FFA23E7092142F2B6
:10DB8000030011F06EFF092104460C3011F028FD4E
:10DB90000023014601F8013BC0F801304B600490BE
:10DBA000FEF7EEF90023049AC1F3072E61F3070391
:10DBB000C2F801006EF30F23080C4FEA102C60F33B
:10DBC00017436CF31F63C2F80530F6E5042142F2F7
:10DBD000020011F046FF042104460C3011F000FD54
:10DBE00000231B210322037041708370C270E4E59F
:10DBF000E06807F083FBE5E6E06807F0CBFAE1E6D2
:10DC000007F0A0FADEE600BFF8120020580100205D
:10DC1000500100204038002018260020022142F246
:10DC20000F0011F01EFF022104460C3011F0D8FC49
:10DC300000220270049007F083FA049B5870BCE540
:10DC4000E368187801F064F9BCE6E16811F8010BAB
:10DC500001F01EFCB6E6E16811F8010B01F0AAFB29
:10DC6000B0E6022142F2070011F0FBFE0221044659
:10DC70000C3011F0B5FC0023037043709DE507F0F4
:10DC8000ADFB9FE6E06807F0EBFB9BE6E06800F188
:10DC90001702C11D08F004F894E6E3685988188853
:10DCA00001F044FF8EE6052142F2230011F0D9FE77
:10DCB000052104460C3011F093FC0AA904900DF1E3
:10DCC000220001F027FF0021BDF82220049BA3F8C9
:10DCD0000120BDF828201970A3F803206DE5E36842
:10DCE0001A88598815469A88A8B201F0DFFE984A2A
:10DCF00006460321108811F0B4FE032104460C30BF
:10DD000011F06EFC0670A0F8015056E5E2680023A1
:10DD1000118892780D46CDE902330221CDE9003316
:10DD2000A8B201F0BDFDE2E70022E46802212388E9
:10DD30001D4663880392B4F808C0A8B2CDF808C0A5
:10DD4000B4F806C0CDF804C0A488009401F0A8FD82
:10DD5000CDE7092142F21C0011F083FE092104469F
:10DD60000C3011F03DFC00237A497B4A016042608F
:10DD7000037222E500220621E3681B8898B204930F
:10DD800007F070F8724A05460321108811F069FE09
:10DD9000032104460C3011F023FC0570049BA0F80D
:10DDA00001300AE5E268002132F8023BE6E709218A
:10DDB00042F2180011F055FE092104460C3011F012
:10DDC0000FFC0023082100F8013B08F027FBF4E4D6
:10DDD000E0680AAA00F1100100230BF03FF95C4B48
:10DDE0001121188811F03DFE112104460C3011F06C
:10DDF000F7FB0023864605460EF8013B0DF1280C83
:10DE0000BCE80F00C5F80100CEF80410CEF80820D9
:10DE1000CEF80C30D1E4E368188801F0F1FD4C4BEA
:10DE200001461888FFF7E7BBE36808211A8842F229
:10DE3000150095B2059211F014FE082104460C302D
:10DE400011F0CEFBC11C0490284601F075FDDDE900
:10DE50000432A3F801201870AFE40022E1684B8877
:10DE6000088803920C890294CC88019489880091D7
:10DE7000114601F015FD364B01461888FFF7BBBB74
:10DE80007B2A14D07C2A7FF4B5ABE26813885188D2
:10DE900098B2049301F0FAFE74E7E3689978188861
:10DEA00001F072FD2A4B01461888FFF7A4BBE36816
:10DEB0000AA91B8898B2049301F0B4FE244A0546CF
:10DEC0000521108811F0CDFD052104460C3011F01C
:10DED00087FB049B0570A0F80130BDF82830A0F83E
:10DEE00003306AE4E36804211A8840F62D401646A0
:10DEF0009A78049211F0B5FD042104460C3011F01B
:10DF00006FFB0546049A0220B1B2EB1CFEF73EF807
:10DF1000A5F80160287050E4E2680121146840F619
:10DF200063400E4B52680FE641EA0302032A09D808
:10DF30004C0702D05A077FF427AD122142F232007B
:10DF4000FFF759BB112142F23200FFF754BB00BF6B
:10DF500040380020008FCC30ECC00100F8120020C7
:10DF60000023F0B583B00B60038A032B2BD9054641
:10DF70000F460C30042111F063FB2B8A4288934238
:10DF800032D31B2A2AD80192068801F035FC019A67
:10DF90000446002837D0B10B4FEA163318D1DBB155
:10DFA000012B15D12179627163F301012171E968B7
:10DFB000E01D15F044FC2146C6F30B0001F028FCDF
:10DFC000C0B903B0F0BD0121204A214811F0D1F8B9
:10DFD0006FF0150003B0F0BD0223E3E701211D4AF5
:10DFE0001B4811F0C6F8F3E701211B4A184811F04D
:10DFF000C0F8EDE70121194A154811F0BAF820469A
:10E0000001F000FCE4E70121154A114811F0B1F8D4
:10E01000144B1B689B0115D54FF0FF324FF0FF33B7
:10E020000220F5F7E7F9022138600C3011F0D8FA38
:10E030004FF48D730380386801210C3011F0D0FA51
:10E04000012303706FF06800BBE700BF6850020057
:10E05000504802009C5002007C500200CC5002004C
:10E06000B8500200580100200F4B1B68DB0600D49B
:10E07000704710B50C3282B00C4601900221104658
:10E08000009211F0ADFA40F20541018004210098A0
:10E0900011F0A6FA4FF000030370019BA0F80140B5
:10E0A0001B78C37002B010BD58010020024A1368EB
:10E0B000013B1360704700BF18260020037F03F068
:10E0C0000303013B012B01D900DE7047034610B565
:10E0D00001F10C0282B001921046DA880421144644
:10E0E000009311F07DFA8446009B019A197F0093FA
:10E0F00001F0030102290CBF44F4005144F48051A3
:10E100000180597F1046ACF80210597F11F068FA6F
:10E11000009B5A7F03F11F0102B0BDE8104015F0CB
:10E120008EBB00BF2DE9F04186B00379C288032B76
:10E1300004460D46164604AF00F11C080BD0173BF1
:10E14000062B21D8DFE813F0250085008B00BA00EC
:10E15000D400E9000C01C37F033B122B14D8DFE885
:10E1600013F0400213001300D5016A021300740279
:10E17000130013001300F101130011021300380201
:10E18000130013003201320100DE0837BD46BDE83E
:10E19000F08118F0010F40F0B782237F9846002BE2
:10E1A00000F05A82B44B5B689800EED5B34B1B6805
:10E1B00003F4007213F0010340F06A811343E4D0CA
:10E1C00005F10C000546B8F1000F40F082820221F3
:10E1D000AB4A13680133136011F002FA41F63E7343
:10E1E00001210380284611F0FBF90A2203461E2173
:10E1F0001A70284611F0F4F90023A0F801600370AA
:10E20000637FC370A37F0371D4F81F30C0F805305B
:10E21000B4F82330A0F80930D4F82B30C0F80B3014
:10E22000B4F82F30A0F80F30D4F82530C0F81130F2
:10E23000B4F82930A0F81530638EA0F81730A38EFB
:10E24000A0F81930E38EA0F81B3094F838304377EB
:10E250009BE70A4640463146FFF706FF95E7864BA7
:10E260005B68990091D5854B1B685A078DD50221B3
:10E2700005F10C0011F0B4F940F63E2301210380B2
:10E2800005F10C0011F0ACF903220346092105F158
:10E290000C001A7011F0A4F918F0010F40F036824A
:10E2A000237FA0F801600370E38BA0F80330238C78
:10E2B000A0F80530638CA0F8073066E76E4B0024A9
:10E2C0005B681B047FF561AF01F10C031846022166
:10E2D0007B6011F085F94FF44C7C0246032178688D
:10E2E000A2F800C011F07CF90470A0F801604CE7BE
:10E2F000644B1B681C027FF548AF022105F10C003E
:10E3000011F06EF940F257220346022105F10C008C
:10E310001A8011F065F9068037E7574B5B68980063
:10E320007FF533AF554B1B6819037FF52EAF0221E4
:10E3300005F10C0011F054F940F23E430121038035
:10E3400005F10C0011F04CF91422034603211A7058
:10E3500005F10C0011F044F90680237F837014E767
:10E36000454B5B689A0003D5444B1B681B0553D48F
:10E37000607FA17F90FAA0F291FAA1F30028B2FA8F
:10E3800082F208BF4FF0FF320029B3FA83F308BFCF
:10E390004FF0FF3394F81CC001326C4601338AB051
:10E3A000062139480C9204AACDF82CC009900D938F
:10E3B0000A9642F8101F00234FF442513348F3F7F6
:10E3C00019FCA546E1E62C4B5B689A007FF5DDAEB3
:10E3D0002A4B1B685B067FF5D8AE022105F10C00C5
:10E3E00011F0FEF840F63E330121038005F10C00E8
:10E3F00011F0F6F8072203460A211A7005F10C0005
:10E4000011F0EEF80680A38C4380E38C8380238C8C
:10E41000C380638C0381B8E6022105F10C0011F082
:10E42000DFF840F23E630121038005F10C0011F09A
:10E43000D7F80C22034605211A7005F10C0011F0E3
:10E44000CFF8237FA0F801600370627F92FAA2F3F5
:10E45000002AB3FA83F308BF4FF0FF330133C370D0
:10E46000A27F92FAA2F3002AB3FA83F308BF4FF017
:10E47000FF330133037188E658010020500100206A
:10E4800018260020F8120020E05002005048020038
:10E4900005F10C00B8F1000F40F0F280A8490B68BC
:10E4A00001330B60002A40F033810221054611F050
:10E4B00097F841F23E3301210380284611F090F88D
:10E4C0000122034612211A70284611F089F880F8BB
:10E4D0000080A0F80160637FC370A37F03F0010395
:10E4E0000371D4F81F30C0F80530B4F82330A0F819
:10E4F0000930638EA0F80B30A38EA0F80D30E38EA8
:10E50000A0F80F3094F8383043743EE68D4B002469
:10E510001B681A067FF539AE01F10C03184602217B
:10E520007B6011F05DF84FF4816C0246042178683D
:10E53000A2F800C011F054F801230470A0F80160A3
:10E54000C37022E67F4B1B681B067FF51EAE01F1F0
:10E550000C03184602217B6094F8204011F040F82B
:10E560004FF4816C024604217868A2F800C011F0D3
:10E5700037F800239C4208BF1F24A0F80160C37035
:10E58000047002E66F4B5B6898006ED56E4B1B689B
:10E5900099066AD5022105F10C0011F021F840F628
:10E5A0003E330121038005F10C0011F019F8062219
:10E5B00003460A211A7005F10C0011F011F80680CB
:10E5C000238C4380638C8380A38CC380E38C038182
:10E5D000DBE590F8203002215C4A5D4810F0D1FD67
:10E5E000D3E5584B5B6898007FF5CFAD564B1B6861
:10E5F000D9067FF5CAAD022105F10C0010F0F0FF3D
:10E6000040F63E530121038005F10C0010F0E8FFB5
:10E61000052203460C211A7005F10C0010F0E0FFF2
:10E62000034623F8026B216A626AC0F802105A603E
:10E63000238D4381A9E590F820300E2B42D0022192
:10E64000444A434810F09DFD9FE50B463246414643
:10E650000020FEF779FE98E5FF22A07F04F1250354
:10E6600004F11F0106F0A8FF9CE500231A220221F5
:10E670003046CDE90233CDE9003301F011F984E5EC
:10E68000002A48D102217A60054610F0A9FF41F224
:10E690003E3301210380284610F0A2FF01240346E7
:10E6A000122128461C7010F09BFF7A6880F80080C9
:10E6B000C0F80120C0F80520C0F80920C0F80D20DE
:10E6C000427462E50B46324600211A20FEF73CFEFA
:10E6D0005BE5022110F084FF41F63E720346012102
:10E6E0001A80284610F07CFF0A2203461E21284685
:10E6F0001A7010F075FF04461D220021601C15F0F1
:10E70000C5F884F8008040E500DE46E500DEC7E598
:10E710000221054660E50221044610F061FF41F642
:10E720003E72034601211A80204610F059FF0A224A
:10E7300003461E2120461A7010F052FF0446DBE704
:10E740001826002058010020500100201C51020012
:10E75000504802000C51020030B500F10C0483B0A7
:10E760000D4620460221019210F03AFF40F2135C60
:10E7700003460521A3F800C0204610F031FF012315
:10E78000019AA0F801500370A0F8032003B030BD37
:10E790000379032B09D0172B05D0183B052B8CBF11
:10E7A00000200320704701207047037F03F003031C
:10E7B000032B14BF05200420704700BF2DE930084B
:10E7C00041F6FF7C4FF0FF3B0021094A0024C2E9DB
:10E7D00000BC0025074A1F2011600021064BC3E939
:10E7E0000045064BC3E90001BDE83008FEF79CBDBB
:10E7F0005801002018260020F812002050010020A7
:10E8000000B583B0DDF814C00D4A0E4BACEB02022C
:10E81000A3FB0232C2F347126AB90232012100207F
:10E82000094BCDF800C0D2B2FDF730FB10F0FD0F60
:10E8300003D103B000BD00DEEFE700DE03B000BD92
:10E84000402600204FECC44EE9E8000070B5036894
:10E8500006465D6DDDB100229C6D5A65F4B1002164
:10E860004FF0170E4FF6FF7C996504F11C0084F8F9
:10E8700004E0A4F806C01E2215F008F83C23A660A8
:10E88000237721462846BDE87040FEF77DB800DEBC
:10E8900000229C6D5D6D5A65002CE0D100DE9C6D00
:10E8A000DDE700BF0E4A0F4B12781A7000B97047AF
:10E8B00010B54B7F82B001EB83031B6A01911B787B
:10E8C0001C46FEF7EDF80199884201D102B010BD57
:10E8D00014F00E0F02D14B69002BF7D000DEF5E7E4
:10E8E0006A3A0020693A002000B1704708B5054B2C
:10E8F0000246996002200121FCF79AF800B908BD90
:10E9000000DE08BDB8040020014608B511F8103B30
:10E910007BB10D4B9960826892B90022DFF82CC060
:10E92000094BC0E902C101201146FCF781F828B962
:10E9300008BD0846BDE80840FFF788BF00DE08BDF7
:10E9400000DE9968E9E700BFA80400204DE8000058
:10E9500038B5134C6569AB6FB3B905F16C0105F1BE
:10E960006800FBF7E1FF0346C0B1AB6728680025EC
:10E9700000F014FFA06D6561FDF7F4FF606DA56503
:10E98000FDF7E4FF656538BD00DE05F16C0105F1BA
:10E990006800FBF7C9FF03460028E6D100DEE4E784
:10E9A0004026002030B5334C85B094F85E0010F05E
:10E9B000010039D0636953B193F82C2042F0020270
:10E9C00083F82C20636993F82C30DA0744D4294863
:10E9D000FEF74EF8A04242D1237EDB0726D403ADDA
:10E9E000022203210020244B00950392FDF74EFAEA
:10E9F0002946FEF727F850BB2048FEF775F8002897
:10EA000031D11C48FEF740F8A0422AD163690BB10E
:10EA1000FFF79EFF94F85E30002023F0010384F896
:10EA20005E3006F077FF002005B030BD4FF0020CDD
:10EA300003AD0321012200200F4B0095CDF80CC03F
:10EA4000FDF724FA2946FDF7FDFF0028C8D0094844
:10EA5000FEF71AF8A0420AD10C2005B030BD00DE46
:10EA6000BAE700DED2E77830CBD000DEC9E700DEBF
:10EA7000F2E700BF4026002081C0000050260020A1
:10EA800000B5037891F801C003F00F03511E0CF19B
:10EA9000100C89B2062B12D8DFE803F004261611F9
:10EAA0001111040043781033DB0003F21B3202EB38
:10EAB000CC0003F5B37313FB010080B200BD40F23C
:10EAC00053204FF4F373F6E790F801C001EB810394
:10EAD000C3EB031040000CF11003DB0000F23B100D
:10EAE00003FB020080B200BD40F2E33040F2162387
:10EAF000E1E700BF10B514464FF6FF728CB09342A9
:10EB00009DF838E01CD0DDF83CC00F991CF8102BA4
:10EB10000132D2B20A70002A4DD000222849C1E940
:10EB20000004887A0B81274B6EF300008872C1F8CD
:10EB30000CC0996001201146FBF77AFF00283CD1F8
:10EB40000F9B187E10F0010205D11F481F4B017862
:10EB50001B788B4201D00CB010BD0133037004212F
:10EB60000BA8099207F07EFC42F2107E184B0F9A18
:10EB70001849DFF864C0059318480B9B511AACFB89
:10EB800001C1A0FB03C0400B0EFB103306924909E4
:10EB9000099A02311046CDE9022204920192013312
:10EBA0000092CAB201210B93FDF74AF910F0FD0F54
:10EBB000D1D000DECFE700DEAFE700DEC0E700BF68
:10EBC00000130020980400206A3A0020693A0020CF
:10EBD000A5E80000402600204FECC44E5917B7D1DD
:10EBE00070B5184C0226204607F0F6FF04F10C0021
:10EBF00007F0F2FF4FF4006506224FF0000E4FF0D1
:10EC0000040C34F8043C94F8421023F4437323F0CA
:10EC1000020343F00E0324F8043C637866F34201D8
:10EC200004EB83035B6884F84210A4F8405083F837
:10EC300000E05A70637B04EB8300036983F800C033
:10EC40005A7070BD5C2600202DE9F0431C46624BD3
:10EC50000E4693F85E50614983B015F001050746F2
:10EC600003C99DF82CC09DF830E000908DF8041089
:10EC70007FD1012E14BF384600200DEB0601A046BF
:10EC800014460A78A3F85C0002F00F0212F00E0F8F
:10EC90000CBF01200020198B0CF0070C0EF0030EA6
:10ECA0004FEA4C0C21F4437121F002014CEA0E2C86
:10ECB0004CEA010C597FA3F818C003EB81010E6ADE
:10ECC000317821F01F0C42EA0C0260F345123270D9
:10ECD00002F00F02012A01F00F0942D093F85E20E2
:10ECE00064F34202510783F85E200BD568F3C30238
:10ECF00083F85E200A9A3A491268C3F85F200A9A9C
:10ED000092888A80327804F0010702F00F0101290D
:10ED100034D07178E9B1B9F1010F4CD0327867F392
:10ED2000861222F08002327093F829201B6103EBD7
:10ED30008203DB6AA40104F040045A7844F004041E
:10ED40001C7012B9062115465970284603B0BDE85B
:10ED5000F08367F3861261F3C71232700622727075
:10ED6000E2E7B9F1010FB9D07278BAB983F834503B
:10ED7000B4E70C25284603B0BDE8F083314667F3BD
:10ED8000861268F3C71201F8082B0C220A98006853
:10ED9000B0600A98808888807270C5E7052A17D904
:10EDA000063AD2B20F4806F1080183F8342014F075
:10EDB00046FD094B92E793F834200A4906F1080012
:10EDC00014F03DFD044B93F8342006327270A5E731
:10EDD00000DE7278E4E700BF4026002064490200AC
:10EDE0009F2600207526002008B5FFF7F9FE0020B9
:10EDF00008BD00BF08B5FFF7D5FD002008BD00BF66
:10EE000008B5054807F0F8FE044807F0F5FEFFF7DF
:10EE1000E7FE002008BD00BF5C2600206826002019
:10EE2000034A044B801AA3FB0030C0F34F10704715
:10EE3000402600204FECC44E044A0068044B801A60
:10EE4000A3FB0030C0F34F10704700BF40260020E6
:10EE50004FECC44E38B9054890F85E3013F0010FFE
:10EE600008BF002070470020704700BF40260020E8
:10EE700028B9044B93F85E0000F0010070470020B1
:10EE8000704700BF4026002040B9054B93F85E2034
:10EE9000D20703D5587E00F003007047002070476A
:10EEA0004026002030B5054683B0807E0C4606F033
:10EEB00055FE30B3237843F0400323700268237873
:10EEC000C4F80220828803F00F03012BE28004F1D2
:10EED000020202D0104603B030BDA87E019206F0B7
:10EEE00055FE019A0028F5D02346217841F0800193
:10EEF00003F8081B0168A16081881046998003B05F
:10EF000030BD2078C0F38010FDF776F8D6E700BF5B
:10EF1000002800F0F3802DE9F047BE4C8EB094F845
:10EF20005E5015F0010540F03D81FF23607EA37621
:10EF300000F0030006F00CFD94F85E00420700F1BB
:10EF4000CE80627F94F8293004EB820204EB8303C5
:10EF5000DB6A166A984686B13146AE48FFF7A2FFD3
:10EF600033785B0605D50621FBF7CEFC002800F0C0
:10EF70004A814146A748FFF795FF337813F00E0FFB
:10EF800040F09B80636923B10C2528460EB0BDE894
:10EF9000F087FDF7D5FC0746002800F04D81FDF70E
:10EFA000DBFC8146002800F0448100F0F1FB0346C1
:10EFB000002800F03B814FF6FF728284D0F8880071
:10EFC00003F1100A002800F0398103F17C0203F1FB
:10EFD00078010B93FBF7A4FC4FF4C02100220B9B9C
:10EFE000C3F88E11B3F87610184621F4EF6121F0C2
:10EFF000070141F48C7141F00101A3F8761093F8F8
:10F000003710C3E9122201F03F0161F07F0183F85C
:10F01000371093F88E10C3F8882021F0070183F889
:10F020008E1093F83C10A3F88C2021F00F0183F888
:10F030003C1083F839205A85C3F82E201A65A3F8AE
:10F040006021A3F89421A3F88A2102F073FE002224
:10F050000B9B83F86421C3F8687100F091FE0B9B51
:10F0600093F89C1160F3020183F89C1100F08EFE6E
:10F070000B9B012193F89CC160F3C50C93F86201CE
:10F0800083F89CC120F0020083F86201184601F069
:10F09000D1FC0B9B03F1E00002F060FC00220B9B13
:10F0A000C4E91579C4F814A0C3E902221A701B61DF
:10F0B00007F066FC002840F0A880237E0121C3F3FE
:10F0C00042030DF133008DF83330FBF7CBFDB8B9B7
:10F0D0006369002B3FF458AFFFF73AFC54E72A4628
:10F0E00004F15F01C0F3C00006F062FDFF28A076C6
:10F0F0003FF427AF284606F045FC22E7FFF752BC55
:10F10000024641463046FFF7BBFC0022B4F85C10D3
:10F11000C4E902220B9122706060FCF72DFF0B996D
:10F12000002200F2131339B9327802F00F02A2F173
:10F130000102B2FA82F25209207E666862F3000090
:10F14000207610F0010032D00020022232490496CD
:10F15000019609910694314F086031490DAE059131
:10F16000CDE9020003210090079708960B930D92BA
:10F17000FCF7F4FD3146FDF765FC0028A8D102221A
:10F180000D92284A03210592274ACDE903000092F7
:10F19000CDE9010001220B9B079708960694FCF726
:10F1A000BDFD21E0002528460EB0BDE8F08740F205
:10F1B0007122A1FB021201914FF6FF710222049607
:10F1C000039106F51C5614491036069402900090DF
:10F1D0000E60099111490DAE0791114908960591EC
:10F1E00003210D92FCF7BAFD3146FDF72BFC0028F8
:10F1F0007FF46EAF012094F85E30034384F85E30F4
:10F2000006F088FBC1E61225BFE6FFF7A1FB032548
:10F21000BBE600BF402600203426002081C000004D
:10F22000F5EA000001E80000728E13004846FDF781
:10F2300099FB3846FDF78AFB0725A6E603F1800017
:10F24000C3F88800C1E600BF70B50446237E8AB0CB
:10F25000C3F342030D460DF12300012116468DF83C
:10F260002330FBF7FFFC314602462846FFF708FC37
:10F2700063680546834221D90022191A0192134A74
:10F28000134B02910221A21AA3FB0232002301EBCD
:10F29000521209910F4909AE059118460321CDE993
:10F2A00003330696D2B20093FCF7CAFD3146FDF750
:10F2B000C9FB38B9656000200AB070BDFBD20021DF
:10F2C000C21ADBE70C200AB070BD00BF4026002048
:10F2D0004FECC44E81C000001F2961D8F0B517461D
:10F2E000427F034600EB8202166A0D46327885B0F3
:10F2F00002F00F02012A55D00DF10F011C300193CD
:10F3000007F0CEFC3146044696F800E090F800C0C5
:10F310000EF00F0E2CF01F0C4CEA0E0C80F800C003
:10F3200096F800C090F800E0CCF3401C6CF3451E4A
:10F3300080F800E036785FFA8EFCC6F3801666F33C
:10F34000861C80F800C011F8026B5FFA8CFCF6098D
:10F3500066F3C71C062200F802CB14F07EFA2A4698
:10F36000394604F1080014F06AFA0635019B65700D
:10F3700093F85E20D20705D49DF80F205A7700201D
:10F3800005B0F0BD93F82920184603EB8202214610
:10F39000D26AFFF759FF019B0028EDD00C20EFE760
:10F3A000122070470A4680F834503946353014F040
:10F3B00046FAE4E70A4601460148FFF78DBF00BF61
:10F3C000402600201F295ED8F0B590F82930174656
:10F3D00000EB8303DB6A04460E4685B0002B43D066
:10F3E0000DF10F0104F12800019307F059FC0622EA
:10F3F00005460378019923F03F0343F004030370AB
:10F4000011F802CB03F03F03CCF3801C06EB020E95
:10F4100043EA8C132B7085F801E0023014F01DFADA
:10F420003246394605F1080014F009FA94F85E30C6
:10F43000DA0706D400209DF80F3084F8293005B093
:10F44000F0BD4123627F04EB8202116A0A7802F068
:10F450000F02D340DB07EDD52A462046FFF7F4FE26
:10F460000028E7D00C20EAE7283007F0B5FBC0B24F
:10F4700058B9042294F8293004EB8303DB6A1A702C
:10F4800006225A70ACE7122070470720D7E700BF6A
:10F490000A4601460148FFF795BF00BF40260020FD
:10F4A000002208B5044B114698600120FBF7C0FA12
:10F4B00000B908BD00DE08BDC804002083685A6892
:10F4C00092F82730DB0901D100DE704700F1080116
:10F4D00005F0D8BA2DE9F0410546076882B04FF42F
:10F4E000D47223493846FBF7F9F9294607F0A8FFFB
:10F4F000E86E01AA05F16801FBF72EFA10B34FF68A
:10F50000FF781C4C94F8412094F84010531CDBB257
:10F51000082B08BF0023994225D0019904EBC20CA7
:10F5200024F83280CCF804100A680260019A106056
:10F53000E86E01AA05F1680184F84130FBF70CFA86
:10F540000028DFD1D7F8680107F5B47138B100237E
:10F55000C7F86831FDF792FB02B0BDE8F08100DE2C
:10F56000D7F86801F3E700DE00231B80FFDE00BF51
:10F57000101300207827002000B583B048B9084652
:10F580000191FDF79FFA0199814200D000DE03B09E
:10F5900000BD00DEF3E700BF00B583B048B9084600
:10F5A0000191FDF783FA0199814200D000DE03B09A
:10F5B00000BD00DEF3E700BF10B50C4640B9074BB5
:10F5C0000246012102209C60FBF732FA20B910BDEF
:10F5D000FDF766FA8442FAD000DE10BDE804002090
:10F5E00000B9704710B50C46FDF778FAA04200D17B
:10F5F00010BDFDF755FA8442FAD000DE10BD00BF01
:10F600002DE9F04104468CB00E46012002211D4632
:10F61000174609F0C1FB0022022180460120FBF7BA
:10F62000CFF94FF4D4721D492046FBF757F91C4B14
:10F63000C21CD2B2009301212B46002001940B92F0
:10F64000FCF75EFC10F0FD0F0B9A25D10894069490
:10F650000197616800204FF6FE742B46114D04910E
:10F660000795114D0121CDE9020400960595FCF79F
:10F6700055FB10F0FD0F0DD1B8F1000F02D10CB009
:10F68000BDE8F0810122022110460CB0BDE8F04136
:10F69000FBF796B900DEEFE700DED7E71013002096
:10F6A00099F5000079F50000D549010008B501225F
:10F6B000194B4FF4D4711948FBF7BEF800224FF4F0
:10F6C000D4711648FBF706F94FF6FF7E8446144BBB
:10F6D000ACF824E0181D03222421FBF7ADF8114BF0
:10F6E0000722181D0821FBF7A7F802F007FB4FF0CF
:10F6F0001B0E4FF4A47103234FF0000C0A4A0B4871
:10F70000A2F800E00A4AC0F800C0118009490A4A7C
:10F710000B70137008BD00BFC82600201013002016
:10F7200008270020CC26002044380020E0270020B5
:10F73000423800206C3A00206B3A0020844608B51D
:10F740001CF8102B7AB10F4BC3F808C08268AAB915
:10F7500000220D490B4BC0E9021C01201146FBF7AA
:10F7600067F948B908BD094B11460120C3F808C024
:10F77000FBF75EF90028F5D000DE08BD00DED3F807
:10F7800008C0E5E7D8040020A1F40000C804002068
:10F790000148FBF777B800BFC82600200149FBF7F6
:10F7A00085B800BFC82600204FF4D4720149FBF78A
:10F7B00095B800BF1013002028B902464FF4D47149
:10F7C0000248FBF787B80020704700BF10130020E5
:10F7D00060B9024608B54FF4D4710648FBF77AF8D1
:10F7E00030B1838C002B18BF002008BD002070476B
:10F7F000002008BD101300200148FBF743B800BFEC
:10F80000082700200149FBF751B800BF0827002056
:10F8100058BB38B502460D461E484FF4D471FBF76D
:10F8200059F80446F0B1828CE2B91B4890F821C027
:10F8300090F820100CF10103DBB2042B08BF134633
:10F84000994224D020F83C2000EBCC0CCCF804509A
:10F8500080F8213023785BB994F93730002B11DB25
:10F86000002038BD6FF0150038BD6FF015007047EF
:10F870000A4B012103209C60FBF7DAF894F937303A
:10F88000002BEDDA0021204605F0C4FAE8E76FF01E
:10F89000680038BD10130020BC270020F8040020A9
:10F8A0002DE9F04784B0BDF83060BDF83470BDF884
:10F8B0003880A0B991460D4602464FF4D4711D48D8
:10F8C0009A46FBF707F8044648B1838C3BB99DB1D3
:10F8D000022D09D00125284604B0BDE8F087022595
:10F8E000284604B0BDE8F0874D46D5B902F06EFC5D
:10F8F000284604B0BDE8F0870F9D3B46019532468F
:10F900005146CDF8008002F0E9FB05460028E7D11A
:10F9100094F937308342E3DA0146204605F07AFA5B
:10F92000DEE74946039302F061FC039D284604B0DC
:10F93000BDE8F08710130020D0B910B502460C4680
:10F9400082B04FF4D4710F48FAF7C4FF68B1828CCB
:10F950005AB9019002F048FB019B58B1036823603B
:10F9600003792371002002B010BD022002B010BD47
:10F9700002207047D3F83220226093F8363023718A
:10F98000F0E700BF1013002010B1022108467047B5
:10F9900000B583B00246019117484FF4D471FAF7CD
:10F9A00099FF019B024618B3818C09BB1A2B17D80B
:10F9B000042B19D91149D940C90715D51946104644
:10F9C000019202F0F7FA014678B9019A92F93730BC
:10F9D00083420ADA0190104605F01CFA019904E00E
:10F9E000292BEBD03B2BE9D01221084603B000BDF8
:10F9F0000C21084603B000BD10130020200038047D
:10FA0000E0B900B5024683B04FF4D4711148FAF75B
:10FA100061FF78B1828C6AB90121019002F076FA17
:10FA2000014620B9019B93F93720824209DB084641
:10FA300003B000BD0221084603B000BD0221084604
:10FA400070470190184605F0E5F90199084603B0A2
:10FA500000BD00BF10130020D8B900B5024683B026
:10FA60004FF4D4711048FAF735FF70B1828C62B947
:10FA7000019002F063FA014620B9019B93F9372007
:10FA8000824209DB084603B000BD0221084603B0EC
:10FA900000BD0221084670470190184605F0BAF9EA
:10FAA0000199084603B000BD1013002038BB30B5E3
:10FAB00015460C46024683B04FF4D4711448FAF749
:10FAC00009FFA0B1828C92B9D0F84021930612D5DB
:10FAD00021462A46019002F099FA014620B9019B7D
:10FAE00093F9372082420DDB084603B030BD022176
:10FAF000084603B030BD1A21084603B030BD0221CC
:10FB0000084670470190184605F084F90199EBE723
:10FB100010130020034A044B12881B8802800B80BC
:10FB2000704700BF4438002042380020024A034B8F
:10FB3000108019800020704744380020423800208F
:10FB400030B54FF4267C1B2445254FF4A47E048059
:10FB50001580A1F800E0A3F800C030BD38B5B8B9F1
:10FB600015460C4602464FF4D4710B48FAF7B2FE24
:10FB700070B1838C63B990F876C0CCF3020C84F832
:10FB800000C090F877101846C1F30201297038BD03
:10FB90000223184638BD00BF10130020024A034B51
:10FBA00010701970002070476C3A00206B3A0020EA
:10FBB00060BBF0B516460D4602464FF4D4711848A6
:10FBC00085B01F46FAF786FE0446B8B1838CABB900
:10FBD000D0F84031DB0515D54FF0010C29463B46E6
:10FBE0003246CDF800C002F0BBF9014618B994F9CD
:10FBF000373083420DDB084605B0F0BD02210846D0
:10FC000005B0F0BD1A21084605B0F0BD0221084636
:10FC100070470390204605F0FDF80399EBE700BF1D
:10FC20001013002060BB10B502460C4615484FF477
:10FC3000D471FAF74FFE08B3838CFBB9C38CB0F8CC
:10FC40008C21052B0ED84FF4FA7101339BB202FBC5
:10FC500003F301FB03F30C4AA2FB03235B0B23809A
:10FC6000002010BD40F2E24103FB02F201FB02F270
:10FC7000054BA3FB0232520B2280F1E7022010BD9C
:10FC800002207047101300205917B7D138BB00B5B8
:10FC900083B00246019113484FF4D471FAF71AFE6B
:10FCA000D0B1828CC2B942F21071C28C019B052A7C
:10FCB00003FB01F18FBF40F2E2434FF4FA730132CC
:10FCC00092B203FB02F201391144B1FBF2F1A0F848
:10FCD0008C11002003B000BD022003B000BD022043
:10FCE000704700BF1013002008B5FFF7DFFC0020AD
:10FCF00008BD00BF38B500224FF4D4711948FAF797
:10FD0000E9FD044658B32146032004F11002FCF734
:10FD100015FF054610B110F1780F0BD10025124ADE
:10FD2000124BC4F888501584A3F84050FFF7BEFC6E
:10FD3000284638BD40F24D730D4A0E490E480EF06C
:10FD4000CDFD2A4600210D480EF0C8FD002383F3A7
:10FD50001188BFF36F8F0323184602DFDEE700DE52
:10FD6000D1E700BF10130020BC2700207827002017
:10FD70004051020088510200A0510200C05102000F
:10FD8000014B1878704700BF6C3A0020014B18787F
:10FD9000704700BF6B3A00208A68086013681878C3
:10FDA00028B19A6852B9084AC3E9022170475268DB
:10FDB00092F82730DB0903D100DE704700DEF2E75E
:10FDC0000846083104F05EBEBDF400000B68DA8816
:10FDD000002A34D130B505460C4683B04FF4D471B7
:10FDE0001F48FAF777FD28B3828C1ABB019002F006
:10FDF00039FAD4F800C0019B9CF81C2002F00302E1
:10FE0000032A0AD10122294618468CF804202268C8
:10FE100003B0BDE8304002F039BA9AB193F86221DC
:10FE2000910705D53D21012283F8641123681A71D9
:10FE300003B030BD012223681A7103B030BD012226
:10FE40001A71704793F86221920704D53D2283F816
:10FE50006421D4F800C001238CF8043003B030BD15
:10FE60001013002010B504464FF6FF70B4F824C0FC
:10FE700084450CD02046A4F82431C4E9471201F08F
:10FE8000D1FF94F8623113F0010002D110BD00DE01
:10FE9000F0E723F0010384F862316FF08B0010BDAE
:10FEA00070B51C4C064694F821201EE04FF4D47126
:10FEB0001948FAF70FFD0346E03003B39B8CF3B902
:10FEC000696801F06DFD94F8201094F821204B1C16
:10FED0008A42DBB206F1FF3004D0042B08BF0023B6
:10FEE00084F8203010F0FF0613D094F820309342AD
:10FEF0000FD034F8332004EBC305002AD6D069684C
:10FF00004FF6FF700B7923F003030B71FCF77CFDB8
:10FF1000D9E770BDBC27002010130020F0B5324B8C
:10FF20000A4619680546884208BF002183B008BF09
:10FF300019601823808C012185F8842185F86C31A3
:10FF4000A5F86E01284601F079FF284601F090FFE0
:10FF500005F1E00001F00EFD05F1E00001F040FDCB
:10FF6000044630B3037905F17C0703F00303032B48
:10FF70000CBF0346002303601C48FAF783FCB0B1B2
:10FF800021463A46FAF7DAFC05F1E00001F028FDD7
:10FF9000044670B1037903F00303032B0CBF03463F
:10FFA000002303601148FAF76DFC0028E8D100DE59
:10FFB000E6E7AA8C0121033220460D4B0095D2B210
:10FFC000FBF764FF10F0FD0F08D14FF6FF73FF2021
:10FFD000AB8403B0BDE8F040FFF762BFFCF760FD03
:10FFE0008542F2D000DEF0E7E0270020CC2600209A
:10FFF000B9F500004FF6FF732DE9F04184688CB02D
:020000021000EC
:10000000A28C9A4200F0B7800746204602F02AF9F7
:100010003B7D012B00F0DA80022B00F0AF8033B97A
:1000200094F88E3003F01803182B00F0148194F824
:100030006461002E40F0A680E38DCDE90A66984603
:100040003B8A94F93720002B00F0A380B242C0F223
:100050001C810023A4F89031BB7CA58D03F0030321
:100060000135012BADB200F00C81B4F89431002BB6
:1000700000F0B280AB4240F22D815B1B9BB2062B9D
:10008000A4F894318CBF0023012300221E46E28590
:1000900094F83C20294663F3820284F83C202046F1
:1000A0000DF1270201F082FE743000F00D81B4F8EA
:1000B0008E312BB1AB4240F2B7805B1BA4F88E317E
:1000C000B4F88A312BB1AB4240F2BE805B1BA4F87E
:1000D0008A31E58D16B9A84500F0A1800135ADB291
:1000E00094F8D13013F001070DD1DDE90AC363BBE9
:1000F000BCF1000F40F095800DB9002E3BD00027D9
:1001000039463B4622E094F9372023F00103002AC8
:1001100084F8D1307BDB94F87600C0F3C00100F0A6
:10012000070006F07DFAB4F86E20B4F86C30616810
:100130001344E28B03F23F13134418448142DDE978
:100140000AC380F0B880471A60600021A28C7F4803
:10015000246903320291059001210020CDE9035664
:1001600006940197CDF800C0D2B2FBF769FE10F0FB
:10017000FD0F40F0B9800CB0BDE8F0813D231E4674
:1001800084F86431314620460CB0BDE8F041FFF7F9
:10019000C5BE9A42B8BF84F8D560BB7CA58D03F07C
:1001A00003030135012BADB26BD0B4F89031002BB5
:1001B0003FF45BAFAB4240F292805B1BA4F89031FE
:1001C000B4F89431002B7FF455AF61E70023A4F815
:1001D0008E31A4F88A312AE7E28C42F21071052AA6
:1001E0008FBF40F2E2434FF4FA73013292B203FB45
:1001F00002F2B4F8923101FB0323013BB3FBF2F3AB
:100200009BB2A4F89431002B7FF434AF40E794F80C
:100210007700012100F0070006F004FA83E7354675
:100220005EE71F46194691E7FCF7DCFB002862D029
:100230000023A4F88E311B23A28C0146C2800371D7
:100240000068FCF7A1FB3BE700232046A4F88A31B5
:1002500001F04AFE3DE7218DB4F88C218B1D9A42B6
:10026000D2BF1346931F5B1AB4F88811C8BF9BB264
:10027000994244D0A4F88831A4F88A31A4F88E2198
:10028000D5E60023A4F8943102E794F8D530002B8A
:100290003BD0013B84F8D53004F1E005284601F05D
:1002A0009DFB00284ED0284601F098FB00283BD04B
:1002B0000023E385CDE6091A60609BBB51EA0C027E
:1002C0003FF41AAF1F4641E720469DF82710FFF77D
:1002D00025FE50E708212046FFF720FE4BE73E2190
:1002E0002046FFF71BFE46E7FCF7DAFBA0423FF48F
:1002F00042AF00DE3FE70123A4F88E31E0E6B4F818
:100300008E1100297FF493AEB6E70AAA38460BA9EE
:10031000FCF7F8FDDDE90A231343BDD0237884F808
:10032000D530B9E7002711E70246D4E91E01FAF7F4
:100330000BFB0028BCD194F83C301B0744BF238D35
:10034000E38586E6FF20FFF7ABFDACE7E1F50000B3
:1003500010B5044682B00120FFF7A2FD04F1E000D1
:1003600001F03EFBB8B1014603790C4803F00303EA
:10037000032B0CBF0B4600230B600191FAF782FAA6
:10038000019930B104F17C0202B0BDE81040FAF7E7
:10039000D5BA00DEF6E702B010BD00BFCC260020C3
:1003A00019B3F8B54D1E00F1E00700F17C0613E02B
:1003B00003790E4803F00303032B0CBF23460023ED
:1003C0002360FAF75FFA70B1013D32462146EDB283
:1003D000FAF7B4FAFF2D05D0384601F001FB0446C8
:1003E0000028E5D1F8BD00DEEEE77047CC260020FE
:1003F0000149FAF75BBA00BFCC260020014B93F805
:10040000410070477827002000B50A4B93F840C0A0
:1004100093F841E0F4450AD080F800E033F83C005E
:1004200003EBCC0308805B681360186800BD0020F4
:1004300000BD00BF78270020074B93F840C08445DB
:1004400008D003EBCC0033F83C300B8043681360DA
:10045000186870470020704778270020094A92F8F2
:10046000401092F841308B4209D04B1CDBB2082B74
:1004700008BF002352F8310082F840307047002056
:10048000704700BF7827002000B50D4A92F841C0A0
:1004900092F840E00CF10103DBB2082B08BF002307
:1004A0009E4508D022F83C0002EBCC0CCCF804109E
:1004B00082F8413000BD00DE00231B80FFDE00BF5C
:1004C00078270020134610B50C465979024682B0B1
:1004D000002940D0197901F0030003280DD04FF610
:1004E000FF70824204BF21F00301197119461046C2
:1004F00002B0BDE81040FCF787BA4FF6FF718A42A0
:1005000006D12168994234D00029EFD000DEEDE712
:100510001ABB4FF4D4711B48CDE90023FAF7DAF97E
:10052000DDE9002300282BD019460192009301F049
:100530007BFE2168009B019A9942E5D100224FF48D
:10054000D4711048FAF7C6F9009B90B1828C002A4A
:1005500018BF00200EE000DEBCE7019200DE0020A4
:100560001946009301F060FE2168009B019A9942B0
:10057000CAD10020194602B0BDE8104001F010BCFD
:1005800000DED1E71013002090F86620B0F85C3050
:10059000C2F30212022A15BFDB089B080A3B0B3B81
:1005A0009BB290F87E101A1F11F0100F92B218BF74
:1005B0001346B0F85800984228BF184680B27047DA
:1005C000704700BF90F8623143F0020380F8623157
:1005D000704700BF90F8623123F0020380F8623167
:1005E000704700BFB0F86031B0F82421981880B28D
:1005F000704700BF0278038E12B1581E80B2704758
:10060000418DB0F824215818104480B2704700BFC3
:100610002DE9F04F044685B0CDE90223B0F86061C2
:10062000B0F8243190F876001E44D4F81C310091C3
:10063000C0F3C00100F00700BDF844B00193BDF85D
:100640003890BDF83C80BDF8407005F0E9FFE28CC1
:10065000A6EB0B0A052A019B1FFA8AFA73D940F20E
:10066000E24C12FB0AF292B24FF09611E161962130
:10067000B9F1050F21845ED9B4F86E50B4F86C104E
:10068000294401F2D51108444D4640F2E2410CFBE9
:1006900002F201FB05F5ABEB06019E1A013A2A4472
:1006A000B2FBF5F2B4F86031B4F82AE06060B4F857
:1006B000240194F837C01144034486440B4492B299
:1006C00071445FEADC1C05FB0266A4F860316185B9
:1006D00040D100DE4FF0000AAB4629462046A4F880
:1006E0002690A4F82880A4F8927101F091FB394B70
:1006F000228DEB18B3FBF5F3911D9A1A98B2063AC6
:10070000A4F88C31884288BF1346A4F88831009B36
:1007100013B10023A4F8943133465A46514620467B
:10072000FEF76EFF94F8623143F0010384F8623102
:1007300005B0BDE8F08F09F101054FF4FA7140F200
:100740001310ADB2A3E7013212FB0AF24FF4FA7CA8
:1007500092B289E70023216CC4F8DC30A36C0192CB
:1007600001FB003301FB1A33A36406F055F98346FD
:1007700094F8D400C0F3420006F050F9834405FB1E
:100780000BFB154B0BF5742B0BF23F2BA3FB0B3B19
:10079000019A4FEA9B4303FB02F22364A5EB030B90
:1007A000A36CB61A1A446B08963B9A4228BF1A46A5
:1007B00040F2E241C4E91132029B039A01FB03F3C8
:1007C0002365064BA3FB023A4FEA9A2A01FB0AFA79
:1007D00083E700BF7FC3C90183DE1B435917B7D12D
:1007E0000B4610B504461A683230C4F832201B7923
:1007F00005210371FAF736FA94F8373060F30503F0
:1008000084F8373010BD00BF4FF426704FF4A47346
:1008100008801380704700BF30B5B0F86020B0F892
:100820005A1003468A4228BF0A4690F87700B3F868
:10083000641000F00700B3F85EC01B2A38BF1B220B
:10084000042814BF4FF4A4704FF42960614528BFF9
:100850006146814238BF0146B3F86E50B3F86A4032
:100860008D4244D0A242A3F86E1001D0A3F86A20B2
:10087000012093F8D12042F0020283F8D120B3F88E
:100880006220B3F8581093F876C08A4228BF0A460F
:100890000CF0070CB3F86610B3F85C501B2A38BF95
:1008A0001B22BCF1040F14BF4FF4A47C4FF4296C3D
:1008B000A94228BF2946614538BF6146B3F86C405C
:1008C000B3F868E08C4216D07245A3F86C1001D0E2
:1008D000A3F8682093F8D12022F0020283F8D120F7
:1008E000012093F8D120024383F8D12030BDA242E9
:1008F000BCD10020C3E77245EAD193F8D11041EA98
:10090000510202F0010221F003010A4383F8D120D1
:100910000028E5D130BD00BF10B5B0F86020B0F8B8
:100920005A1003468A4228BF0A4690F87700B3F867
:10093000641000F00700B3F85E401B2A38BF1B228A
:10094000042814BF4FF4A4704FF42960A14228BFBB
:100950002146814238BF0146B3F86EE0B3F86AC061
:100960008E450DD09445A3F86E1001D0A3F86A20EF
:1009700093F8D120012042F0020283F8D12010BD6B
:100980009445F3D1002010BD10B5B0F86220B0F846
:10099000581003468A4228BF0A4690F87600B3F8FA
:1009A000661000F00700B3F85C401B2A38BF1B221A
:1009B000042814BF4FF4A4704FF42960A14228BF4B
:1009C0002146814238BF0146B3F86CE0B3F868C0F5
:1009D0008E4513D06245A3F86C1001D0A3F86820AF
:1009E0000122104693F8D11042EA510202F00102AE
:1009F00021F003010A4383F8D12010BD6245EDD1F7
:100A000093F8D110002001F00102EDE71B2928BF67
:100A10001B21B2F5A47F28BF4FF4A472044BA0F8A9
:100A20007210C365A0F87020A0F85810704700BF7E
:100A30004801980210B5324B324A1B8812881B2B92
:100A400028BF1B23B2F5A47F28BF4FF4A4724FF038
:100A5000000CA0F87230A0F8583090F87730A0F869
:100A6000702003F0070301F00302042B02F12803B6
:100A700002F15202C1F340014FEAC3034FEAC2023E
:100A800023FA01F322FA01F29BB292B214BF4FF49F
:100A9000A4714FF429619342A0F86430A0F8663045
:100AA00028BF1346C0F868C0C0F86CC0A0F874C076
:100AB0004FF0450CA0F85E204FF4A4728B4238BF73
:100AC0000B46A0F85AC01B214FF01B1CA0F85C205D
:100AD00090F8D120044642F0020280F8D120A0F81C
:100AE0006E30C0F860C0A0F86A10FFF74DFF012219
:100AF00094F8D13084F87420134384F8D13010BDB9
:100B0000443800204238002008B50022D0E91E01F8
:100B1000F9F71AFFB0FA80F0400908BD30B583B08C
:100B200005460C4601F036F830B9204601F078F859
:100B30000323A37203B030BD2146284601F032F8EA
:100B40000146002838D00B1D18460193009102F091
:100B500045FC00992846CA79627301F039F82846A5
:100B600003F0D0FC0022019B009958689B68C4F8F0
:100B70004300C4F847300B69C5F8AC30A369A261E3
:100B8000E3B14FF0030C1A7983F804C0AD8C204612
:100B900003F11C01DD800192009302F009FC019A2F
:100BA0002E2A03D00423A37203B030BD0099086835
:100BB000FBF7EAFE0423F6E700DEC4E700DEE0E729
:100BC00070B582B004460D4600F0E4FF18B9062364
:100BD000AB7202B070BD04F18F03002205F13B013E
:100BE00005F12B00019308F039FA0022019B94F8DB
:100BF000C800D3F804E0D3F808C0DB6862F3000053
:100C0000C4F8BC30D4F8A83084F89F2084F8A02021
:100C100084F8A12084F8A22084F8A32084F8A420DA
:100C200084F8A52084F8A620C4F8C9300022002347
:100C300094F8A710C4E93023D4F88F60D4F8AC300E
:100C400041F0010184F8C80084F8A7102046294625
:100C5000C4F8B060C4F8B4E0C4F8B8C0C4F8CD308B
:100C600000F0A0FF0146B8B1081D019102F0CEFBD3
:100C700001992046CB796B7300F0AAFF204603F060
:100C800041FC4FF4C1636B8194F88E3043F008034C
:100C900084F88E3002B070BD00DEE5E730B5054661
:100CA000887A0C4683B00D2800F22A81DFE800F034
:100CB00060686B949E07070C1836393E5154002A21
:100CC00000F0A68003B030BD002AFBD121462846A3
:100CD00000F060FF002840F0EB800723A372F1E7EB
:100CE000022AEFD10023A069A361002800F0278128
:100CF00003230371AB8CC380237A052B00F005819D
:100D0000062B00F0FF8000DE2146284600F042FF5F
:100D1000002840F084800923A372D3E7002AD1D1B0
:100D2000F2E7002ACED10B23A372CBE7072AC9D161
:100D30002846012100F050FF2846FFF743FC2146DA
:100D4000284600F027FF002840F094800C23A3726F
:100D5000B8E7002AB6D1F2E7082AB3D140F202334D
:100D6000638195F88E3023F0100385F88E30A9E763
:100D7000002AA7D1237A062BD5D00223A372A1E79C
:100D8000002AFAD09EE7012A9CD1114628460193F9
:100D900000F022FF2846FFF715FC284602F060F815
:100DA000019B284659689A68C4F82110C4F8252088
:100DB0001A7B84F829205A7B84F82A20D3F80E1055
:100DC000D3F81220C4F83B10C4F83F20D3F81630F3
:100DD0002146C5F8A83004E0002A7FF473AF21460D
:100DE000284603B0BDE83040FFF798BE032A0CD078
:100DF000042A7FF467AF062140F20362072384F8D8
:100E00002010A4F84D20A3725CE70523A37259E7D4
:100E10002146284603B0BDE83040FFF7D1BE214649
:100E2000284600F0BFFE0146002800F08C80081D17
:100E3000019102F0F5FA01992846CB79637300F02D
:100E4000C7FE284603F05EFB284603F0DBFC0023C8
:100E50000121A372284600F0D7FE2846FFF7BAFB0F
:100E6000284602F001F895F88E3043F0100385F81B
:100E70008E3027E72146284600F094FE01460028E0
:100E80005FD0081D019102F0D5FA01992846CB796F
:100E9000637300F09DFE284603F034FB40F60D33EB
:100EA000638195F88E3023F0080385F88E3009E7CA
:100EB0002146284600F076FE0346002845D095F8E6
:100EC000302194F84E10181D1AB1D5F84021520760
:100ED0001FD4019302F0B8FA019BDA7919466273C4
:100EE000284600F075FE284603F00CFB284603F068
:100EF00089FC94F82030062B13D0242B3FF4E2AE6B
:100F000000DEDFE61A230371FEE61C3002F088FAE9
:100F1000FAE60A4694F84D10019302F0A1FA019BFB
:100F2000DBE701212846A17200F06EFE2846FFF79C
:100F300051FB284603B0BDE8304001F095BF00DE0C
:100F4000D6E600DE9DE700DE71E700DEB7E700BF12
:100F500092F81FC002F11C03ACF1030CBCF1080FA6
:100F600006D8DFE80CF01205050F0505050C090091
:100F70003D2380F8643170470822FFF78FBE0722B7
:100F8000FFF78CBE0222FFF789BE0122FFF786BE63
:100F90008B7A042B06D002D9053B082B00D870476A
:100FA00000DEFCE705238B72704700BF8B7A042BB1
:100FB00006D002D9053B082B00D8704700DEFCE7BD
:100FC000062040F20362072381F82000A1F84D209B
:100FD0008B727047887AA0F10400B0FA80F0400963
:100FE000704700BF13460022FFF758BE00B591F8C6
:100FF0002C3085B0042B11D991F82DC04FF0110E73
:10100000012281F828E043EA0C0313F0070315D10D
:1010100081F828300122104605B000BD032B09D00D
:1010200091F82DC0BCF1040FE8D8BCF1030F01D03A
:101030000022E8E71123012281F828304B8D02922B
:1010400001930391FFF7D6FA019B029AC01A10F49C
:10105000004FE0D12823039981F82830DAE700BF58
:10106000F0B50F4683B00DF1060201A90446B0F8B1
:101070006C50B0F86E60FFF7C7FB97F82D2012BBDD
:1010800097F82C30002B5BD1B4F86C30AB420ED308
:10109000BDF806209A420AD3B4F86E30B34206D3A4
:1010A000BDF804209A4202D3002003B0F0BD012015
:1010B00094F8D130A4F86C500343A4F86E6084F81F
:1010C000D13003B0F0BD94F93700002802DB97F867
:1010D0002C30EBB194F8761094F8685001F00303CB
:1010E0002B440D33DB00C1F34001CB409BB2B3F581
:1010F000A47F38BF4FF4A473BDF806509D4228BFAB
:101100001D4612B3002803DA97F82C30002BBBD011
:1011100094F8772094F86A1002F003030B440D331F
:10112000DB00C2F34002D3409BB2B3F5A47F38BFCB
:101130004FF4A473BDF804609E4228BF1E46A3E787
:1011400094F937009042C5DAE2E797F82C30002B8B
:101150009AD0904298DADBE710B500230C468969F3
:10116000A36131B394F82130DB071DD50B792E2B09
:101170001DD11D230B71838CCB8094F828300B7705
:1011800090F87730C3F302038B7790F87630C3F38F
:1011900002034B770868FBF7F7FB94F8213023F044
:1011A000010384F8213010BD01230B71F2E700DE4A
:1011B000DFE700DED6E700BF10B591F821200C462E
:1011C00092074B6A82B003D4CBB101221A710AE0B4
:1011D000BBB103221A71828C03F11C01DA800193E6
:1011E00002F092FA019B19461868FBF7CDFB00222A
:1011F00094F82130626223F0020384F8213002B0B7
:1012000010BD00DEE5E700BF30B583B00C460546F3
:1012100000F0DCFC6062D8B10021627BE369172A30
:101220006361E1610AD000DE2846194600F0D0FC77
:10123000284603B0BDE8304003F064B9191D2846C4
:10124000019302F049F941F60302019B6281EBE749
:1012500000DEE1E730B5CB690C46054683B0002BD4
:1012600050D0637B162B30D195F93730002B2CDB17
:101270000022E369E261636194F8202095F89C11F3
:10128000C2F3C20262F3C50185F89C1194F82010E4
:1012900095F89C21204661F3020285F89C2194F880
:1012A000202095F87610C2F3801262F3C30185F80E
:1012B0007610191D019302F0EBF80221284600F088
:1012C0008BFC0222019BA27212E000F077FC18B99D
:1012D0000723A37203B030BD00F078FC606298B1C0
:1012E0000021627BE369162A6361E161C4D000DEFC
:1012F0002846194600F06CFC284603B0BDE8304093
:1013000001F0B6BD00DEACE700DEE9E738B5054622
:101310000C4601F09DFD10B10123A37238BD284693
:1013200003F0DEF80028F7D12146284600F032FC11
:101330000028F1D0284603F0D1F80728ECD0284641
:10134000012103F0C5F828460D2103F0C5F8162346
:1013500021466373284600F025FC0346E3612146DD
:101360002846BDE83840FFF775BF00BF38B50546D1
:101370000C4603F0BFF810B10223A37238BD21461A
:10138000284600F007FC0028F6D0284603F0A6F80F
:101390000728F1D00D21284603F09EF81723214697
:1013A0002846637300F0FEFBE06158B100F006FCD4
:1013B00010B90723A37238BD21462846BDE838403E
:1013C000FFF722BF00DEF1E770B50646887A0C46CB
:1013D00084B0092806D8DFE800F0080D4B4E05055B
:1013E0007393A0C400DE04B070BD002AFBD10123BA
:1013F000A372F8E719462046019202F05FF894F8CC
:10140000201096F89C31C1F3C20CC3F3C20000EA6D
:101410000C00C1F3020C03EA0C0343EAC00321F001
:101420003F010B4384F8203096F93730019A002BA6
:101430000BDB94F8203013F0380F40F0A78094F8BD
:10144000203023F03F0384F82030022130460192FF
:1014500000F0C2FB019A012AC5D196F83730DB09AA
:10146000C0D02146304604B0BDE87040FFF77EBFD3
:10147000002AB8D1F5E7022AB5D196F93730002B0A
:1014800080F2C980664B94F820C093E8030096F878
:101490007630CDE902011A4643EA0C0303F0070354
:1014A0006B4493F808C03046062302216CF3061201
:1014B00086F87620A37204B0BDE8704000F0A4BBAB
:1014C000032A90D11946204602F01CF821463046E6
:1014D000FFF78CFD0546204600F0A2FB002D60D0F2
:1014E00094F8283096F87620282B08BF86F86431C7
:1014F0001346092162F3061386F87630A17272E76B
:10150000002A7FF470AFE369002B79D000F056FB1E
:1015100000283FD10723A37265E7002A7FF463AF59
:1015200030460192FFF75EF8638DC01A03043FF561
:101530005AAF019A84F8282096F93730002B36DB11
:10154000002294F82130092162F3000384F821304D
:1015500096F87620134662F3061386F87630A17269
:1015600041E7042A7FF43FAF21463046FFF7F4FD00
:1015700021463046FFF720FE304603F043F90021B4
:10158000304602F0A9FF0023A3722CE759077FF42D
:101590005CAF54E72146304604B0BDE87040FFF729
:1015A00033BE304602F0B4FF0823A3721BE794F861
:1015B0002D1096F8772094F82C3011F0030102F0EA
:1015C000070C03F003031DD096F87600864661F3FE
:1015D000020E00F0070086F876E0F3B163F3020232
:1015E000884286F8772013D021463046FFF738FD31
:1015F00094F82130012260F3410384F82130A0E700
:1016000000DE83E7002B9BD063F3020286F877208D
:101610006345E9D194E700DE34E78842E4D18FE7FF
:101620006C49020070B5D37F0546112B0C4602F1C0
:101630001C0625D0182B09D0072B10D0242380F8A6
:10164000643101F0DBFC0023A37270BD8B7A062BA2
:101650003FD088BF073B022BF7D900DE70BD8B7AE5
:10166000062BF6D1002102F033FF1A22D5F84031C3
:10167000204623F48073C5F8403184F828200FE019
:101680008B7A062BE5D13146204601F0F9FE94F81D
:101690004E302846002184F8283002F019FF2046F9
:1016A00000F0BEFA94F821304FF0090C43F001032A
:1016B00084F8213095F876202846134662F3061305
:1016C00085F8763084F80AC00221BDE8704000F049
:1016D0009BBA90F93730002B3FDA0221284602F0FE
:1016E000F7FE3146204601F00DFF21462846FFF760
:1016F0007DFC0646204600F093FA9EB994F82D3002
:101700002BB195F8762063F3061285F876202846EB
:1017100001F0B8FB0823A3722846BDE870400221FF
:1017200000F072BA0021284602F0D2FE94F8283068
:101730000BB185F8643194F8203094F82120DB094E
:1017400063F3000284F8212095F8761009230A46F5
:1017500061F3061285F87620DDE700DEBDE700BF05
:101760008B7A092B09D8DFE803F00606050808087C
:10177000050A0C057047FFF7C9BD00DE7047FFF78B
:1017800069BD70B582B0019104460546FEF72AFF97
:10179000019B598D401A020401D502B070BD94F925
:1017A000371000291DDB00212846019302F090FE2E
:1017B0000020019B93F8201083F82800C90993F8B2
:1017C00021004FF0090C61F3000083F8210095F827
:1017D0007600014660F3061185F8761083F80AC09A
:1017E000DBE793F82DC094F8770093F82C101CF0E9
:1017F000030C00F0070601F0030126D094F876E010
:1018000072466CF302020EF0070E84F8762029B3BC
:1018100061F30200E64584F877001CD0194628469B
:101820000193FFF71DFC019B002193F821C060F399
:10183000410C83F821C02846019302F049FE0020A4
:10184000019B012183F82800B9E70029ABD061F39F
:10185000020085F87700B142E0D1A4E7E645DDD18A
:10186000A1E700BF8B7A022B06D000D87047063B59
:10187000032BFBD900DE70470A4690F837108446E8
:10188000C909F7D030B59CF8761092F820E00D46E3
:101890000D4883B041EA0E0E03C8CDE90001284689
:1018A0000EF0070EEE4419469EF8003063F3061062
:1018B0008CF8760041F606036046538103B0BDE81C
:1018C000304000F0A1B900BF6C49020038B58B7AF6
:1018D000082B04D8033B022B00D800DE38BD092BAF
:1018E000FBD104460D46FFF737FC29462046FFF79B
:1018F00063FC204601F082FB0021204602F0ECFD53
:101900000023AB7238BD00BF92F81FC002F11C0368
:10191000BCF1160F12D0BCF1180F0CD010B582B06C
:101920000191242180F8641102F06CFF0022019BD8
:101930009A7202B010BD0322FFF746BD0122FFF7E5
:1019400043BD00BF13460022FFF73EBD13460222EF
:10195000FFF73ABD00230422FFF736BD0023C0E99C
:101960000133C0E903330370704700BF03780133CC
:1019700003707047037823B1013BDBB2037003B1FE
:101980007047C368002BFBD002691AB1816829B186
:101990000B6082600023C0E9033370474360F8E7BF
:1019A00003783BB100230C300B60436843B11960EE
:1019B00041607047002304300B604368002BF6D170
:1019C000C0E90011704700BF00230B60836813B1AA
:1019D000196081607047C0E9011170474068704725
:1019E00043682BB181681A688B42426008BF8260ED
:1019F000184670474078A0F10C00B0FA80F040091A
:101A0000704700BF4078A0F10800B0FA80F04009AC
:101A1000704700BF4078A0F10200B0FA80F04009A2
:101A2000704700BF4078A0F11700B0FA80F040097D
:101A3000704700BF4078A0F10100B0FA80F0400983
:101A4000704700BF4078A0F10900B0FA80F040096B
:101A5000704700BF4078A0F10600B0FA80F040095E
:101A6000704700BF4078A0F11800B0FA80F040093C
:101A7000704700BF4078A0F10300B0FA80F0400941
:101A8000704700BF4078A0F10500B0FA80F040092F
:101A9000704700BF30B5054683B008460C46F8F7DE
:101AA000F1FE034690B10021446005722C22C3E987
:101AB00005112030019311F0E9FE4FF47F42FF2021
:101AC0000021019B99735A8158729A81184603B07C
:101AD00030BD00BF4078A0F10200B0FA80F04009AC
:101AE000704700BF4078A0F10200B0FA80F04009D2
:101AF000704700BF4078A0F10200B0FA80F04009C2
:101B0000704700BF4078A0F10100B0FA80F04009B2
:101B1000704700BF4078A0F10100B0FA80F04009A2
:101B2000704700BF4078A0F10100B0FA80F0400992
:101B3000704700BF4078A0F10900B0FA80F040097A
:101B4000704700BF4078A0F10900B0FA80F040096A
:101B5000704700BF4078A0F11800B0FA80F040094B
:101B6000704700BF4078A0F10300B0FA80F0400950
:101B7000704700BF4078A0F10300B0FA80F0400940
:101B8000704700BF416809B1F8F790BE00DE4168B8
:101B9000F8F78CBE024B1868003818BF0120704758
:101BA0001805002010B50448F8F76CFE0446043010
:101BB000FEF706FD204610BD1805002008B50120DF
:101BC000FAF7F6FE003818BF012008BDFAF70ABF81
:101BD000E030FFF7F9BE00BF90F8562103461AB176
:101BE000114380F85611704700B5E03083B0019181
:101BF0000093FFF7BBFE009B019993F85621114318
:101C000083F8561103B000BD90F8563123EA010164
:101C100080F8561101B17047E030FFF7ABBE00BF4E
:101C2000836943B11A792E2A04D02E221A7183694E
:101C300002691A60704700DE8369F3E783694BB17C
:101C40001A792E2A00D0704701221A71816908681A
:101C5000FAF79ABE00DE8369F2E700BF8B6913B121
:101C60001A792E2A0BD00B7A072B16D0CB692BB101
:101C7000D0F85C211A60CB69C0F85C317047012252
:101C80001B68D0F858C1C3F804C08B691A718B69FE
:101C9000C0F858310B7A072BE8D14B6A002BE5D0FE
:101CA00001221B68D0F858C1C3F804C04B6A1A71EE
:101CB0004B6AC0F85831D9E710B5044682B00E48D7
:101CC000F8F7E0FD0346A0B100210B48C3E9051178
:101CD00058602C221C7203F12000019311F0D6FDF4
:101CE0004FF47F42FF200021019B99735A81587263
:101CF0009A81184602B010BD0805002010B50A4BA5
:101D0000062258685021F8F797FD084B01225868C1
:101D10005021F8F791FDBDE81040054B04222C211D
:101D20005868F8F789BD00BF10050020080500209D
:101D30001805002038B50446002501F029F9204691
:101D4000C4E93E5584F8045102F03EFDC4F8285120
:101D5000C4E9425584F81651A4F81451A4F8185156
:101D6000C4F82B51A4F84851C4F83051C4F8345188
:101D7000C4F83851C4F83C51C4F84051C4F8445137
:101D8000FAF7FEF894F88E30C4E95001C4E95655CC
:101D900023F0180384F88E3084F85651258638BD18
:101DA00008460149F8F782BD18050020B0F8023155
:101DB000844623B199420ED25B1AA0F80231BCF8D6
:101DC000123123B1994217D25B1AACF812310023B9
:101DD00018461370704700B583B0019200F0E0FF21
:101DE000019A034688B1197A0A2909D022236FF093
:101DF0007300137003B000BD22236FF07300E8E797
:101E00006FF0730093F82030F3E700DEEBE700BFDC
:101E1000034BCB18B3FBF1F3A0F81831704700BFA8
:101E2000FF59620200B583B0019002F0D5FC019821
:101E300003B05DF804EB01F0B3B800BF00B583B0A8
:101E400061B1012901D003B000BD019002F00EFD87
:101E5000019803B05DF804EB01F008B9019002F0BD
:101E6000F1FC019803B05DF804EB01F0F1B800BF9C
:101E700038B5D0F85841054634B120682146446849
:101E8000FAF776FD002CF8D12346D5F85C41C5F869
:101E9000583134B1204624680349F8F707FD002C77
:101EA000F8D1C5F85C4138BD1805002090F93730ED
:101EB000002B14DA70B50C4606460A490320154675
:101EC000FFF7E8FD014640B1304681F8204081F837
:101ED000215000F02FFF002070BD0C2070BD0C20A1
:101EE000704700BF1005002010B5074904460120C7
:101EF000FFF7D0FD28B10146204600F01BFF00206F
:101F000010BD0C2010BD00BF1005002038B50546DF
:101F10000C4602200849FFF7BDFD58B1014690F874
:101F20002030284664F3000381F8203000F002FFDF
:101F3000002038BD0C2038BD1005002010B5074921
:101F400004460420FFF7A6FD28B10146204600F014
:101F5000F1FE002010BD0C2010BD00BF10050020B8
:101F600070B5064682B00D4607201149CDE9003212
:101F70009DF81840FFF78EFDB0B10146009B019A15
:101F8000DB0005F0070003F03803920102F0400285
:101F90000343134343EAC413304681F8203000F072
:101FA000C9FE002002B070BD0C2002B070BD00BFA1
:101FB0001005002038B504460D4601F09BF8204678
